:020000040800F2
:1000000000060020E1010008E3010008E301000808
:10001000E3010008E3010008E3010008E301000830
:10002000E3010008E3010008E3010008752F000860
:10003000E3010008E3010008E3010008E301000810
:10004000E3010008E3010008E3010008E301000800
:10005000E3010008E30100081D32000845320008F2
:100060006D32000895320008BD320008E301000837
:10007000E3010008E3010008E3010008E3010008D0
:10008000E3010008E3010008E3010008E3010008C0
:10009000E3010008E3010008E3010008E53200087D
:1000A000E3010008E3010008E3010008E3010008A0
:1000B000B9330008E3010008E3010008E301000888
:1000C000E3010008E3010008E3010008E301000880
:1000D000E3010008E3010008E3010008E301000870
:1000E00049330008E3010008E3010008E3010008C8
:1000F000E3010008E3010008E3010008E301000850
:10010000E3010008E3010008E3010008E30100083F
:10011000E3010008E3010008E3010008E30100082F
:10012000E3010008E3010008E3010008E30100081F
:10013000E3010008E3010008E3010008E30100080F
:10014000E3010008E3010008E30100082927000893
:10015000E3010008E3010008E3010008E3010008EF
:10016000E3010008E3010008E3010008E3010008DF
:10017000E3010008E3010008E3010008E3010008CF
:10018000E3010008E3010008E3010008E3010008BF
:10019000E3010008E3010008E3010008E3010008AF
:1001A000E3010008E3010008E3010008E30100089F
:1001B000E3010008E3010008E3010008E30100088F
:1001C000E3010008E3010008E3010008E30100087F
:1001D000E3010008E3010008E3010008E30100086F
:1001E00002E000F000F8FEE772B6374880F30888B6
:1001F000364880F3098836483649086040F20000E6
:10020000CCF200004EF63471CEF200010860BFF36C
:100210004F8FBFF36F8F40F20000C0F2F0004EF638
:100220008851CEF200010860BFF34F8FBFF36F8F8C
:100230004FF00000E1EE100A4EF63C71CEF20001E4
:100240000860062080F31488BFF36F8F01F034FF3D
:1002500002F02EFE4FF055301F491B4A91423CBF21
:1002600041F8040BFAE71D49184A91423CBF41F896
:10027000040BFAE71A491B4A1B4B9A423EBF51F83E
:10028000040B42F8040BF8E700201849184A914281
:100290003CBF41F8040BFAE701F012FF02F05CFEEC
:1002A000144C154DAC4203DA54F8041B8847F9E7A7
:1002B00000F042F8114C124DAC4203DA54F8041B22
:1002C0008847F9E701F0FABE00060020002200206E
:1002D0000000000808ED00E00000002000060020FB
:1002E0008837000800220020402200204022002001
:1002F000602E0020E0010008E0010008E001000895
:10030000E00100082DE9F04F2DED108AC1F80CD066
:10031000C3689D46BDEC108ABDE8F08F002383F3CF
:1003200011882846A047002001F074FAFEE701F08A
:1003300003FA00DFFEE7000038B500F0BFFB01F074
:100340008BFE054601F0AEFE0446C8B90E4B9D4239
:1003500018D001339D4218BF044641F2883504BFCE
:1003600001240025002001F081FE0CB100F074F89A
:1003700000F002FD284600F0C3F800F06DF8F9E740
:100380000025EFE70546EDE7010007B008B500F0EE
:1003900067FBA0F120035842584108BD07B541F260
:1003A0001203022101A8ADF8043000F077FB03B07E
:1003B0005DF804FB38B5302383F3118817480368D0
:1003C0000BB101F0F3FA164A144800234FF47A7186
:1003D00001F0E2FA002383F31188124C236813B171
:1003E0002368013B2360636813B16368013B63606A
:1003F0000D4D2B7833B963687BB9022000F026FCE1
:10040000322363602B78032B07D163682BB902205A
:1004100000F01CFC4FF47A73636038BD402200206A
:10042000B50300086023002058220020084B1870F4
:1004300003280CD8DFE800F008050208022000F0CD
:10044000FDBB022000F0F0BB024B00225A60704757
:100450005822002060230020244B254A10B51C465A
:100460001968013140D004339342F9D16268214BBD
:100470009A4239D9204B9B6803F1006303F580331E
:100480009A4231D2002000F033FB0220FFF7CEFF6A
:100490001A4B1A6C00221A64196E1A66196E596C7E
:1004A0005A64596E5A665A6E5A6942F080025A610D
:1004B0005A6922F080025A615A691A6942F0005260
:1004C0001A611A6922F000521A611B6972B64FF064
:1004D000E0233021C3F8084DD4E9003281F31188BC
:1004E0009D4683F30888104710BD00BF0000010837
:1004F00020000108FFFF0008002200200038024011
:100500002DE9F04F93B0AA4B00902022FF210AA8BA
:100510009D6800F0DBFBA74A1378A3B9A648012128
:1005200003601170302383F3118803680BB101F06D
:100530003DFAA24AA04800234FF47A7101F02CFA48
:10054000002383F31188009B13B19D4B009A1A601E
:100550009C4A009C1378032B1EBF00231370984AFB
:100560004FF0000A18BF5360D3465646D1460120CB
:1005700000F064FB24B1924B1B68002B00F0118249
:10058000002000F06DFA0390039B002BF2DB0120AA
:1005900000F04AFB039B213B162BE8D801A252F83E
:1005A00023F000BF0106000829060008BD06000868
:1005B0006F0500086F0500086F0500084707000871
:1005C000170900083108000893080008BB08000854
:1005D000E10800086F050008F30800086F0500082F
:1005E00065090008A10600086F050008A9090008B0
:1005F0000D060008A10600086F0500089308000812
:100600000220FFF7C3FE002840F0F581009B022185
:10061000BAF1000F08BF1C4605A841F21233ADF82D
:10062000143000F03BFAA2E74FF47A7000F018FAA9
:10063000071EEBDB0220FFF7A9FE0028E6D0013FF2
:10064000052F00F2DA81DFE807F0030A0D101336F8
:1006500005230593042105A800F020FA17E054486B
:100660000421F9E758480421F6E758480421F3E744
:100670004FF01C08404600F03DFA08F104080590D0
:10068000042105A800F00AFAB8F12C0FF2D10120DC
:1006900000FA07F747EA0B0B5FFA8BFB4FF00009F4
:1006A00000F060FB26B10BF00B030B2B08BF0024FE
:1006B000FFF774FE5BE746480421CDE7002EA5D086
:1006C0000BF00B030B2BA1D10220FFF75FFE0746B7
:1006D00000289BD0012000F00BFA0220FFF7A6FEB5
:1006E00000261FFA86F8404600F012FA044690B140
:1006F0000021404600F01CFA01360028F1D1BA462C
:10070000044641F21213022105A8ADF814303E460A
:1007100000F0C4F92BE70120FFF788FE2546244BA3
:100720009B68AB4207D9284600F0E4F9013040F05D
:1007300067810435F3E7234B00251D70204BBA4633
:100740005D603E46ACE7002E3FF460AF0BF00B035C
:100750000B2B7FF45BAF0220FFF768FE322000F026
:100760007FF9B0F10008FFF651AF18F003077FF4EE
:100770004DAF0F4A926808EB050393423FF646AF30
:10078000B8F5807F3FF742AF124B0193B84523DDA8
:100790004FF47A7000F064F90390039A002AFFF690
:1007A00035AF019B039A03F8012B0137EDE700BF3A
:1007B000002200205C23002040220020B503000816
:1007C000602300205822002004220020082200205C
:1007D0000C2200205C220020C820FFF7D7FD07462E
:1007E00000283FF413AF1F2D11D8C5F12002424558
:1007F0000AAB25F0030028BF424683490192184402
:1008000000F03EFA019A8048FF2100F05FFA4FEABB
:10081000A8037D490193C8F38702284600F05EFAD9
:10082000064600283FF46DAF019B05EB830537E7D3
:100830000220FFF7ABFD00283FF4E8AE00F0A4F97A
:1008400000283FF4E3AE0027B846704B9B68BB42DC
:1008500018D91F2F11D80A9B01330ED027F003039C
:1008600012AA134453F8203C05934046042205A9DC
:1008700000F0ACFA04378046E7E7384600F03AF972
:100880000590F2E7CDF81480042105A800F006F9E0
:1008900006E70023642104A8049300F0F5F800287B
:1008A0007FF4B4AE0220FFF771FD00283FF4AEAE36
:1008B000049800F051F90590E6E70023642104A8AC
:1008C000049300F0E1F800287FF4A0AE0220FFF7C7
:1008D0005DFD00283FF49AAE049800F04DF9EAE778
:1008E0000220FFF753FD00283FF490AE00F05CF9C2
:1008F000E1E70220FFF74AFD00283FF487AE05A993
:10090000142000F057F904210746049004A800F0D1
:10091000C5F83946B9E7322000F0A2F8071EFFF605
:1009200075AEBB077FF472AE384A926807EB0903D5
:1009300093423FF66BAE0220FFF728FD00283FF4FC
:1009400065AE27F003074F44B9453FF4A9AE4846CA
:1009500000F0D0F80421059005A800F09FF809F1F7
:100960000409F1E74FF47A70FFF710FD00283FF417
:100970004DAE00F009F9002844D00A9B01330BD09A
:1009800008220AA9002000F0A9F900283AD0202264
:10099000FF210AA800F09AF9FFF700FD1C4800F0BB
:1009A0003FFF13B0BDE8F08F002E3FF42FAE0BF0E9
:1009B0000B030B2B7FF42AAE0023642105A80593BB
:1009C00000F062F8074600287FF420AE0220FFF70F
:1009D000DDFC804600283FF419AEFFF7DFFC41F252
:1009E000883000F01DFF059800F0EEF9464600F053
:1009F000B9F93C46BBE5064652E64FF0000905E66C
:100A0000BA467EE637467CE65C22002000220020C3
:100A1000A086010070B50F4B1B780133DBB2012BB0
:100A20000C4611D80C4D29684FF47A730E6AA2FB5C
:100A30000332014622462846B047844204D1074B80
:100A400000221A70012070BD4FF4FA7000F0E8FE29
:100A50000020F8E710220020082600209423002020
:100A600007B50023024601210DF107008DF807307C
:100A7000FFF7D0FF20B19DF8070003B05DF804FB3D
:100A80004FF0FF30F9E700000A4608B50421FFF7F0
:100A9000C1FF80F00100C0B2404208BD30B4054C37
:100AA0002368DD69044B0A46AC460146204630BC4B
:100AB000604700BF08260020A086010070B501F045
:100AC000D1F9094E094D30800024286833888342CB
:100AD00008D901F0C1F92B6804440133B4F5803F13
:100AE0002B60F2D370BD00BF962300206823002046
:100AF00001F066BA00F1006000F5803000687047D0
:100B000000F10060920000F5803001F0F1B90000C2
:100B1000054B1A68054B1B889B1A834202D9104467
:100B200001F09AB900207047682300209623002026
:100B300038B5084D044629B128682044BDE838403E
:100B400001F0AAB92868204401F08EF90028F3D0FA
:100B500038BD00BF6823002010F003030AD1B0F5B0
:100B6000047F05D200F10050A0F51040D0F8003805
:100B7000184670470023FBE700F10050A0F5104035
:100B8000D0F8100A70470000064991F8243033B1BC
:100B90000023086A81F824300822FFF7B1BF012042
:100BA000704700BF6C230020014B1868704700BFDE
:100BB000002004E070B5194B1D68194B0138C5F3CE
:100BC0000B0408442D0C04221E88A6420BD15C683D
:100BD0000A46013C824213460FD214F9016F4EB10E
:100BE00002F8016BF6E7013A03F10803ECD1814208
:100BF0000B4602D22C2203F8012B0A4A0524168840
:100C0000AE4204D1984284BF967803F8016B013C50
:100C100002F10402F3D1581A70BD00BF002004E0B5
:100C20009C34000888340008022802BF024B4FF4AD
:100C300000129A61704700BF00040240022802BF00
:100C4000014B20229A61704700040240022801BF34
:100C5000024A536983F02003536170470004024045
:100C600070B504464FF47A764CB1412C254628BF26
:100C7000412506FB05F000F0D3FD641BF4E770BDD1
:100C800010B50023934203D0CC5CC4540133F9E780
:100C900010BD000010B5013810F9013F3BB191F9CA
:100CA00000409C4203D11AB10131013AF4E71AB174
:100CB00091F90020981A10BD1046FCE70346024641
:100CC000D01A12F9011B0029FAD1704702440346D9
:100CD000934202D003F8011BFAE770472DE9F8436D
:100CE0001F4D144695F824200746884652BBDFF86E
:100CF00070909CB395F824302BB92022FF214846F0
:100D00002F62FFF7E3FF95F82400C0F10802A2422A
:100D100028BF2246D6B24146920005EB8000FFF77D
:100D2000AFFF95F82430A41B1E44F6B2082E1744DA
:100D30009044E4B285F82460DBD1FFF725FF00285A
:100D4000D7D108E02B6A03EB82038342CFD0FFF7B1
:100D50001BFF0028CBD10020BDE8F8830120FBE772
:100D60006C230020024B1A78024B1A70704700BFA8
:100D7000942300201022002010B5104C104800F0E1
:100D8000B5F821460E4800F0DDF82468626DD2F80F
:100D9000043843F00203C2F804384FF47A70FFF7C6
:100DA0005FFF0849204600F0D3F9626DD2F804389D
:100DB00023F00203C2F8043810BD00BF68350008F4
:100DC00008260020703500087047000030B5094D36
:100DD0000A4491420DD011F8013B5840082340F3DA
:100DE0000004013B2C4013F0FF0384EA5000F6D1CD
:100DF000EFE730BD2083B8ED02684368114301601E
:100E000003B118477047000013B5446BD4F894340D
:100E10001A681178042915D1217C022912D1197977
:100E2000128901238B4013420CD101A904F14C001B
:100E300001F0FAFED4F89444019B2179024620681F
:100E400000F0D0F902B010BD143001F07DBE0000FA
:100E50004FF0FF33143001F077BE00004C3001F04A
:100E60004FBF00004FF0FF334C3001F049BF00008E
:100E7000143001F04BBE00004FF0FF31143001F090
:100E800045BE00004C3001F01BBF00004FF0FF32A8
:100E90004C3001F015BF00000020704710B5D0F8AD
:100EA00094341A6811780429044617D1017C022968
:100EB00014D15979528901238B4013420ED1143039
:100EC00001F0DEFD024648B1D4F894444FF480733B
:100ED00061792068BDE8104000F072B910BD0000D3
:100EE000406BFFF7DBBF0000704700007FB5124B7F
:100EF000036000234360C0E90233012502260F4B43
:100F0000057404460290019300F18402294600967C
:100F10004FF48073143001F08FFD094B0294CDE93A
:100F2000006304F523724FF48073294604F14C00EA
:100F300001F056FE04B070BDBC340008E10E00089C
:100F4000090E00080B68302282F311880A7903EB3E
:100F5000820290614A79093243F822008A7912B1FB
:100F600003EB820398610223C0F8941403740020F9
:100F700080F311887047000038B5037F044613B131
:100F800090F85430ABB9201D01250221FFF734FF42
:100F900004F1140025776FF0010100F069FC84F87A
:100FA000545004F14C006FF00101BDE8384000F0EE
:100FB0005FBC38BD10B5012104460430FFF71CFFAB
:100FC0000023237784F8543010BD000038B5044660
:100FD0000025143001F048FD04F14C00257701F0A4
:100FE00017FE201D84F854500121FFF705FF20460D
:100FF000BDE83840FFF752BF90F8443003F060037B
:10100000202B07D190F84520212A4FF0000303D868
:101010001F2A06D800207047222AFBD1C0E90E33D0
:1010200003E0034A82630722C2630364012070471E
:101030001122002037B5D0F894341A6811780429A9
:1010400004461AD1017C022917D11979128901238A
:101050008B40134211D100F14C05284601F098FE57
:1010600058B101A9284601F0DFFDD4F89444019B52
:1010700021790246206800F0B5F803B030BD0000C9
:10108000F0B500EB810385B09E6904460D46FEB1C4
:10109000302383F3118804EB8507301D0821FFF707
:1010A000ABFEFB685B691B6806F14C001BB101904D
:1010B00001F0C8FD019803A901F0B6FD024648B150
:1010C000039B2946204600F08DF8002383F3118806
:1010D00005B0F0BDFB685A691268002AF5D01B8A7A
:1010E000013B1340F1D104F14402EAE7093138B57C
:1010F00050F82140DCB1302383F31188D4F89424D4
:101100001368527903EB8203DB689B695D6845B124
:1011100004216018FFF770FE294604F1140001F065
:10112000B9FC2046FFF7BAFE002383F3118838BDCF
:101130007047000001F018B8012303700023C0E9D4
:101140000133C36183620362C36243620363704716
:1011500038B50446302383F311880025C0E90355D0
:10116000C0E90555416001F00FF80223237085F3B3
:101170001188284638BD000070B500EB8103054694
:101180005069DA600E46144618B110220021FFF7AC
:101190009DFDA06918B110220021FFF797FD31468F
:1011A0002846BDE8704001F0B9B80000826802F03E
:1011B000011282600022C0E90422826101F03AB982
:1011C000F0B400EB81044789E4680125A4698D40EF
:1011D0003D43458123600023A2606360F0BC01F0C1
:1011E00055B90000F0B400EB81040789E4680125DB
:1011F00064698D403D43058123600023A2606360E4
:10120000F0BC01F0CFB9000070B502230025044600
:101210000370C0E90255C0E90455C564856180F8D2
:10122000345001F017F863681B6823B12946204643
:10123000BDE87040184770BD0378052B10B5044613
:101240000AD080F850300523037043681B680BB147
:10125000042198470023A36010BD000001780529F0
:1012600006D190F85020436802701B6803B11847FC
:101270007047000070B590F83430044613B1002375
:1012800080F8343004F14402204601F0F5F8636838
:101290009B68B3B994F8443013F0600535D0002151
:1012A000204601F095FB0021204601F087FB636892
:1012B0001B6813B1062120469847062384F8343072
:1012C00070BD204698470028E4D0B4F84A30E26B5D
:1012D0009A4288BFE36394F94430E56B002B4FF0EA
:1012E000300380F20381002D00F0F280092284F89F
:1012F000342083F311880021D4E90E232046FFF720
:1013000071FF002383F31188DAE794F8452003F096
:101310007F0343EA022340F20232934200F0C58089
:1013200021D8B3F5807F48D00DD8012B3FD0022BB8
:1013300000F09380002BB2D104F14C02A263022290
:10134000E2632364C1E7B3F5817F00F09B80B3F5CE
:10135000407FA4D194F84630012BA0D1B4F84C3092
:1013600043F0020332E0B3F5006F4DD017D8B3F568
:10137000A06F31D0A3F5C063012B90D8636894F8B7
:1013800046205E6894F84710B4F848302046B047CD
:10139000002884D04368A3630368E3631AE0B3F5CD
:1013A000106F36D040F6024293427FF478AF5C4B28
:1013B000A3630223E3630023C3E794F84630012BC1
:1013C0007FF46DAFB4F84C3023F00203C4E90E553E
:1013D000A4F84C30256478E7B4F84430B3F5A06F36
:1013E0000ED194F8463084F84E30204600F08AFF43
:1013F00063681B6813B101212046984703232370BB
:101400000023C4E90E339CE704F14F03A3630123D7
:10141000C3E72378042B10D1302383F311882046AF
:10142000FFF7C4FE85F311880321636884F84F50E9
:1014300021701B680BB12046984794F84630002B6A
:10144000DED084F84F300423237063681B68002BC0
:10145000D6D0022120469847D2E794F848301D069E
:1014600003F00F0120460AD500F0F8FF012804D050
:1014700002287FF414AF2B4B9AE72B4B98E700F030
:10148000DFFFF3E794F84630002B7FF408AF94F8C1
:10149000483013F00F01B3D01A06204602D501F0F0
:1014A000ABFAADE701F09EFAAAE794F84630002BBC
:1014B0007FF4F5AE94F8483013F00F01A0D01B066E
:1014C000204602D501F084FA9AE701F077FA97E70F
:1014D000142284F8342083F311882B462A462946A7
:1014E0002046FFF76DFE85F31188E9E65DB1152210
:1014F00084F8342083F311880021D4E90E23204698
:10150000FFF75EFEFDE60B2284F8342083F311889A
:101510002B462A4629462046FFF764FEE3E700BF34
:10152000EC340008E4340008E834000838B590F8DA
:1015300034300446002B3ED0063BDAB20F2A34D8B2
:101540000F2B32D8DFE803F0373131082232313146
:101550003131313131313737C56BB0F84A309D42C6
:1015600014D2C3681B8AB5FBF3F203FB12556DB9A5
:10157000302383F311882B462A462946FFF732FE93
:1015800085F311880A2384F834300EE0142384F89C
:101590003430302383F3118800231A46194620463D
:1015A000FFF70EFE002383F3118838BD036C03B1EF
:1015B00098470023E7E70021204601F009FA0021BF
:1015C000204601F0FBF963681B6813B10621204631
:1015D00098470623D7E7000010B590F83430142B55
:1015E000044629D017D8062B05D001D81BB110BD51
:1015F000093B022BFBD80021204601F0E9F900212C
:10160000204601F0DBF963681B6813B10621204610
:101610009847062319E0152BE9D10B2380F83430C5
:10162000302383F3118800231A461946FFF7DAFDA9
:10163000002383F31188DAE7C3689B695B68002B9A
:10164000D5D1036C03B19847002384F83430CEE73A
:1016500000230375826803691B6899689142FBD275
:101660005A68036042601060586070470023037539
:10167000826803691B6899689142FBD85A680360C5
:10168000426010605860704708B50846302383F305
:1016900011880B7D032B05D0042B0DD02BB983F3C0
:1016A000118808BD8B6900221A604FF0FF338361F7
:1016B000FFF7CEFF0023F2E7D1E9003213605A6052
:1016C000F3E70000FFF7C4BF054BD9680875186839
:1016D00002681A60536001220275D860FEF712BEDC
:1016E0009823002030B50C4BDD684B1C87B00446B6
:1016F0000FD02B46094A684600F04EF92046FFF706
:10170000E3FF009B13B1684600F050F9A86907B0E9
:1017100030BDFFF7D9FFF9E79823002089160008AC
:10172000044B1A68DB6890689B68984294BF00205D
:101730000120704798230020084B10B51C68D8681A
:1017400022681A60536001222275DC60FFF78EFF69
:1017500001462046BDE81040FEF7D4BD9823002086
:1017600038B5074C074908480123002523706560F8
:1017700001F046FB0223237085F3118838BD00BFBA
:1017800000260020F43400089823002000F044B91B
:10179000034A516853685B1A9842FBD8704700BFF0
:1017A000001000E08B60022308618B8208467047BE
:1017B0008368A3F1840243F8142C026943F8442C93
:1017C000426943F8402C094A43F8242CC26843F884
:1017D000182C022203F80C2C002203F80B2C044ACC
:1017E00043F8102CA3F12000704700BF1D03000830
:1017F0009823002008B5FFF7DBFFBDE80840FFF79E
:1018000061BF0000024BDB6898610F20FFF75CBFEF
:1018100098230020302383F31188FFF7F3BF0000E3
:1018200008B50146302383F311880820FFF75AFFDB
:10183000002383F3118808BD064BDB6839B1426889
:1018400018605A60136043600420FFF74BBF4FF0ED
:10185000FF307047982300200368984206D01A682A
:101860000260506099611846FFF72CBF7047000076
:1018700038B504460D462068844200D138BD03685F
:1018800023605C608561FFF71DFFF4E710B5036816
:101890009C68A2420CD85C688A600B604C60216036
:1018A000596099688A1A9A604FF0FF33836010BDBF
:1018B0001B68121BECE700000A2938BF0A2170B52B
:1018C00004460D460A26601901F094FA01F080FAE8
:1018D000041BA54203D8751C2E460446F3E70A2EC6
:1018E00004D9BDE87040012001F0CABA70BD000003
:1018F000F8B5144B0D46D96103F1100141600A2A75
:101900001969826038BF0A22016048601861A8180E
:10191000144601F061FA0A2701F05AFA431BA34268
:10192000064606D37C1C281901F064FA2746354682
:10193000F2E70A2F04D9BDE8F840012001F0A0BA6F
:10194000F8BD00BF98230020F8B506460D4601F00B
:101950003FFA0F4A134653F8107F9F4206D12A469A
:1019600001463046BDE8F840FFF7C2BFD169BB6809
:10197000441A2C1928BF2C46A34202D92946FFF746
:101980009BFF224631460348BDE8F840FFF77EBF83
:1019900098230020A823002010B4C0E903230023CB
:1019A0005DF8044B4361FFF7CFBF000010B5194C41
:1019B000236998420DD0D0E90032816813605A60E3
:1019C0009A680A449A60002303604FF0FF33A361D2
:1019D00010BD2346026843F8102F536000220260B6
:1019E00022699A4203D1BDE8104001F0FDB9936825
:1019F00081680B44936001F0EBF92269E169926818
:101A0000441AA242E4D91144BDE81040091AFFF774
:101A100053BF00BF982300202DE9F047DFF8BC80BA
:101A200008F110072C4ED8F8105001F0D1F9D8F871
:101A30001C40AA68031B9A423ED81444D5E90032E0
:101A40004FF00009C8F81C4013605A60C5F80090B8
:101A5000D8F81030B34201D101F0C6F989F31188EA
:101A6000D5E9033128469847302383F311886B6901
:101A7000002BD8D001F0ACF96A69A0EB04094A4503
:101A800082460DD2022001F0FBF90022D8F8103076
:101A9000B34208D151462846BDE8F047FFF728BFBA
:101AA000121A2244F2E712EB090938BF4A462946C6
:101AB0003846FFF7EBFEB5E7D8F81030B34208D050
:101AC0001444211AC8F81C00A960BDE8F047FFF7CC
:101AD000F3BEBDE8F08700BFA823002098230020B4
:101AE00000207047FEE70000704700004FF0FF3015
:101AF0007047000002290CD0032904D001290748AF
:101B000018BF00207047032A05D8054800EBC20023
:101B10007047044870470020704700BFCC3500086C
:101B2000202200208035000870B59AB0054608468E
:101B300001A9144600F0C2F801A8FFF7BFF8431C42
:101B40005B00C5E900340022237003236370C6B232
:101B500001AB02341046D1B28E4204F1020401D826
:101B60001AB070BD13F8011B04F8021C04F8010C34
:101B70000132F0E708B5302383F311880348FFF7FB
:101B800059FA002383F3118808BD00BF08260020FE
:101B900090F8443003F01F02012A07D190F8452045
:101BA0000B2A03D10023C0E90E3315E003F06003D4
:101BB000202B08D1B0F848302BB990F84520212AC5
:101BC00003D81F2A04D8FFF717BA222AEBD0FAE766
:101BD000034A82630722C26303640120704700BF87
:101BE0001822002007B5052917D8DFE801F01916DB
:101BF00003191920302383F31188104A0190012121
:101C0000FFF7BAFA01980E4A0221FFF7B5FA0D481C
:101C1000FFF7DCF9002383F3118803B05DF804FBC0
:101C2000302383F311880748FFF7A6F9F2E7302342
:101C300083F311880348FFF7BDF9EBE7203500086F
:101C4000443500080826002038B50C4D0C4C0D49D1
:101C50002A4604F10800FFF767FF05F1CA0204F104
:101C600010000949FFF760FF05F5CA7204F118007A
:101C70000649BDE83840FFF757BF00BFD02A002013
:101C800020220020003500080A350008153500081C
:101C900070B5044608460D46FFF710F8C6B2204658
:101CA000013403780BB9184670BD32462946FEF759
:101CB000F1FF0028F3D10120F6E700002DE9F047FD
:101CC00005460C46FEF7FAFF2C49C6B22846FFF738
:101CD000DFFF08B10C36F6B229492846FFF7D8FFD6
:101CE00008B11036F6B2632E0BD8DFF89080DFF81B
:101CF0009090244FDFF898A02E7846B92670BDE862
:101D0000F08729462046BDE8F04701F09FBB252E0D
:101D100030D1072241462846FEF7BCFF80B91A4B56
:101D2000224603F1100153F8040B42F8040B8B42D6
:101D3000F9D119889B781180937007351334DBE74C
:101D4000082249462846FEF7A5FF98B90F4BA21C6A
:101D5000197809090232C95D02F8041C13F8011B45
:101D600001F00F015345C95D02F8031CF0D118348E
:101D70000835C1E704F8016B0135BDE7EC35000813
:101D80001535000808360008F4350008107AFF1FE2
:101D90001C7AFF1FBFF34F8F024AD368DB03FCD4CA
:101DA000704700BF003C024008B5094B1B7873B96F
:101DB000FFF7F0FF074B1A69002ABFBF064A5A60B7
:101DC00002F188325A601A6822F480621A6008BDF3
:101DD0002E2D0020003C02402301674508B50B4B27
:101DE0001B7893B9FFF7D6FF094B1A6942F00042FE
:101DF0001A611A6842F480521A601A6822F48052FA
:101E00001A601A6842F480621A6008BD2E2D002004
:101E1000003C02400B28F0B516D80C4C0C49237836
:101E20007BB90C4D0E460C234FF0006255F8047B35
:101E300046F8042B013B13F0FF033A44F6D101238B
:101E4000237051F82000F0BD0020FCE7602D002039
:101E5000302D00201C360008014B53F8200070473D
:101E60001C3600080C2070470B2810B5044601D919
:101E7000002010BDFFF7CEFF064B53F82430184466
:101E8000C21A0BB90120F4E712680132F0D1043B09
:101E9000F6E700BF1C3600080B2810B5044621D811
:101EA000FFF778FFFFF780FF0F4AF323D360C300EB
:101EB000DBB243F4007343F002031361136943F48C
:101EC00080331361FFF766FFFFF7A4FF074B53F85A
:101ED000241000F0D9F8FFF781FF2046BDE810403C
:101EE000FFF7C2BF002010BD003C02401C360008B6
:101EF000F8B512F00103144642D18218B2F1016F15
:101F000057D82D4B1B6813F0010352D02B4DFFF710
:101F10004BFFF323EB60FFF73DFF40F20127032C5B
:101F200015D824F001046618244C401A40F2011719
:101F3000B142236900EB010524D123F001032361A1
:101F4000FFF74CFF0120F8BD043C0430E7E78307AE
:101F5000E7D12B6923F440732B612B693B432B6141
:101F600051F8046B0660BFF34F8FFFF713FF036850
:101F70009E42E9D02B6923F001032B61FFF72EFF6E
:101F80000020E0E723F44073236123693B4323618E
:101F90000B882B80BFF34F8FFFF7FCFE2D8831F8A5
:101FA000023BADB2AB42C3D0236923F001032361EE
:101FB000E4E71846C7E700BF00380240003C024093
:101FC000084908B50B7828B11BB9FFF7EDFE0123CE
:101FD0000B7008BD002BFCD0BDE808400870FFF76F
:101FE000FDBE00BF2E2D002010B50244064BD2B21C
:101FF000904200D110BD441C00B253F8200041F8BB
:10200000040BE0B2F4E700BF502800400F4B30B59E
:102010001C6F240407D41C6F44F400741C671C6FED
:1020200044F400441C670A4C236843F48073236023
:102030000244084BD2B2904200D130BD441C00B2E1
:1020400051F8045B43F82050E0B2F4E70038024056
:10205000007000405028004007B5012201A900206F
:10206000FFF7C2FF019803B05DF804FB13B5044607
:10207000FFF7F2FFA04205D0012201A90020019440
:10208000FFF7C4FF02B010BD70470000034B1A6891
:102090001AB9034AD2F874281A607047642D0020D8
:1020A0000030024008B5FFF7F1FF024B1868C0F39B
:1020B000407008BD642D002070470000FEE700005E
:1020C0000A4B0B480B4A90420BD30B4BDA1C121AEB
:1020D000C11E22F003028B4238BF00220021FEF70E
:1020E000F5BD53F8041B40F8041BECE7C8370008A3
:1020F000602E0020602E0020602E002070B5D0E9F8
:1021000015439E6800224FF0FF3504EB4213510146
:10211000D3F800090028BEBFD3F8000940F0804082
:10212000C3F80009D3F8000B0028BEBFD3F8000B9A
:1021300040F08040C3F8000B013263189642C3F8A8
:102140000859C3F8085BE0D24FF00113C4F81C38FB
:1021500070BD0000890141F02001016103699B0607
:10216000FCD41220FFF714BB10B5054C2046FEF737
:10217000E3FF4FF0A0436365024BA36510BD00BFB2
:10218000682D00207036000870B50378012B0546D5
:1021900050D12A4B446D98421BD1294B5A6B42F0C7
:1021A00080025A635A6D42F080025A655A6D5A692C
:1021B00042F080025A615A6922F080025A610E216F
:1021C00043205B6900F022FC1E4BE3601E4BC4F809
:1021D00000380023C4F8003EC02323606E6D4FF426
:1021E0000413A3633369002BFCDA012333610C2051
:1021F000FFF7CEFA3369DB07FCD41220FFF7C8FAE9
:102200003369002BFCDA0026A6602846FFF776FF2C
:102210006B68C4F81068DB68C4F81468C4F81C68FC
:102220004BB90A4BA3614FF0FF336361A36843F0DE
:102230000103A36070BD064BF4E700BF682D0020CA
:10224000003802404014004003002002003C30C02F
:10225000083C30C0F8B5446D054600212046FFF724
:1022600079FFA96D00234FF001128F68C4F834384C
:102270004FF00066C4F81C284FF0FF3004EB431207
:1022800001339F42C2F80069C2F8006BC2F8080926
:10229000C2F8080BF2D20B686A6DEB65636210231B
:1022A0001361166916F01006FBD11220FFF770FAC1
:1022B000D4F8003823F4FE63C4F80038A36943F46B
:1022C000402343F01003A3610923C4F81038C4F875
:1022D00014380A4BEB604FF0C043C4F8103B084B76
:1022E000C4F8003BC4F81069C4F80039EB6D03F181
:1022F000100243F48013EA65A362F8BD4C3600086F
:1023000040800010426D90F84E10D2F8003823F44F
:10231000FE6343EA0113C2F8003870472DE9F84321
:1023200000EB8103456DDA68166806F00306731E3C
:10233000022B05EB41130C4680460FFA81F94FEA58
:1023400041104FF00001C3F8101B4FF0010104F1E0
:10235000100398BFB60401FA03F391698EBF334EA0
:1023600006F1805606F5004600293AD0578A04F156
:102370005801490137436F50D5F81C180B43C5F875
:102380001C382B180021C3F8101953690127611E4E
:10239000A7409BB3138A928B9B08012A88BF5343A3
:1023A000D8F85C20981842EA034301F1400205EB9B
:1023B0008202C8F85C00214653602846FFF7CAFE37
:1023C00008EB8900C3681B8A43EA845348346401DC
:1023D0001E432E51D5F81C381F43C5F81C78BDE8A4
:1023E000F88305EB4917D7F8001B21F40041C7F823
:1023F000001BD5F81C1821EA0303C0E704F13F03D2
:1024000005EB83030A4A5A6028462146FFF7A2FEDD
:1024100005EB4910D0F8003923F40043C0F8003927
:10242000D5F81C3823EA0707D7E700BF0080001063
:1024300000040002826D1268C265FFF75FBE0000F3
:102440005831436D49015B5813F4004004D013F434
:10245000001F0CBF02200120704700004831436D6F
:1024600049015B5813F4004004D013F4001F0CBF63
:10247000022001207047000000EB8101CB68196A3F
:102480000B6813604B6853607047000000EB8103DA
:1024900030B5DD68AA691368D36019B9402B84BFD1
:1024A000402313606B8A1468426D1C44013CB4FBEA
:1024B000F3F46343033323F0030302EB411043EAD5
:1024C000C44343F0C043C0F8103B2B6803F0030340
:1024D000012B09B20ED1D2F8083802EB411013F4E7
:1024E000807FD0F8003B14BF43F0805343F000538B
:1024F000C0F8003B02EB4112D2F8003B43F004432A
:10250000C2F8003B30BD00002DE9F041244D6E6D56
:1025100006EB40130446D3F8087BC3F8087B380762
:102520000AD5D6F81438190706D505EB84032146D9
:10253000DB6828465B689847FA071FD5D6F8143839
:10254000DB071BD505EB8403D968CCB98B69488AB6
:102550005A68B2FBF0F600FB16228AB91868DA68EE
:1025600090420DD2121AC3E90024302383F311885C
:102570000B482146FFF78AFF84F31188BDE8F081FC
:10258000012303FA04F26B8923EA02036B81CB680F
:10259000002BF3D021460248BDE8F041184700BFA8
:1025A000682D002000EB810370B5DD68436D6C6918
:1025B0002668E6604A0156BB1A444FF40020C2F870
:1025C00010092A6802F00302012A0AB20ED1D3F8D8
:1025D000080803EB421410F4807FD4F8000914BFFC
:1025E00040F0805040F00050C4F8000903EB421264
:1025F000D2F8000940F00440C2F80009D3F83408CA
:10260000012202FA01F10143C3F8341870BD19B96F
:10261000402E84BF4020206020682E8A8419013C0F
:10262000B4FBF6F440EAC44040F000501A44C6E758
:102630002DE9F8433B4D6E6D06EB40130446D3F88D
:102640000889C3F8088918F0010F4FEA40171AD01B
:10265000D6F81038DB0716D505EB8003D9684B692F
:102660001868DA68904230D2121A4FF000091A60E6
:10267000C3F80490302383F3118821462846FFF7DE
:1026800091FF89F3118818F0800F1CD0D6F83438E8
:102690000126A640334216D005EB84036D6DD3F8B6
:1026A0000CC0DCF814200134E4B2D2F800E005EBF1
:1026B00004342F445168714515D3D5F8343823EAD2
:1026C0000606C5F83468BDE8F883012303FA04F26E
:1026D0002B8923EA02032B818B68002BD3D0214660
:1026E00028469847CFE7BCF81000AEEB01038342C1
:1026F00028BF0346D7F8180980B2B3EB800FE2D8A1
:102700009068A0F1040959F8048FC4F80080A0EB88
:1027100009089844B8F1040FF5D818440B449060A8
:102720005360C7E7682D00202DE9F74FA24C656D77
:102730006E69AB691E4016F480586E6107D0204662
:10274000FEF762FD03B0BDE8F04F00F047BC002E7D
:1027500012DAD5F8003E98489B071EBFD5F8003E18
:1027600023F00303C5F8003ED5F8043823F0010335
:10277000C5F80438FEF772FD370505D58E48FFF71A
:10278000BDFC8D48FEF758FDB0040CD5D5F80838CF
:1027900013F0060FEB6823F470530CBF43F410538F
:1027A00043F4A053EB6031071BD56368DB681BB9AA
:1027B000AB6923F00803AB612378052B0CD1D5F866
:1027C000003E7D489A071EBFD5F8003E23F0030364
:1027D000C5F8003EFEF742FD6368DB680BB1764842
:1027E0009847F30274D4B70227D5D4F85490DFF891
:1027F000C8B100274FF0010A09EB4712D2F8003B9D
:1028000003F44023B3F5802F11D1D2F8003B002B05
:102810000DDA62890AFA07F322EA0303638104EB03
:102820008703DB68DB6813B1394658469847A36DC8
:1028300001379B68FFB29F42DED9F00617D5676D5E
:102840003A6AC2F30A1002F00F0302F4F012B2F572
:10285000802F00F08580B2F5402F08D104EB830370
:102860000022DB681B6A07F5805790426AD130036B
:10287000D5F8184813D5E10302D50020FFF744FE30
:10288000A20302D50120FFF73FFE630302D5022019
:10289000FFF73AFE270302D50320FFF735FE750345
:1028A0007FF550AFE00702D50020FFF7C1FEA1077A
:1028B00002D50120FFF7BCFE620702D50220FFF718
:1028C000B7FE23077FF53EAF0320FFF7B1FE39E7E0
:1028D000636DDFF8E4A0019300274FF00109A36DB9
:1028E0009B685FFA87FB9B453FF67DAF019B03EB3F
:1028F0004B13D3F8001901F44021B1F5802F1FD1FB
:10290000D3F8001900291BDAD3F8001941F09041DF
:10291000C3F80019D3F800190029FBDB5946606D94
:10292000FFF718FC218909FA0BF321EA030323813D
:1029300004EB8B03DB689B6813B1594650469847FC
:102940000137CCE7910708BFD7F80080072A98BF66
:1029500003F8018B02F1010298BF4FEA182884E7BF
:10296000023304EB830207F580575268D2F818C08F
:10297000DCF80820DCE9001CA1EB0C0C00218842EB
:102980000AD104EB830463689B699A6802449A60E5
:102990005A6802445A606AE711F0030F08BFD7F87B
:1029A00000808C4588BF02F8018B01F1010188BFCE
:1029B0004FEA1828E3E700BF682D0020436D03EBC2
:1029C0004111D1F8003B43F40013C1F8003B7047BC
:1029D000436D03EB4111D1F8003943F40013C1F802
:1029E00000397047436D03EB4111D1F8003B23F4EC
:1029F0000013C1F8003B7047436D03EB4111D1F860
:102A0000003923F40013C1F80039704700F1604326
:102A100003F561430901C9B283F80013012200F0F4
:102A20001F039A4043099B0003F1604303F5614390
:102A3000C3F880211A60704730B5039C01720433DB
:102A400004FB0325C0E90653049B03630021059B97
:102A5000C160C0E90000C0E90422C0E90842C0E941
:102A60000A11436330BD0000416A0022C0E904112D
:102A7000C0E90A22C2606FF00101FEF7F9BE000052
:102A8000D0E90432934201D1C2680AB9181D7047D7
:102A90000020704703691960C2680132C260C269D0
:102AA000134482690361934224BF436A0361002196
:102AB000FEF7D2BE38B504460D46E3683BB1626905
:102AC000131D1268A3621344E362002007E0237A17
:102AD00033B929462046FEF7AFFE0028EDDA38BDAF
:102AE0006FF00100FBE70000C368C269013BC360EF
:102AF0004369134482694361934224BF436A43613B
:102B000000238362036B03B11847704770B530230D
:102B1000044683F31188866A3EB9FFF7CBFF05466A
:102B200018B186F31188284670BDA36AE26A13F8CB
:102B3000015BA362934202D32046FFF7D5FF002337
:102B400083F31188EFE700002DE9F84F04460E46A5
:102B5000174698464FF0300989F311880025AA4698
:102B6000D4F828B0BBF1000F09D141462046FFF749
:102B7000A1FF20B18BF311882846BDE8F88FD4E976
:102B80000A12A7EB050B521A934528BF9346BBF1D7
:102B9000400F1BD9334601F1400251F8040B43F8B2
:102BA000040B9142F9D1A36A40334036A362403509
:102BB000D4E90A239A4202D32046FFF795FF8AF30D
:102BC0001188BD42D8D289F31188C9E730465A46E8
:102BD000FEF756F8A36A5B445E44A3625D44E7E7F0
:102BE00010B5029C0172043303FB0421C0E90613F3
:102BF0000023C0E90A33039B0363049BC460C0E95C
:102C00000000C0E90422C0E90842436310BD00008F
:102C1000026AC260426AC0E904220022C0E90A22B4
:102C20006FF00101FEF724BED0E904239A4201D1DE
:102C3000C26822B9184650F8043B0B607047002365
:102C40001846FAE7C368C2690133C3604369134495
:102C500082694361934224BF436A43610021FEF7C6
:102C6000FBBD000038B504460D46E3683BB123695F
:102C70001A1DA262E2691344E362002007E0237A8E
:102C800033B929462046FEF7D7FD0028EDDA38BDD6
:102C90006FF00100FBE7000003691960C268013AA8
:102CA000C260C269134482690361934224BF436ACC
:102CB000036100238362036B03B118477047000070
:102CC00070B530230D460446114683F31188866A99
:102CD0002EB9FFF7C7FF10B186F3118870BDA36A44
:102CE0001D70A36AE26A01339342A36204D3E169CF
:102CF00020460439FFF7D0FF002080F31188EDE76C
:102D00002DE9F84F04460D46904699464FF0300A9B
:102D10008AF311880026B346A76A4FB94946204670
:102D2000FFF7A0FF20B187F311883046BDE8F88F88
:102D3000D4E90A073A1AA8EB0607974228BF1746B4
:102D4000402F1BD905F1400355F8042B40F8042B04
:102D50009D42F9D1A36A4033A3624036D4E90A23E5
:102D60009A4204D3E16920460439FFF795FF8BF3BB
:102D700011884645D9D28AF31188CDE729463A46CB
:102D8000FDF77EFFA36A3B443D44A3623E44E5E772
:102D9000D0E904239A4217D1C3689BB1836A8BB1EF
:102DA000043B9B1A0ED01360C368013BC360C36928
:102DB0001A44836902619A4224BF436A0361002373
:102DC00083620123184670470023FBE700F030B907
:102DD0004FF08043586A70474FF080430022586399
:102DE0001A610222DA6070474FF080430022DA60F5
:102DF000704700004FF0804358637047FEE70000C3
:102E000070B51B4B01630025044686B0586085628F
:102E10000E4600F0BFF804F11003C4E904334FF08C
:102E2000FF33C4E90635C4E90044A560E562FFF755
:102E3000CFFF2B460246C4E9082304F134010D4AB2
:102E4000256580232046FEF7ADFC0123E0600A4A99
:102E50000375009272680192B268CDE90223074BB4
:102E60006846CDE90435FEF7C5FC06B070BD00BF6D
:102E7000002600207C36000881360008FD2D000861
:102E8000024AD36A1843D062704700BF98230020DB
:102E90004B6843608B688360CB68C3600B69436198
:102EA0004B6903628B6943620B68036070470000E3
:102EB00008B5264B26481A6940F2FF110A431A61E9
:102EC0001A6922F4FF7222F001021A611A691A6B60
:102ED0000A431A631A6D0A431A651E4A1B6D11468E
:102EE000FFF7D6FF02F11C0100F58060FFF7D0FF6D
:102EF00002F1380100F58060FFF7CAFF02F15401CA
:102F000000F58060FFF7C4FF02F1700100F58060FA
:102F1000FFF7BEFF02F18C0100F58060FFF7B8FFFC
:102F200002F1A80100F58060FFF7B2FF02F1C401D1
:102F300000F58060FFF7ACFF02F1E00100F5806072
:102F4000FFF7A6FFBDE8084000F0EEB800380240E9
:102F5000000002408836000808B500F059FAFEF774
:102F6000FFFBFFF793F8BDE80840FEF76DBE0000D9
:102F700070470000EFF3098305494A6B22F0010214
:102F80004A63683383F30988002383F31188704709
:102F900000EF00E0302080F3118862B60C4B0D4A40
:102FA000D96821F4E0610904090C0A43DA60D3F816
:102FB000FC20094942F08072C3F8FC200A6842F004
:102FC00001020A602022DA7783F82200704700BFEE
:102FD00000ED00E00003FA05001000E010B530231A
:102FE00083F311880E4B5B6813F4006314D0F1EE89
:102FF000103AEFF30984683C4FF08073E361094BAA
:10300000DB6B236684F30988FEF78AFB10B1064B5D
:10301000A36110BD054BFBE783F31188F9E700BFFF
:1030200000ED00E000EF00E02F030008320300088D
:103030000F4B1A6C42F001021A641A6E42F0010240
:103040001A660C4A1B6E936843F0010393604FF0BD
:10305000804353229A624FF0FF32DA6200229A6173
:103060005A63DA605A6001225A611A60704700BFE1
:1030700000380240002004E04FF0804208B511699A
:10308000D3680B40D9B2C9439B07116107D53023E0
:1030900083F31188FEF77AFB002383F3118808BDC0
:1030A0001F4B1A696FEAC2526FEAD2521A611A694B
:1030B000C2F308021A614FF0FF301A695A69586169
:1030C00000215A6959615A691A6A62F080521A627B
:1030D0001A6A02F080521A621A6A5A6A58625A6A66
:1030E00059625A6A1A6C42F080521A641A6E42F09F
:1030F00080521A661A6E0B4A106840F48070106095
:10310000186F00F44070B0F5007F1EBF4FF48030A0
:1031100018671967536823F40073536000F054B9BB
:103120000038024000700040334B4FF080521A6468
:10313000324A4FF4404111601A6842F001021A60AD
:103140001A689107FCD59A6822F003029A602A4B0C
:103150009A6812F00C02FBD1196801F0F9011960AC
:103160009A601A6842F480321A601A689203FCD599
:103170005A6F42F001025A671F4B5A6F9007FCD5F5
:103180001F4A5A601A6842F080721A601B4A5368DC
:103190005904FCD5184B1A689201FCD5194A9A605B
:1031A000194B1A68194B9A42194B21D1194A1168C7
:1031B000194A91421CD140F205121A60144A136850
:1031C00003F00F03052BFAD10B4B9A6842F0020271
:1031D0009A609A6802F00C02082AFAD15A6C42F4FA
:1031E00080425A645A6E42F480425A665B6E70475F
:1031F00040F20572E1E700BF003802400070004075
:103200000854400700948838002004E0116400202E
:10321000003C024000ED00E041C20F41074A08B502
:10322000536903F00103536123B1054A13680BB1DD
:1032300050689847BDE80840FFF7D0BE003C014009
:10324000E02D0020074A08B5536903F002035361DB
:1032500023B1054A93680BB1D0689847BDE8084090
:10326000FFF7BCBE003C0140E02D0020074A08B536
:10327000536903F00403536123B1054A13690BB189
:1032800050699847BDE80840FFF7A8BE003C0140E0
:10329000E02D0020074A08B5536903F00803536185
:1032A00023B1054A93690BB1D0699847BDE808403E
:1032B000FFF794BE003C0140E02D0020074A08B50E
:1032C000536903F01003536123B1054A136A0BB12C
:1032D000506A9847BDE80840FFF780BE003C0140B7
:1032E000E02D0020164B10B55C6904F478725A6129
:1032F000A30604D5134A936A0BB1D06A98476006B7
:1033000004D5104A136B0BB1506B9847210604D5B6
:103310000C4A936B0BB1D06B9847E20504D5094A70
:10332000136C0BB1506C9847A30504D5054A936CF8
:103330000BB1D06C9847BDE81040FFF74FBE00BFFF
:10334000003C0140E02D0020194B10B55C6904F4ED
:103350007C425A61620504D5164A136D0BB1506D5B
:103360009847230504D5134A936D0BB1D06D984748
:10337000E00404D50F4A136E0BB1506E9847A104B8
:1033800004D50C4A936E0BB1D06E9847620404D5F5
:10339000084A136F0BB1506F9847230404D5054AB0
:1033A000936F0BB1D06F9847BDE81040FFF716BE82
:1033B000003C0140E02D002008B5FFF75DFEBDE8B0
:1033C0000840FFF70BBE0000062108B50846FFF7CE
:1033D0001DFB06210720FFF719FB06210820FFF738
:1033E00015FB06210920FFF711FB06210A20FFF734
:1033F0000DFB06211720FFF709FB06212820FFF708
:1034000005FBBDE8084007211C20FFF7FFBA0000BC
:1034100008B5FFF745FE00F00BF8FDF78BFEFDF752
:1034200063FDFFF7A5FDBDE80840FFF7CFBC000036
:103430000023054A19460133102BC2E9001102F19D
:103440000802F8D1704700BFE02D0020034611F8B4
:10345000012B03F8012B002AF9D1704753544D3347
:1034600032463F3F3F0053544D33324634307800AC
:1034700053544D3332463432780053544D33324630
:103480003434365858000000012033000010410049
:1034900001105A000310590007103100000000000D
:1034A0005C340008130400006634000819040000AE
:1034B00070340008210400007A3400080000000085
:1034C000650E0008510E00088D0E0008790E0008E8
:1034D000850E0008710E00085D0E0008490E0008F8
:1034E000990E00080000000001000000000000002C
:1034F00063300000F0340008F02300200026002094
:103500004172647550696C6F740025424F4152449A
:10351000252D424C002553455249414C25000000C1
:10352000020000000000000081100008ED100008FB
:1035300040004000A02A0020B02A00200200000025
:10354000000000000300000000000000311100082E
:103550000000000010000000C02A00200000000051
:103560000100000000000000682D002001010200A1
:10357000E51B0008F51A0008911B0008751B0008E0
:10358000430000008835000809024300020100C022
:1035900032090400000102020100052400100105A7
:1035A000240100010424020205240600010705820B
:1035B000030800FF09040100020A000000070501DA
:1035C00002400000070581024000000012000000D8
:1035D000D4350008120110010200004009124157C1
:1035E00000020102030100000403090425424F41C7
:1035F000524425006F6D6E69627573663470726F28
:103600002D626473686F740030313233343536376D
:103610003839414243444546000000000040000064
:1036200000400000004000000040000000000100D9
:103630000000020000000200000002000000020082
:103640000000020000000200000002000000000074
:10365000751200082D150008D9150008400040001B
:10366000C82D0020C82D002001000000D82D00200A
:103670008000000040010000030000006D61696EE1
:103680000069646C650000000001804200000000D9
:10369000AAAAAAAA00010040FFFF00000000000043
:1036A00000A00A004005000100000000AAAAAAAA82
:1036B00040020001CFFF00000000000000000000F9
:1036C0000000000000000000AAAAAAAA0000000052
:1036D000FFFF0000000000000000000000000000EC
:1036E00000000000AAAAAAAA00000000FFFF000034
:1036F00000000000000000000000000000000000CA
:10370000AAAAAAAA00000000FFFF00000000000013
:10371000000000000000000000000000AAAAAAAA01
:1037200000000000FFFF000000000000000000009B
:103730000000000000000000AAAAAAAA00000000E1
:10374000FFFF00000000000000000000000000007B
:10375000000000000A00000000000000030000005C
:103760000000000000000000000000000000000059
:103770000000000000000000000000000000000049
:1037800000000000000000008300000000000000B6
:1037900000000F0000000000FF009600000000087D
:1037A000009600000000080004000000E835000852
:1037B0000000000000000000000000000000000009
:1037C0000000000000000000FFFFFFFFFFFFFFFF01
:1037D000FFFFFFFFFFFFFFFFFFFFFFFFFFFFFFFFF9
:1037E000FFFFFFFFFFFFFFFFFFFFFFFFFFFFFFFFE9
:1037F000FFFFFFFFFFFFFFFFFFFFFFFFFFFFFFFFD9
:10380000FFFFFFFFFFFFFFFFFFFFFFFFFFFFFFFFC8
:020000040801F1
:100000000006002099120108152607087125070827
:10001000DD25070871250708A92507089B12010897
:100020009B1201089B1201089B1201082DAD0908C3
:100030009B1201089B1201089B1201089B120108E8
:100040009B1201089B1201089B1201089B120108D8
:100050009B1201089B120108C5B80908EDB80908F0
:1000600015B909083DB9090865B90908E95D090824
:10007000115E09083D5E0908695E0908955E090878
:10008000BD5E0908E95E09086D5D09089B1201085B
:100090009B1201089B1201089B1201088DB90908E7
:1000A000B1BA0908B5BA0908C9BA0908CDBA090828
:1000B000D1BA0908E5BA0908F9BA09089B1201087A
:1000C0009B120108756409081D6609089B12010846
:1000D0009B12010861BA09089B12010875BA090848
:1000E000F1B909089B1201089B1201081DBB090800
:1000F00021BB090835BB090839BB0908155F090888
:100100009B1201089B1201080DBB09089B120108F4
:1001100089BA09089B1201089B1201089B12010869
:10012000415F0908695F0908955F0908C15F09080F
:10013000ED5F09089B1201089B1201089B12010840
:100140009B1201089B1201089B12010859B409086F
:1001500015600908416009086D6009089DBA090821
:100160009B1201089B1201089B1201089B120108B7
:100170009B1201089B1201089B1201089B120108A7
:100180009B1201089B1201089B1201089B12010897
:100190009B1201089B1201089B1201089B12010887
:1001A0009B1201089B1201089B1201089B12010877
:1001B0009B1201089B1201089B1201089B12010867
:1001C0009B1201089B1201089B1201089B12010857
:1001D0009B1201089B1201089B1201089B12010847
:1001E000CD25010841AF010845A204085DC30408FC
:1001F000412E0508053605083D390508DD9D050831
:1002000021BB050801480608395D0608916A060801
:1002100005170708A91C0708A9E607087129080897
:100220004D4A08080198080819BF080841D5080870
:10023000E9040908C90B09080000000000000000DB
:1002400081F0004102E000BF83F0004330B54FEA87
:1002500041044FEA430594EA050F08BF90EA020FF4
:100260001FBF54EA000C55EA020C7FEA645C7FEA87
:10027000655C00F0E2804FEA5454D4EB5555B8BFAA
:100280006D420CDD2C4480EA020281EA030382EA1B
:10029000000083EA010180EA020281EA0303362DAD
:1002A00088BF30BD11F0004F4FEA01314FF4801C80
:1002B0004CEA113102D0404261EB410113F0004F92
:1002C0004FEA03334CEA133302D0524263EB430349
:1002D00094EA050F00F0A780A4F10104D5F1200EE7
:1002E0000DDB02FA0EFC22FA05F2801841F1000142
:1002F00003FA0EF2801843FA05F359410EE0A5F116
:1003000020050EF1200E012A03FA0EFC28BF4CF046
:10031000020C43FA05F3C01851EBE37101F00045FC
:1003200007D54FF0000EDCF1000C7EEB00006EEB09
:100330000101B1F5801F1BD3B1F5001F0CD3490893
:100340005FEA30004FEA3C0C04F101044FEA4452EA
:1003500012F5800F80F09A80BCF1004F08BF5FEA71
:10036000500C50F1000041EB045141EA050130BD51
:100370005FEA4C0C404141EB0101013C28BFB1F563
:10038000801FE9D291F0000F04BF01460020B1FAAE
:1003900081F308BF2033A3F10B03B3F120020CDA81
:1003A0000C3208DD02F1140CC2F10C0201FA0CF05F
:1003B00021FA02F10CE002F11402D8BFC2F1200CC4
:1003C00001FA02F120FA0CFCDCBF41EA0C0190407A
:1003D000E41AA2BF01EB0451294330BD6FEA0404C3
:1003E0001F3C1CDA0C340EDC04F11404C4F12002AE
:1003F00020FA04F001FA02F340EA030021FA04F3C0
:1004000045EA030130BDC4F10C04C4F1200220FA16
:1004100002F001FA04F340EA0300294630BD21FA54
:1004200004F0294630BD94F0000F83F4801306BF1A
:1004300081F480110134013D4EE77FEA645C18BF0E
:100440007FEA655C29D094EA050F08BF90EA020FA5
:1004500005D054EA000C04BF1946104630BD91EA9D
:10046000030F1EBF0021002030BD5FEA545C05D1A0
:100470004000494128BF41F0004130BD14F58004DF
:100480003CBF01F5801130BD01F0004545F0FE4153
:1004900041F470014FF0000030BD7FEA645C1ABF88
:1004A000194610467FEA655C1CBF0B46024650EABF
:1004B000013406BF52EA033591EA030F41F40021EB
:1004C00030BD00BF90F0000F04BF0021704730B571
:1004D0004FF4806404F132044FF000054FF0000146
:1004E00050E700BF90F0000F04BF0021704730B507
:1004F0004FF4806404F1320410F0004548BF4042DC
:100500004FF000013EE700BF42004FEAE2014FEA30
:1005100031014FEA02701FBF12F07F4393F07F4F0B
:1005200081F06051704732F07F4208BF704793F00E
:100530007F4F04BF41F40021704730B54FF4607421
:1005400001F0004521F000411CE700BF50EA010224
:1005500008BF704730B54FF000050AE050EA0102CD
:1005600008BF704730B511F0004502D5404261EB3D
:1005700041014FF4806404F132045FEA915C3FF47E
:10058000D8AE4FF003025FEADC0C18BF03325FEA1B
:10059000DC0C18BF033202EBDC02C2F1200300FACC
:1005A00003FC20FA02F001FA03FE40EA0E0021FAF1
:1005B00002F11444BDE600BF70B54FF0FF0C4CF4DF
:1005C000E06C1CEA11541DBF1CEA135594EA0C0F91
:1005D00095EA0C0F00F0DEF82C4481EA030621EACC
:1005E0004C5123EA4C5350EA013518BF52EA033507
:1005F00041F4801143F4801338D0A0FB02CE4FF0B9
:100600000005E1FB02E506F00042E0FB03E54FF0E8
:100610000006E1FB03569CF0000F18BF4EF0010EE0
:10062000A4F1FF04B6F5007F64F5407404D25FEADC
:100630004E0E6D4146EB060642EAC62141EA55518F
:100640004FEAC52040EA5E504FEACE2EB4F1FD0CD1
:1006500088BFBCF5E06F1ED8BEF1004F08BF5FEA4F
:10066000500E50F1000041EB045170BD06F0004601
:1006700046EA010140EA020081EA0301B4EB5C04AE
:10068000C2BFD4EB0C0541EA045170BD41F48011A6
:100690004FF0000E013C00F3AB8014F1360FDEBFCB
:1006A000002001F0004170BDC4F10004203C35DAA7
:1006B0000C341BDC04F11404C4F1200500FA05F32A
:1006C00020FA04F001FA05F240EA020001F00042CB
:1006D00021F0004110EBD37021FA04F642EB060141
:1006E0005EEA430E08BF20EAD37070BDC4F10C046B
:1006F000C4F1200500FA04F320FA05F001FA04F22F
:1007000040EA020001F0004110EBD37041F100011A
:100710005EEA430E08BF20EAD37070BDC4F1200525
:1007200000FA05F24EEA020E20FA04F301FA05F28D
:1007300043EA020321FA04F001F0004121FA04F235
:1007400020EA020000EBD3705EEA430E08BF20EA05
:10075000D37070BD94F0000F0FD101F0004640003F
:1007600041EB010111F4801F08BF013CF7D041EAC1
:10077000060195F0000F18BF704703F000465200C5
:1007800043EB030313F4801F08BF013DF7D043EA96
:100790000603704794EA0C0F0CEA135518BF95EA4C
:1007A0000C0F0CD050EA410618BF52EA4306D1D1D3
:1007B00081EA030101F000414FF0000070BD50EAF2
:1007C000410606BF1046194652EA430619D094EA7C
:1007D0000C0F02D150EA013613D195EA0C0F05D166
:1007E00052EA03361CBF104619460AD181EA0301BA
:1007F00001F0004141F0FE4141F470014FF0000072
:1008000070BD41F0FE4141F4780170BD70B54FF00C
:10081000FF0C4CF4E06C1CEA11541DBF1CEA13558C
:1008200094EA0C0F95EA0C0F00F0A7F8A4EB05046E
:1008300081EA030E52EA03354FEA013100F0888065
:100840004FEA03334FF0805545EA131343EA12632E
:100850004FEA022245EA111545EA10654FEA0026E3
:100860000EF000419D4208BF964244F1FD0404F59C
:10087000407402D25B084FEA3202B61A65EB0305F8
:100880005B084FEA32024FF480104FF4002CB6EBB5
:10089000020E75EB030E22BFB61A754640EA0C0035
:1008A0005B084FEA3202B6EB020E75EB030E22BF75
:1008B000B61A754640EA5C005B084FEA3202B6EBB6
:1008C000020E75EB030E22BFB61A754640EA9C0075
:1008D0005B084FEA3202B6EB020E75EB030E22BF45
:1008E000B61A754640EADC0055EA060E18D04FEA03
:1008F000051545EA16754FEA06164FEAC30343EAA3
:1009000052734FEAC2025FEA1C1CC0D111F4801F6F
:100910000BD141EA00014FF000004FF0004CB6E768
:1009200011F4801F04BF01430020B4F1FD0C88BF07
:10093000BCF5E06F3FF6AFAEB5EB030C04BFB6EB12
:10094000020C5FEA500C50F1000041EB045170BD05
:100950000EF0004E4EEA113114EB5C04C2BFD4EB32
:100960000C0541EA045170BD41F480114FF0000EB6
:10097000013C90E645EA060E8DE60CEA135594EA32
:100980000C0F08BF95EA0C0F3FF43BAF94EA0C0F35
:100990000AD150EA01347FF434AF95EA0C0F7FF4AA
:1009A00025AF104619462CE795EA0C0F06D152EAFE
:1009B00003353FF4FDAE1046194622E750EA4106E2
:1009C00018BF52EA43067FF4C5AE50EA41047FF4F3
:1009D0000DAF52EA43057FF4EBAE12E74FF0FF3C58
:1009E00006E000BF4FF0010C02E000BF4FF0010C29
:1009F0004DF804CD4FEA410C7FEA6C5C4FEA430CA2
:100A000018BF7FEA6C5C1BD001B050EA410C0CBFF0
:100A100052EA430C91EA030F02BF90EA020F002052
:100A2000704710F1000F91EA030F58BF994208BFB9
:100A300090422CBFD8176FEAE37040F00100704776
:100A40004FEA410C7FEA6C5C02D150EA013C07D1CD
:100A50004FEA430C7FEA6C5CD6D152EA033CD3D018
:100A60005DF8040B704700BF8446104662468C4612
:100A70001946634600E000BF01B5FFF7B7FF002845
:100A800048BF10F1000F01BD4DF808EDFFF7F4FF6E
:100A90000CBF012000205DF808FB00BF4DF808EDF9
:100AA000FFF7EAFF34BF012000205DF808FB00BF1C
:100AB0004DF808EDFFF7E0FF94BF012000205DF83E
:100AC00008FB00BF4DF808EDFFF7CEFF94BF0120F3
:100AD00000205DF808FB00BF4DF808EDFFF7C4FFEC
:100AE00034BF012000205DF808FB00BF4FEA410C35
:100AF0007FEA6C5C02D150EA013C0AD14FEA430C18
:100B00007FEA6C5C02D152EA033C02D14FF0000054
:100B100070474FF0010070474FEA410212F5001292
:100B200015D211D56FF47873B3EB625212D94FEA34
:100B3000C12343F0004343EA505311F0004F23FA1E
:100B400002F018BF404270474FF00000704750EA73
:100B5000013005D111F0004008BF6FF00040704730
:100B60004FF00000704700BF4A0011D212F500128A
:100B700011D20DD56FF47873B3EB62520ED44FEAF5
:100B8000C12343F0004343EA505323FA02F0704775
:100B90004FF00000704750EA013002D14FF0FF30B3
:100BA00070474FF0000070474FEA4102B2F1E04356
:100BB00024BFB3F5001CDCF1FE5C0DD901F0004C44
:100BC0004FEAC0024CEA5070B2F1004F40EB830094
:100BD00008BF20F00100704711F0804F21D113F1C0
:100BE0003872BCBF01F00040704741F480114FEAF9
:100BF0005252C2F11802C2F1200C10FA0CF320FA82
:100C000002F018BF40F001004FEAC1234FEAD3239E
:100C100003FA0CFC40EA0C0023FA02F34FEA430308
:100C2000CCE77FEA625307D150EA01331EBF4FF091
:100C3000FE4040F44000704701F0004040F0FE40AC
:100C400040F40000704700BF80F0004002E000BFA9
:100C500081F0004142001FBF5FEA410392EA030FA7
:100C60007FEA226C7FEA236C6AD04FEA1262D2EBF1
:100C70001363C1BFD218414048404140B8BF5B42F6
:100C8000192B88BF704710F0004F40F4000020F08F
:100C90007F4018BF404211F0004F41F4000121F0A5
:100CA0007F4118BF494292EA030F3FD0A2F10102EF
:100CB00041FA03FC10EB0C00C3F1200301FA03F12D
:100CC00000F0004302D5494260EB4000B0F5000F50
:100CD00013D3B0F1807F06D340084FEA310102F10F
:100CE0000102FE2A51D2B1F1004F40EBC25008BFC1
:100CF00020F0010040EA03007047490040EB00008B
:100D0000013A28BFB0F5000FEDD2B0FA80FCACF18B
:100D1000080CB2EB0C0200FA0CF0AABF00EBC250B8
:100D200052421843BCBFD0401843704792F0000FA6
:100D300081F4000106BF80F400000132013BB5E7F9
:100D40004FEA41037FEA226C18BF7FEA236C21D06F
:100D500092EA030F04D092F0000F08BF08467047D4
:100D600090EA010F1CBF0020704712F07F4F04D1A2
:100D7000400028BF40F00040704712F100723CBFB5
:100D800000F50000704700F0004343F0FE4040F4DF
:100D9000000070477FEA226216BF08467FEA23639D
:100DA0000146420206BF5FEA412390EA010F40F488
:100DB000800070474FF0000304E000BF10F00043D4
:100DC00048BF40425FEA000C08BF704743F09643BB
:100DD00001464FF000001CE050EA010208BF7047D6
:100DE0004FF000030AE000BF50EA010208BF70475D
:100DF00011F0004302D5404261EB41015FEA010C72
:100E000002BF84460146002043F0B64308BFA3F169
:100E10008053A3F50003BCFA8CF2083AA3EBC2534B
:100E200010DB01FA02FC634400FA02FCC2F120026A
:100E3000BCF1004F20FA02F243EB020008BF20F0A1
:100E40000100704702F1200201FA02FCC2F1200207
:100E500050EA4C0021FA02F243EB020008BF20EAFC
:100E6000DC7070477BB972B90029BEBF00204FF01B
:100E7000004106E008BF00281CBF6FF000414FF0A2
:100E8000FF3000F007BAADF1080C6DE904CE00297F
:100E900009DB002B1ADB00F095F8DDF804E0DDE952
:100EA000022304B07047404261EB4101002B1BDB81
:100EB00000F088F8DDF804E0DDE9022304B04042E8
:100EC00061EB4101524263EB43037047524263EBD3
:100ED000430300F077F8DDF804E0DDE9022304B015
:100EE000404261EB41017047524263EB430300F023
:100EF00069F8DDF804E0DDE9022304B0524263EB57
:100F00004303704753B94AB9002908BF00281CBFE2
:100F10004FF0FF314FF0FF3000F0BCB9ADF1080CDD
:100F20006DE904CE00F04EF8DDF804E0DDE90223BF
:100F300004B07047430803F05533C01A830803F028
:100F4000333300F03330184400EB101000F00F3052
:100F500000EB002000EB0040000E704707EE900A07
:100F6000F5EEC07AF1EE10FA01D400F00BB8F1EE14
:100F7000677A08B517EE900A00F004F8404261EB7A
:100F8000410108BDD0B5FFF7BFFA0C4B0022064661
:100F90000F46FFF711FBFFF7E7FD0446FFF792FA54
:100FA000074B0022FFF708FB02460B463046394646
:100FB000FFF74AF9FFF7D8FD2146D0BD0000F03D0C
:100FC0000000F0412DE9F047089D04468E46002BB5
:100FD0004DD18A42944669D9B2FA82F252B101FAED
:100FE00002F3C2F1200120FA01F10CFA02FC41EAFD
:100FF000030E94404FEA1C48210CBEFBF8F61FFA82
:101000008CF708FB16E341EA034306FB07F199421C
:101010000AD91CEB030306F1FF3080F01F819942CF
:1010200040F21C81023E63445B1AA4B2B3FBF8F0A9
:1010300008FB103344EA034400FB07F7A7420AD930
:101040001CEB040400F1FF3380F00A81A74240F258
:1010500007816444023840EA0640E41B00261DB1C3
:10106000D4400023C5E900433146BDE8F0878B42F8
:1010700009D9002D00F0EF800026C5E900013046B7
:101080003146BDE8F087B3FA83F6002E4AD18B4291
:1010900002D3824200F2F980841A61EB030301203B
:1010A0009E46002DE0D0C5E9004EDDE702B9FFDE27
:1010B000B2FA82F2002A40F09280A1EB0C014FEAD2
:1010C0001C471FFA8CFE0126200CB1FBF7F307FB2F
:1010D000131140EA01410EFB03F0884208D91CEBD2
:1010E000010103F1FF3802D2884200F2CB8043466F
:1010F000091AA4B2B1FBF7F007FB101144EA01444E
:101100000EFB00FEA64508D91CEB040400F1FF31DC
:1011100002D2A64500F2BB800846A4EB0E0440EACA
:1011200003409CE7C6F12007B34022FA07FC4CEAD3
:10113000030C20FA07F401FA06F31C43F9404FEAC6
:101140001C4900FA06F3B1FBF9F8200C1FFA8CFEDB
:1011500009FB181140EA014108FB0EF0884202FA2F
:1011600006F20BD91CEB010108F1FF3A80F08880F0
:10117000884240F28580A8F102086144091AA4B2AD
:10118000B1FBF9F009FB101144EA014100FB0EFE2E
:101190008E4508D91CEB010100F1FF346CD28E455D
:1011A0006AD90238614440EA0840A0FB0294A1EBEE
:1011B0000E01A142C846A64656D353D05DB1B3EB4B
:1011C000080261EB0E0101FA07F722FA06F3F1407B
:1011D0001F43C5E9007100263146BDE8F087C2F122
:1011E0002003D8400CFA02FC21FA03F3914001439A
:1011F0004FEA1C471FFA8CFEB3FBF7F007FB1036D3
:101200000B0C43EA064300FB0EF69E4204FA02F47E
:1012100008D91CEB030300F1FF382FD29E422DD9D1
:10122000023863449B1B89B2B3FBF7F607FB163306
:1012300041EA034106FB0EF38B4208D91CEB010186
:1012400006F1FF3816D28B4214D9023E6144C91A06
:1012500046EA004638E72E46284605E70646E3E616
:101260001846F8E64B45A9D2B9EB020864EB0C0E20
:101270000138A3E74646EAE7204694E74046D1E72F
:10128000D0467BE7023B614432E7304609E76444DD
:10129000023842E7704700BF02E000F000F8FEE7C6
:1012A00072B6374880F30888364880F30988364894
:1012B0003649086040F20000CCF200004EF634716E
:1012C000CEF200010860BFF34F8FBFF36F8F40F283
:1012D0000000C0F2F0004EF68851CEF20001086026
:1012E000BFF34F8FBFF36F8F4FF00000E1EE100A96
:1012F0004EF63C71CEF200010860062080F314889F
:10130000BFF36F8F89F070FD88F0D6FD4FF0553038
:101310001F491B4A91423CBF41F8040BFAE71D49A3
:10132000184A91423CBF41F8040BFAE71A491B4A9C
:101330001B4B9A423EBF51F8040B42F8040BF8E7EE
:1013400000201849184A91423CBF41F8040BFAE7C3
:1013500089F04EFD88F004FE144C154DAC4203DAC2
:1013600054F8041B8847F9E701F020F9114C124D9D
:10137000AC4203DA54F8041B8847F9E789F036BD1C
:1013800000060020002200200000010808ED00E017
:10139000000000200006002068D60B080022002074
:1013A000A8250020A8250020702A0120E0010108BE
:1013B0003802010838020108380201082DE9F04F0F
:1013C0002DED108AC1F80CD0C3689D46BDEC108A83
:1013D000BDE8F08F002383F311882846A047002042
:1013E00088F0F0FAFEE788F04DF900DFFEE7000034
:1013F00001F0FF01102A2BDB10F0070F08D010F8C6
:10140000013B013A8B422DD010F0070F42B3F6D1C9
:10141000F0B441EA012141EA014122F007047FF0E2
:1014200000070023F0E80256083C85EA010586EA39
:10143000010685FA47F5A3FA87F586FA47F6A5FA75
:1014400087F68EB9EED1F0BC01F0FF0102F0070281
:1014500032B110F8013B013A83EA010313B1F8D12C
:101460000020704701387047002D06BF354603380D
:10147000073815F0010F07D1013015F4807F02BF46
:10148000013015F4C03F0130F0BC0138704700BF97
:1014900010F8012B11F8013B012A28BF9A42F7D01E
:1014A000D01A7047034613F8012B002AFBD1181AF3
:1014B0000138704738B50022002304460D46FFF777
:1014C000EDFA28B920462946BDE8384000F00AB8B0
:1014D000204605F1004100F005F8404261EB410172
:1014E00038BD00BFD0B50C4B002206460F46FFF7B3
:1014F00063F8FFF739FB0446FEF7E4FF074B0022D1
:10150000FFF75AF802460B4630463946FEF79CFE76
:10151000FFF72AFB2146D0BD0000F03D0000F0415E
:10152000036800221B6818470120704737B50191F6
:10153000202104465EF078F9D0B10E4B93F98A145D
:10154000A1B1B3F98C14D3F85C3C019AB3F90A50F9
:1015500001F10A039D4203DD40F28D33994205DC1F
:101560002046054B20215EF067F9002003B030BD16
:101570000120FBE7B0450020EC2F0A0807B504481E
:101580005FF0E0FB00F0010003B05DF804FB00BF7A
:10159000245B00202DE9F0438FB00E46054605F090
:1015A000E3FD002780462E22394602A801978DF0E0
:1015B0003DFB322301AA3946404605F01FF9044697
:1015C00048B9184A01AB314628465EF03DFB20463B
:1015D0000FB0BDE8F083DFF85890D9F8880A0368A7
:1015E0009B6898470028F2D0A9F5405003F0B0FD61
:1015F000814630B90C4A314628465EF025FB4C4600
:10160000E5E76946404604F04FFF0028DFD09DF82B
:1016100001305B06DBD5054A314628465EF014FBF7
:101620003C46D4E700300A0809300A0820300A088E
:10163000B055002008B5064B93F8F13E9B0704D542
:10164000044A5EF001FB002008BD0120FCE700BF5A
:10165000B045002030300A0870B50C4C0546D4F86F
:10166000880A0368DB680E46984710B101242046BB
:1016700070BDA4F5405003F089FD04460028F5D163
:10168000034A314628465EF0DFFAF0E7B055002005
:1016900040300A082DE97043264BD3F8F43E1D7BF9
:1016A000804689465DB9244B1B68986A03685B6B6A
:1016B000984738B9214A494640465EF0C5FA28465F
:1016C000BDE8708348F0CEFD202149F045FD38B1DA
:1016D00048F0C8FD1F2149F03FFD08B1184AEAE76C
:1016E000D8F808303BB9D8F80030494640465B6B23
:1016F000BDE87043184749464046FFF717FF494683
:10170000064640465EF04CFF2021064040465EF013
:101710008BF849464046FFF78DFFF5B20540494634
:101720004046FFF799FF4946054040465FF00EF9F5
:101730000540C4E7B04500204061002054300A084D
:101740006B300A0808B5FFF7A5FF054A92F8E01EBE
:1017500060F3410182F8E01E024A907108BD00BFAB
:10176000B0450020CD610020F7B505460F465EF07C
:1017700097F8044678B1022128465EF055F80646EF
:1017800048B115485FF0DEFAC205C0F30723C0F385
:10179000002403D53446204603B0F0BD9B07F9D59D
:1017A0000D485FF0D9FA0D4B03F27C43D3ED007A7C
:1017B000F8EEE77A30EE670ADFED097AB0EEC00A9C
:1017C000B4EEE70AF1EE10FAE4DD064B3A460221E8
:1017D00028465EF031F8DEE7245B0020B05500209B
:1017E0000000C84288300A08F8B504460F465EF08B
:1017F000D3FA1021054620465EF016F858B120466F
:10180000FFF7BCFE064630B9044B3A46102120468D
:101810005EF012F835462846F8BD00BF9C300A0835
:1018200070B505460E465DF0A7FF044678B18021ED
:1018300028465DF0F9FF50B1094B93F8793443B174
:10184000084B3246802128465DF0F6FF00242046F2
:1018500070BD31462846BDE870405EF065BC00BFF3
:10186000B0550020B0300A082DE9F04180460E4600
:10187000FFF790FE1A4F044610B90024FC710AE0ED
:10188000184D05F54053D3F8880A03689B689847BC
:1018900020B90123FB712046BDE8F08108214046B4
:1018A0005DF0C2FF0028F4D095F81434B02202FB9A
:1018B000035305F50055B3F81E22B5F988349A4252
:1018C00006DD094B3246082140465DF0B5FFD4E7FE
:1018D000314640465EF0DCF80028DAD1CDE700BFA3
:1018E000CD610020B0250020C4300A085EF01CBD88
:1018F00070B505460E46FFF74DFE084B0446D871FD
:1019000031462846FFF7A8FE31460028284608BF82
:1019100000245EF0CBFE204070BD00BFCD610020F2
:101920002DE9F843414F3B788146002B7BD1404C59
:10193000D4F8F45E2D7B01263E701DB13B70284625
:10194000BDE8F8835FF0BCF8054630B9394A387015
:10195000137843F001031370F1E7DFF8F4803CF0F3
:10196000A3FC31463BF08CFC88F804600B2635F074
:1019700043F8013E34F0F6FF16F0FF06F7D12E498A
:1019800048465EF0B7FF05F0EFFBD0F80022C4F840
:10199000042F90F87C32DA0733D404F095FF3CF042
:1019A00083FC3C213CF018FA04F6EC6300221A6038
:1019B000224B1B68D86A036801211B689847D4F83A
:1019C000F42E137B1BB90123137388F804303CF009
:1019D0006BFC94F8E52E94F8E41E3BF02DFE39F0F4
:1019E00045FC38F085FF00233B7060F049FE144B46
:1019F000C3F8780A94F8E13E43F0200384F8E13E0E
:101A00009DE79B07D4D431460E4802F0F3F90E4807
:101A10005FF0A2F9DFED0D7A20EE270A04F6EC6301
:101A200083ED000AC4E7002589E700BFA825002050
:101A3000B0450020EC610020D4300A08406100204D
:101A4000B0550020B0250020245B00200AD7233C9D
:101A5000CD6100202DE9F0432B4DD5F8F43E1B7BE2
:101A600087B00646002B4CD05FF0E0F80446002813
:101A700043D0264930465EF03DFF05F075FB074632
:101A800009F0DCFF8046384604F0DAF9D8B198F95D
:101A90002430022B17D100264FF00009F1B203AA1F
:101AA00038460191CDF80C90CDF81090CDF81490F7
:101AB00004F040FD019918B103AA404609F0CAFCA0
:101AC0000136032EEAD1D5F8F42E137B1BB1002387
:101AD00013730F4A13713CF0E7FB00213BF0D0FB7E
:101AE0000C4B1B68D86A036800211B68984795F85F
:101AF000E13E6FF3451385F8E13E204607B0BDE8AF
:101B0000F0830124F9E700BFB0450020E4300A0863
:101B1000CD6100204061002008B500F5005090F82C
:101B2000E03EC3F380028A420BD061F3820380F867
:101B3000E03E31B13CF0B8FBBDE808400F213CF07D
:101B40004BB908BD10B500F500520C4692F8F13EB5
:101B500003F00101A14209D064F3000382F8F13ED1
:101B6000DB0704D402F096FB024B9C7210BD02F01E
:101B700045FCF9E7CD61002000F5005090F8F13EFA
:101B800061F3410380F8F13E014B1973704700BFC8
:101B9000CD61002000207047002070470020704772
:101BA00000207047002070470020704700207047D9
:101BB00000207047002070470020704700207047C9
:101BC0007047000000F51250183070470048704709
:101BD0008C5D0A0800F5005090F8E40E7047000094
:101BE000034808601D21117008221A60704700BF69
:101BF000C0330A0839F084BA18F04CBA3BF0C2BCC2
:101C000047F07CBF46F0B2B802F064BB02F096BA6F
:101C100002F0BCB934F0A6BE4CF0E4BE03F07EB8CE
:101C200048F06EBA12F030BC02F0D2B802F096BDA5
:101C300002F04CBA02F0EABC03F05AB818F01CBE2D
:101C400003F0BCBA02F07CBB02F034BC70B5224B8E
:101C5000036000F500550446D5F8740E1F4BC5F817
:101C6000B83C08B109F07EF91D4B236095F8EC30C3
:101C700043B9D5F8E8502DB1284616F099FF28460B
:101C800009F06CF904F59A500C305DF029F804F570
:101C9000985010304AF0F8F804F6E46504F68466CB
:101CA000B54204D0183D284616F0F2FBF8E70D4B7C
:101CB000C4F8C83804F628203EF08CFC04F6FC106A
:101CC0003EF088FC04F65C103EF084FC04F51360E2
:101CD0003EF080FC204670BD10360A080C120B083E
:101CE000E0EF0A08F4C60A0838B54D4B044640F840
:101CF000043B4BF0FDF904F1100008F01BFD04F16A
:101D0000680038F08BFF04F5907011F01FF804F5AF
:101D10008C6007F09BFA04F2845009F025F904F670
:101D2000C80017F0FDFF04F566604BF069F904F593
:101D3000736038F027FC04F58F503BF0F1F904F59F
:101D40009750143050F0E6FE04F5985010304AF0E9
:101D500083F804F59A500C305CF0AEFF04F59B500C
:101D6000083039F01DFB04F59C500C304CF09EFB04
:101D700004F5805300252B4A83F8B05304F59D5396
:101D8000103304F59E50136034F060FC04F5A0504D
:101D90002946103003F046FD04F5D350183057F0B3
:101DA000B9F804F5FB501C3059F0BEFF04F50250A1
:101DB00014305CF0DBF804F5035038305CF010FDB3
:101DC00004F50550103003F08DFB04F50A50303057
:101DD00057F094FD04F50C501349083037F0C6FC59
:101DE00004F50C50203051F039F904F50F501C3037
:101DF0005DF0FEFA04F5005304F5115083F83454F5
:101E00000A4D0C305DF016FC2B6813B1084860F0E9
:101E100005FC2046074937F0A9FC2C60204638BD58
:101E2000E0EF0A08546B0020787C0B08A4620020C5
:101E300038310A08F8EE0A0810B503F0ADF848F09A
:101E400011FA0368BDE810405B681847FFF7F4BF5C
:101E500038B500F53C5508350446284608F044FBE3
:101E600009F0ECFD90F92130D3B190F84033BBB1CB
:101E70002846002108F0CCF8DFED0A7A04F2DC7382
:101E800093ED287A20EE270ADFED077AA7EE270ADE
:101E900004F2845083ED280ABDE8384009F0DEBC26
:101EA00038BD00BFCDCCCC3D6666663FFFF7D0BFE6
:101EB00010B50121044603F0A5F910B1204601F048
:101EC000E7F84FF48051204603F09CF920B12046FA
:101ED000BDE8104001F09EB810BD0000FFF7E8BF5C
:101EE00013B50221044603F08DF938B101212046D3
:101EF00003F088F910B9204601F0CAF80221204603
:101F000003F080F950B3204601F0D0F8402120467C
:101F100003F078F960B104F58F5001903AF0FEFCBF
:101F200004F58053019893F910330BB13AF038FE61
:101F30004FF48061204603F065F918B104F58F5025
:101F40003AF086FD8021204603F05CF968B119F073
:101F50008FFE02B0BDE8104017F0DABC0121204628
:101F600003F050F90028CED1D0E74FF4802120466D
:101F700003F048F90028EAD14FF40021204603F08D
:101F800041F90028E3D102B010BD0000FFF7A8BF5F
:101F900010B50121044603F035F910B1204601F0D7
:101FA00085F88021204603F02DF928B119F060FE54
:101FB000BDE8104017F088BC10BD0000FFF7E8BF77
:101FC00038B54FF6FF71044603F01CF904F50055CF
:101FD00028B1D5F8E02E0721204601F06FF849F02E
:101FE00099FD49F03DFB95F8E03E074A83F0100368
:101FF000C3F30013537139F039F938F0A1FDBDE88E
:102000003840024856F064BACD610020405F00209D
:10201000FFF7D6BF2DE9F04F2DED028B00F5A05450
:102020001034A3B005460121204605F023F805F53C
:1020300052511C31204604F0A9FE05F552513431AD
:10204000204603F09FFF05F5BA5104F545700831AD
:102050001CF0ECFC05F5405405F5535704F29C4880
:1020600004F5946A87ED000A3846D8F80020DAF8BB
:102070000030209220A9083021933FF075FA05F531
:10208000525105F5545024310C30B0EE608AF0EE18
:10209000408A3FF0EBF804F5956904F5966304F285
:1020A000AC4BC9ED008A39468BED008A05F55550D9
:1020B00083ED000A1D933FF0D9F804F2C44282ED8B
:1020C000000A1C923CF0F0F8054660F0E1FA1B9122
:1020D0002C4906460868FEF717FACDE9180104F204
:1020E000BC410868FEF710FACDE9160104F59761C6
:1020F0000868FEF709FACDE9140104F2B44104F2CC
:10210000A4440868FEF700FACDE912011C9A106891
:10211000FEF7FAF9CDE910013868FEF7F5F9CDE9D7
:102120000E011D9B1868FEF7EFF9CDE90C01206840
:10213000FEF7EAF9CDE90A01DBF80000FEF7E4F961
:10214000CDE90801DAF80000FEF7DEF9CDE9060175
:10215000D9F80000FEF7D8F9CDE90401D8F800005D
:10216000FEF7D2F91B9B0193CDE90201064B074A0A
:102170000749009628463BF0C3FC23B0BDEC028B18
:10218000BDE8F08FCC3B00204C310A085A310A08D8
:1021900087310A08FFF73EBF10B5044602F06EFF14
:1021A0001021204603F02EF828B119F061FDBDE89A
:1021B000104017F085BC10BDFFF7EEBF00F5A05032
:1021C000D0ED985AD0ED9B6AD1ED017A91ED006A7D
:1021D00026EEE77A67EEA57AA6EE257AE6EE267A6F
:1021E00081ED007AC1ED017A7047000000F5A05042
:1021F000D0ED985AD0ED9B6AD1ED017A91ED006A4D
:1022000027EEA67A67EEA57AA6EE257AE6EE667A3E
:1022100081ED007AC1ED017A704700002DE9F043AD
:102220002DED028B044687B0FFF75EFDC74B2360A0
:1022300004F513500C3001F061FC04F5005504F571
:102240001253103304F531562C36C5F8643C06237E
:1022500085F8683C30465DF09BFA0DF11008BC4BE8
:10226000C5F86C3C301D0123414604F532578DF80A
:102270001030383738F052F8B64BC5F8B83C07F193
:1022800014005FF0CDF804F5335604F535593036B7
:1022900009F114093046143643F030FE4E45F9D1A9
:1022A0000723C5F8783E0023A5F87C3E4FF4CB7099
:1022B00008F052FEC5F8740E04F53A505FF0B0F81D
:1022C00004F53B5004305FF0ABF8A34B1A6802B939
:1022D0001F60A24BC5F8B83C04F53B500123A5F89C
:1022E000E43E26305EF0C2FC9D4B05939D4B04946A
:1022F000009304F53C5098E80C004FF4007108304E
:1023000007F038FDF7EE008A03A904F55250CDED31
:10231000038A3EF017FD04F552509FED938A04F5B1
:1023200040550C3008F018FB05F29C4383ED008A01
:1023300083ED018A83ED028A05F5956383ED008ABA
:1023400083ED018A83ED028A05F2B44383ED008AAE
:1023500083ED018A83ED028A05F2EC4383ED008A66
:1023600083ED018A05F2F44383ED008A83ED018A4F
:1023700005F2FC4383ED008A83ED018A05F20453E4
:1023800083ED008A83ED018A05F2745383ED008AA0
:1023900083ED018A83ED028A04F556539FED732A7B
:1023A00083ED008A83ED018A83ED028A04F5A05350
:1023B0001033B0EE083A04F55650C5F88C35F0EEFF
:1023C000432AF0EE420AB0EE430AF0EE481AB0EEAD
:1023D000481A103056F01AFAB0EE083A04F55B507D
:1023E000F0EE432AB0EE682AF0EE481AB0EE481A32
:1023F000F7EE080AB1EE0C0A1C3056F0EBFBB0EE1B
:10240000083A04F55D50F0EE432AB0EE430A9FED22
:10241000572ADFED570AF0EE481AB0EE481A14308A
:1024200056F0D8FBB0EE083A04F55F50F0EE432AC0
:102430009FED502ADFED500AF0EE481AB0EE481A30
:10244000B0EE680A0C3056F0E1F9B0EE083A04F547
:102450006450F0EE432A9FED490AB0EE482AF0EEB0
:10246000481AB0EE481AF0EE480A183056F0B2FB9F
:10247000F0EE083A04F566509FED410AB0EE485A76
:10248000F0EE684AB0EE484AB0EE633AF0EE632AE6
:10249000B0EE002AF0EE481AB0EE481AF6EE000A46
:1024A000103055F0C5FF374937480860002304F560
:1024B0006A5285F87D3A043214279EB207FB060162
:1024C0000133097C0029F8D1304B1E80304B19684C
:1024D00011B1304860F0A2F804F56A500C30C5F82C
:1024E000880A1A6002F0F4F82B4BC5F88C3A04F510
:1024F0006A503C3002F0ECF8284BC5F8BC3A04F5C1
:102500006B502C3002F0E4F8254BC5F8EC3A04F59A
:102510006C501C3002F0DCF8224BC5F81C3B04F573
:102520006D5005F64C3383ED008A83ED018A83ED0F
:10253000028A1C3002F0CCF81B4BC5F85C3B2046ED
:1025400007B0BDEC028BBDE8F08300BF10360A086F
:1025500000310A080C120B08E8650020C8360A088A
:10256000491C010804360A0800000000CDCC4C3E8E
:10257000CDCCCC3ECDCCCC3DCDCC4C3D3333333F1C
:102580009A99993F68620020706F0A08666200207D
:10259000246200208C310A0804790A084C780A0861
:1025A000B0790A08A8780A0850790A0838B5054BA6
:1025B0001C6823680A461D68034B01462046A8474D
:1025C000002038BD40610020B025002010B55FF02C
:1025D00067FB064C064B18602046FFF71FFE20469F
:1025E000044A0549BDE8104089F0F2BDB02500203D
:1025F0004061002050BF00204D1C010810B504466A
:102600000180024937F0B2F8204610BD90360A0822
:1026100010B500234FF07C52274C03654FF07E51DC
:10262000C0F88030C0F89030C0F8A030C0F8C0309A
:102630004365C0F88430C0F89430C0F8A430C0F8C6
:10264000C43083668367C0F89830C0F8A830C0F8FB
:10265000B830C366C367C0F89C30C0F8AC30C0F86F
:10266000BC304FF03F430267C0F8B0204267C0F86B
:10267000B420C0F88820C0F8C820C0F88C200166BB
:1026800044668465C165C0F8CC304FF47A7121206E
:1026900048F06EFF4FF47A71222048F069FF4FF442
:1026A0007A71232048F064FFBDE810404FF47A713E
:1026B000242048F05DBF00BF000080BFF8B52DEDBD
:1026C000068B037B044643B90023C0F8D430C0F81E
:1026D000D830C0F8E030C0F8DC30D4ED371A94EDD3
:1026E000381AD4ED360A94ED350A8548DFED858A2F
:1026F00000F024FC5820B7EE001AFFEE000A94ED1B
:10270000350A19F0D3FF592084ED350AB7EE001AC7
:10271000FFEE000A94ED360A19F0C8FF5A2084ED46
:10272000360AB7EE001AFFEE000A94ED380A19F0E7
:10273000BDFF5B2084ED380AB7EE001AFFEE000AF9
:1027400094ED370A19F0B2FF84ED370A5FF08CFF81
:1027500007EE900A9FED6C7AF8EE677A04F11005A7
:1027600067EE877A2126C4ED027A2F46F7EE009AAB
:1027700094ED35AAD5ED100AB0EE680A6AEE200A8B
:1027800089F0D2FE94ED368AD5ED140AB0EE409A67
:1027900068EE200AB0EE680A89F0C6FED4ED385A19
:1027A000D5ED186A94ED376A95ED1C7A65EEA66A48
:1027B00079EE007AF0EEE66A26EE077A77EEA67AF0
:1027C000B0EEC77A77EE877AB5EEC09AE5EC017A7B
:1027D00095ED235AC5ED079A28EE058A95ED1F5A07
:1027E000AAEE058A95ED275AA5EE858AD5ED2B5AD6
:1027F000A6EE258AF1EE10FACCBF01230023B5EE38
:10280000C00A85ED038AF1EE10FA84F8D030C8BF13
:1028100094F8D030F5EEC06AC4BF013384F8D030EC
:10282000F1EE10FAC8BF94F8D030B5EEC07AC4BF4C
:10283000013384F8D030F1EE10FAC2BF94F8D030F2
:10284000013384F8D03094F9D030002BC1BF07EEAB
:10285000103AB8EEC77AC8EE076AC5ED036A95ED7F
:10286000038AB0EEC87A77EE877AF4EEE97AF1EE71
:1028700010FAC4BF79EEC77A45ED017A94F9E830D1
:1028800015ED019A83B1DFED217AB4EEE79AF1EE0E
:1028900010FA09D8DFED1E7AB4EEE77AF1EE10FAFD
:1028A000A4BF4FF08043EB6194ED390AD5ED077A70
:1028B00020EE270AD4ED027A20EE270ADFED157A02
:1028C00030EE000A20EE270A89F0A8FDA9EE008A62
:1028D00030B201369FED100A85ED0B8A28EE000A12
:1028E000B6B248F021FE252E7FF442AFBDEC068B38
:1028F00004F1200239460248BDE8F84000F050BB20
:10290000B025002000000000BD3786359A99193F98
:10291000CDCCCC3EDB0F494000007A440022C0F809
:10292000D420C0F8D820C0F8E020C0F8DC20FFF7A1
:10293000C5BE00000020704700207047012070478E
:1029400090F89C308B4286BF283150F8210000203F
:102950007047000090F89C308B4286BF283150F8B9
:102960002100002070470000FA207047014B93F8C7
:102970007A047047B0450020D0E90B3242F4E052AF
:102980000263426B43F4F84342F4E0524263C36291
:1029900070470000014802F04FBC00BFB025002086
:1029A00013B54FF44470CDE9002108F0CFFA044686
:1029B00028B1DDE9002146F07FF9024B2360204673
:1029C00002B010BDB0380A08704700007047000020
:1029D00000207047704700000020704770470000DB
:1029E000704700000320704708207047064BD3F85B
:1029F000F43E3BB11B7B002B0CBF5020D02040F09D
:102A0000010070475020FAE7B045002070470000F1
:102A1000014B93F87C047047B0450020034B93F9B9
:102A2000D004003818BF0120704700BFB045002017
:102A3000014B93F97E047047B045002070470000B9
:102A400010B52DED028B174BD3F8F44E3CB3D4EDFB
:102A5000360A94ED380AF0EEE00AB0EEC00A89F0CA
:102A600063FDD4ED370AB0EE408A94ED350AF0EEFE
:102A7000E00AB0EEC00A89F057FDF0EE400AB0EE71
:102A8000480A89F051FDDFED087A20EE270ABDEEF5
:102A9000C00A10EE103A18B2BDEC028B10BD2046F1
:102AA000FAE700BFB04500200000C84244F0FEBF76
:102AB00010B5044642F036FB054802F0BDFB054A5E
:102AC000034606212046BDE8104042F013BB00BF7C
:102AD000B025002000370A0841F002BC08B50846BE
:102AE00008F042F800280CBF0420002008BD0000B8
:102AF000162A01D041F034B903220A700120704730
:102B000010B44B7A8C7ACA7A43EA042343EA02432C
:102B1000863B012B03D95DF8044B45F0ABBE5DF855
:102B2000044B704708B541F077FB40F41C6040F05F
:102B30000D0008BD10B5044608F010FA204610BD7F
:102B400008B5094B93F8E02ED2060BD403F5805359
:102B5000D3F8880A03689B6A984700280CBF0220B4
:102B6000042008BD0120FCE7B0450020044B187884
:102B700020B9044B93F8E10EC0F38010704700BFFA
:102B80009C610020B04500201FB5002301930293F3
:102B9000039304F0E9FA01A904F0D4F828B101A8DC
:102BA0001CF0C6FA05B05DF804FB11F0ABFC90F820
:102BB000F432B02202FB030090ED3B0AF2E7000082
:102BC0000C4B93F879248AB9A3F5805393F8F12E2E
:102BD00051070BD193F8E02ED20609D493F8E13EC9
:102BE00013F0020F14BF0420012070470520704726
:102BF00003207047B05500202DE9F04F354F97F86E
:102C0000E43E012B8DB0044652D9334EDFF8E8A0E4
:102C1000082516F9018BB7F9A43408F1FF3B43FAF4
:102C20000BF3D90740D5207C3FF064FF8146207C20
:102C300040F064FE00F12103994505D2207C0DB0DF
:102C4000BDE8F04F3FF0D2B9BBF1070F2CD8DFE859
:102C50000BF03E04323436383A3C204B186959693F
:102C60005A6AD3F804B0D3F818E0D3F80CC0D3ED07
:102C7000007A1B6ACDF82520CDF829306222212365
:102C8000CDE9003207900891207CCDED037A19231D
:102C900003AAC221CDF810B0CDF814E0CDF818C0C9
:102CA0008DF824803FF090FF013D15F0FF05B0D175
:102CB0000DB0BDE8F08F0A4BD0E70A4BCEE70A4BC8
:102CC000CCE70A4BCAE75346C8E7094BC6E7094BAE
:102CD000C4E700BFB045002084390A08AC5B00207F
:102CE000BC5C0020345D0020BC5D0020E85D00205D
:102CF000D45F0020805B0020F85E0020094BD3F8F1
:102D0000D424920701D441F01FB803F5805303F592
:102D1000926393ED000ADFED047AB8EEC00A20EE6C
:102D2000270A7047B04500200AD7233C10B594B05D
:102D3000044603A807F010FE1A4BD3F8880A03686C
:102D400003A91B6B984750B3247C5FF099FC059B4B
:102D5000DDED047A0893069B09930023F8EEE77AE9
:102D60009FED117A0B930C930D930E930F93109389
:102D7000119312934FF6F853ADF84C30002396227E
:102D800067EE877A8DF84E303323CDE90032079015
:102D900007AA57212046CDED0A7A3FF015FF14B05F
:102DA00010BD00BFB05500200AD7233C014802F0F7
:102DB00041BA00BFB0250020014B93F8E40E7047E4
:102DC000B0450020024B93F8E10EC0F3400070477D
:102DD000B045002030B52DED028B154B91ED018AE9
:102DE0000546D3F8880A036885B0DB690C46984726
:102DF00028B9BDEEC88A18EE103ADB0712D5D4E91F
:102E0000040119F059FE68B1684607F0A5FD6A464D
:102E10002146284645F0A2F820B10649684607F049
:102E2000AFFE00B1022005B0BDEC028B30BD00BF8B
:102E3000B05500203C5A00208B8B162B05D0C02BA0
:102E400001D1FFF7C7BF46F03BBB00207047000031
:102E500030B52DED028B8DB000230546039304930E
:102E6000059304F081F903A903F06CFF58B304F053
:102E70007BF900F55A7393E8070006AC84E8070075
:102E8000DDED060A9DED070A2D7CF1EE600AB1EE3C
:102E9000400A89F0E5FC2046B0EE408A1CF048F973
:102EA000DFED0B7A089B0B93012228EE278A0C2377
:102EB000CDE90032A82109AA28468DED098A8DEDB9
:102EC0000A0A3FF081FE0DB0BDEC028B30BD00BFA1
:102ED000E02E6542242938B505460FD003D81B29BA
:102EE00007D1012412E04029FBD0A1F14203012BBC
:102EF000F7D92846BDE8384045F0EEB90C213FF03F
:102F000087F8044610B12846FFF7A2FF204638BDD7
:102F100008B591ED007AF6EE007AB4EEE77AF1EEBC
:102F200010FA06DD044801220521FEF793FD00207A
:102F300008BD0420FCE700BF1C5200202DE9F04131
:102F400088B080461B22002101A810EE107A10EEF6
:102F5000906A11EE105A11EE904A8BF067FEA3238F
:102F60008DF8043095238DF805300B238DF806304D
:102F70005FF08EFB1B22CDF80700CDF80B1008F593
:102F80008F5001A9CDF80F70CDF81360CDF8175010
:102F9000CDF81B403AF090F908B0BDE8F081000090
:102FA00070B58CB00D46144606462B22002101A8B0
:102FB0008BF03CFEA3238DF8043095238DF805306B
:102FC0000C238DF806305FF063FB2B68CDF80F30D3
:102FD0002368CDF813306B68CDF817306368CDF8EF
:102FE0001B30AB68CDF81F30A368CDF82330EB68F9
:102FF000CDF80700CDF80B10CDF827302B22E36871
:10300000CDF82B3001A906F58F503AF055F90CB0E8
:1030100070BD000070B500F58F5500F5565604469A
:1030200006F1500228460E213AF00AF806F17C0219
:1030300028460F213AF004F804F55C5228460C3279
:10304000102139F0FDFF04F55E52284604F55F5665
:103050000432112139F0F4FF06F14C0228466E21AA
:1030600039F0EEFF06F1780228466F2139F0E8FFCB
:1030700004F56552284608320D2139F0E1FF04F5C8
:10308000685228462432BDE870406B2139F0D8BF21
:103090001FB500F5A050002301A910300193029341
:1030A000039302F0C9FA05B05DF804FB08B504F01B
:1030B0005BF8BDE8084003F0F7BD00007FB50E46A1
:1030C0004FF6FF710446154602F09CF8E0B110225D
:1030D000002168468BF0AAFDA3238DF800309523CC
:1030E0008DF8013004238DF802305FF0D1FA102200
:1030F000CDF80300CDF8071004F58F5069468DF820
:103100000B6003953AF058F904B070BDA3207047E6
:1031100038B5044600F58F5502F08EF80C4902468A
:1031200028463AF065FA04F50053284693F8E52E50
:1031300093F8E41E3AF080FA04F5A050103004F041
:1031400023FA04F59070BDE8384010F045BA00BF8E
:1031500000370A0837B5069D044600B92C7801B936
:10316000697802B9AA7803B9EB78002064F3070004
:1031700061F30F2062F3174063F31F6003B030BDAB
:103180002DE9F04F2DED0C8B9DB0DC4C0D93D4ED63
:10319000379ADFEDDB5A90ED006A04F50054F7EE44
:1031A000006AD4F8F43ED3ED367A93ED387AF0EE37
:1031B000E77AB0EEC77A77EE877A9246F4EEE67A4F
:1031C000F1EE10FAC8BF86EEA78A06460F46DFED7D
:1031D000CD7AD8BFB0EE668A28EE277AA6EE257A99
:1031E00080ED007AD4F8F43E93ED357A93ED376AAA
:1031F000B0EEC77AB0EEC66A37EE067AB4EEE67A7B
:10320000F1EE10FACCBFC6EE878AF7EE008A90ED99
:10321000017A68EEA77AE7EE257AC0ED017A3BF0F5
:1032200043F805465FF034FA814618EE900A884666
:10323000FDF76AF9CDE9080118EE100AFDF764F907
:10324000CDE906017068FDF75FF9CDE9040130684A
:10325000FDF75AF9AC4BAD4ACDE90201CDE9009832
:103260002846AB49AB4D3AF04BFCAB4995ED00AA73
:1032700038461BF049FB8DED160A9AED000ACDED9C
:10328000170A30EE4A0A8DED181A19F0FBF904F20C
:10329000C4439DED167AD3ED007AB0EEC77AB4EE52
:1032A000E77AA5F21C63F1EE10FA0B9300F1298284
:1032B000D4F8F43E1B7B002B00F02382B4F8C294B8
:1032C000C9F340099DED177AB0EEC77AF4EEC77ADC
:1032D000F1EE10FA00F31882D4F8F43E1B7B002BB9
:1032E00000F01282B4F8C23403F001039DED187AA5
:1032F0000A93B0EEC77AF4EEC77AF1EE10FA00F353
:103300000582D4F8F43E1B7B002B00F0FF81B4F85B
:10331000C234C3F38008B0EEC00AF4EEC07AF1EE16
:1033200010FA00F3F681D4F8F43E1B7B002B00F07A
:10333000F081B4F8C234C3F3C00B0DAB00930A990B
:103340009FED768A5B4642464846FFF703FFC3B2CD
:103350000BEE103AC0F307230AEE903AC0F307438E
:103360000CEE903A030E0DEE103A9DF834300F90AB
:10337000002B40F0D1819DF83530002B40F0CC81FE
:10338000F8EE4B7A644ACDED197AF8EE6A7AB0EE2F
:10339000690ACDED1A7AF8EE6C7A19AB394602F566
:1033A0004670CDED1B7A55F0F3FB8DED140ACDED93
:1033B000150AB0EE409AF0EE608A9DF83630584C0F
:1033C000002B40F0AE8104F2BC431CEE901AD3ED0A
:1033D000000A97ED020AB0EE691A04F6181055F0CB
:1033E000F5FCB0EE40CA9DF83730002B40F09C81D0
:1033F0009AED000A30EE4A0A19F044F91DEE101A4F
:103400004848F0EE690A55F0C3F904F62423DAF8C7
:1034100000201A6004F62823F0EE40BA83ED00AADB
:10342000414D95ED001A4720F1EE410AB0EE490AF0
:1034300019F03CF92B46B3EC011AB0EE40AAF1EEBC
:10344000410A4820B0EE680A0C9319F02FF90C9B42
:1034500093ED001AB0EE409AF1EE410A4920B0EE29
:103460004C0A19F023F995ED021AF0EE408A4A2031
:10347000B0EE6B0AF1EE410A19F018F996ED007AF8
:10348000D6ED017A8DED148A6AEE076A04F595632C
:10349000CDED106A69EE276AF0EE40BACDED116A03
:1034A000D3ED006A8DED158A04F2AC4327EE267A3F
:1034B000D3ED006A9DF834308DED127A67EEA67A6E
:1034C000A5F59565CDED137A93BB9DF835307BBBA3
:1034D000B8EE4BBAF8EE6AAAB0EE690A13488DED61
:1034E00019BA19AB12AA10A9CDED1AAA55F01CFAF7
:1034F0008DED140ACDED150A1AE000BFB0250020AD
:10350000A4707D3F00D7233C453F0A08346C0A086D
:103510004D6C0A08CC3B0020645A002000000000DB
:10352000B0550020405F0020584A0020405B00203A
:103530009DF83630002B40F0FA8004F5966396ED46
:10354000000AD3ED000A924860EE200A1CEE901AA1
:1035500028EE800AB0EE691A55F038FCF0EE40AA69
:103560008C4814A9FEF742FE9DF83730002B40F03E
:10357000E18004F2C44396ED010AD3ED000A8648C7
:1035800060EE200AB0EE691A1DEE101A20EE2B0A2A
:1035900055F01CFCF0EE409AD5F8F43E1B7B7BBB4B
:1035A00019A97E488DED198A8DED1A8A55F006FB12
:1035B0009FED7B0A7B4855F025FC9FED790A7A4800
:1035C00055F010F919A979488DED198A8DED1A8AEF
:1035D00055F0F4FA9FED720A6D4855F013FC6E48F1
:1035E0009FED6F0A55F00EFC04F2B44393E8070018
:1035F0000B9B87E8070003F21C631B68CAF80030C6
:10360000B9F1000F00F09980D5F8F43E83ED368AC9
:103610000A9B002B00F09C80D5F8F43E83ED358AA0
:10362000B8F1000F00F09F80D5F8F43E83ED388AA2
:10363000BBF1000F00F0A180D5F8F43E83ED378A8E
:1036400004F59563D3ED002A9FED598A9FED544A06
:10365000D7ED000A04F2B44393ED001A62EE882A13
:103660002AEE082A21EE081A60EE880AF0EE443AA3
:10367000B0EE443AF0EE441AB0EE440A5DF038FE83
:1036800004F2AC43D3ED002A9FED454AD7ED010A81
:1036900004F5976393ED001A62EE882A29EE082A52
:1036A00021EE081A60EE880AF0EE443AB0EE443A91
:1036B000F0EE441AB0EE440A5DF01EFE04F5966387
:1036C00004F2BC449FED364AD3ED002A94ED001A73
:1036D000D7ED020A62EEC82A28EEC82A21EE481A5F
:1036E00060EEC80AF0EE443AB0EE443AF0EE441A06
:1036F000B0EE440A5DF004FE1DB0BDEC0C8BBDE8DD
:10370000F08F4FF00109DDE50123EFE54FF00108EF
:1037100001E64FF0010B10E6F0EE488AB0EE489A51
:103720004BE69FED1FCA5EE6DFED1DBA78E6DFEDE2
:103730001CAA15E7DFED1A9A2EE79DF83430002B0E
:103740007FF466AFD5F8F43E149AC3F8D8205FE74B
:103750009DF83530002B7FF463AFD5F8F43E159A11
:10376000C3F8D4205CE79DF83630002B7FF460AFBF
:10377000D5F8F43EC3ED38AA5AE79DF83730002B50
:103780007FF45EAFD5F8F43EC3ED379A58E700BF3B
:103790008C5C0020B0250020045D00207C5D0020B2
:1037A00000000000C85E0020405F0020405B002059
:1037B0000000C8422DE9F04F2DED068B8FB0C84CAC
:1037C0000393D4ED37AA04F500548046D4F8F43EB0
:1037D0001B7B0E461746002B00F04C81B4F8C254F8
:1037E000C5F3400B05F0010AC5F3800915F0080583
:1037F00000D0012503AB4A465146009358462B465C
:10380000FFF7A8FC04F5956393ED001A96ED000A06
:103810000590F1EE410A9A20029318F047FF029BAF
:1038200093ED001AF0EE409AF1EE410A96ED010A8E
:103830009B2018F03BFF04F2AC4393ED001AB0EE6E
:10384000409AF1EE410A96ED020A9C2018F02EFFF4
:1038500004F5966393ED001A9D20F0EE408AF1EE98
:10386000410A97ED000A18F021FF98ED007AD8ED93
:10387000017A9C4869EE876A0346CDED066A69EED7
:10388000276A0027CDED076AF3EC016A0A9727EE55
:10389000267AD3ED006A9DF80C308DED087A67EE3C
:1038A000A67AB0EE408ACDED097A0B97A0F5956621
:1038B000F3B99DF80D30DBB99DF8143007EE103ADE
:1038C0009DF8153007EE903AB8EE477AF8EE677A31
:1038D000B0EE6A0A0CAB08AA06A9E8308DED0C7AA6
:1038E000CDED0D7A55F020F88DED0A0ACDED0B0ADD
:1038F0009DF80E30002B40F0C28006F5966398EDDF
:10390000000AD3ED000A9DF81610774860EE200AF1
:10391000B0EE6A1A28EE800A55F058FAB0EE40AAC6
:103920006F480AA9FEF762FC9DF80F30002B40F0AB
:10393000A98006F2C44398ED010AD3ED000A9DF870
:1039400017106A4860EE200AB0EE6A1A20EE080AE4
:1039500055F03CFAB0EE408AD4F8F43E1B7B7BB9BC
:1039600063480C970CA90D9755F028F99FED610A53
:103970005D4855F047FA9FED5F0A5C4855F042FA02
:10398000BBF1000F00F08180D4F8F43EC3F8D8708A
:10399000BAF1000F00F08480D4F8F43EC3F8D4707C
:1039A000B9F1000F00F08780D4F8F43EC3F8E0705E
:1039B000002D00F08A80D4F8F43EC3F8DC7006F5E0
:1039C0009563D3ED002A9FED4C8A9FED4A4A06F29B
:1039D000B44393ED001A62EE882A29EE882A21EE7C
:1039E000081AF0EE443AB0EE443AF0EE441AF0EE23
:1039F000440AB0EE440A5DF07BFC06F2AC43D3ED22
:103A0000002A9FED3C4A06F5976393ED001A62EE9B
:103A1000882A29EE082A21EE081AF0EE443AB0EE80
:103A2000443AF0EE441AF0EE440AB0EE440A5DF077
:103A300063FC06F5966306F2BC469FED2E4AD3ED75
:103A4000002A96ED001A62EEC82A28EEC82A21EE56
:103A5000481AF0EE443AB0EE443AF0EE441AF0EE72
:103A6000440AB0EE440A5DF04BFC0FB0BDEC068B8F
:103A7000BDE8F08F4FF00109CA46CB46B9E69FED8D
:103A80001DAA4DE79FED1B8A66E79DF80C30002BC1
:103A90007FF47EAFD4F8F43E0A9AC3F8D82077E7D3
:103AA0009DF80D30002B7FF47BAFD4F8F43E0B9AD9
:103AB000C3F8D42074E79DF80E30002B7FF478AF64
:103AC000D4F8F43E83ED38AA72E79DF80F30002B4E
:103AD0007FF475AFD4F8F43E83ED378A6FE700BF0B
:103AE000B0250020585A00208C5C0020045D002086
:103AF000405B0020000000000000C84270B5044692
:103B0000143046F01DFA0B4E0B4B636164256019AF
:103B100046F0DEFB66513035B5F5597FF7D104F537
:103B2000597047F0CFFE2046044935F01FFE20466D
:103B300070BD00BF0C760A0820760A08D06E0A080D
:103B400037B500F5115101223831044638F0C2F87A
:103B5000184A1368D90706D4174904F50A533033B5
:103B60000B600123136004F51350134901220C303C
:103B7000012535F033FA114A0095002304F58F51E1
:103B8000FD2035F0D9F90E4B1A68D20705D40D4A3D
:103B90001D6004F59B54083414600A48012135F077
:103BA00039FA35F0E9FF084A138843F040031380DF
:103BB00003B030BD446100200022002004F70A0851
:103BC000486100200C220020586200200069C0F3E8
:103BD000401070470F299DBF302303FB0100503078
:103BE00000207047014B93F996047047B0450020C0
:103BF000024B93F8F10E00F001007047B045002031
:103C0000014BD3F8600C7047B0450020054A92F88C
:103C1000F13E92F8F02E03F0010313430CBF012094
:103C200000207047B0450020002910B517DB104C6C
:103C300094F8682CCBB29A4211D3D4F8643C012298
:103C4000595CA4F5005000F0AFFD94F8E13E38B99E
:103C50009A0704D5074A137843F00403137010BD84
:103C60009B07FCD5034A137843F00203F6E700BF35
:103C7000B0450020EC610020022A10B50F4C12D193
:103C80003522A4F5005000F08FFD94F8E13E9B072B
:103C900005D50B4B1A7818B142F002021A7010BD0C
:103CA00042F00402FAE794F8E42E8A42F7D146F093
:103CB000D9FABDE8104046F05FBA00BFB045002019
:103CC000EC61002010B500F50053DFED186AD3F861
:103CD000582CD3F8543CB2F90820B3F908309FEDC2
:103CE000147A07EE902AF8EEE77A0446C7EEA60AA1
:103CF00000F5A0500121103007EE903AF8EEE77A77
:103D000060EE870A87EEA60A20EE070A03F0B6FAED
:103D10003AF0CAFA26213AF05FF804F53250054A23
:103D2000BDE81040062138303DF040BF0000C842D9
:103D300035FA8E3C5C740A08332901D047F072B81A
:103D400070470000332910B519D0382913D0052940
:103D500017D1022A0DD10D4890F8E43E012B08D866
:103D6000D0F85C3CB3F908301BB9A0F50050FFF760
:103D7000A9FF012010BD0321FFF77EFFF9E7012114
:103D8000FAE7BDE8104046F0ABBD00BFB0450020EB
:103D900030B5044689B0684604F5A05506F0DCFD50
:103DA000103504A806F0D8FD6946284602F092FFB7
:103DB00060B104A9284602F0DDFF38B1059B0193EC
:103DC00023680022DB6C69462046984709B030BD65
:103DD00000F5805292F88C26D2070AD400F50052E2
:103DE000D2F8F42E117B09B1FFF7D2BF03689B6CA8
:103DF0001847704710B586B0044602A8019106F036
:103E0000ABFD04F5A05002A9103002F063FF28B109
:103E10002368019ADB6C02A92046984706B010BDC2
:103E2000F0B5044685B004F5A056684610360F4636
:103E3000154606F091FD6946304602F09BFF10B929
:103E4000002005B0F0BD3946304602F01FFE0028C4
:103E5000F6D0002DF5D004F58054284694F88C3621
:103E600043F0020384F88C36EBE7000010B500F550
:103E70001254D4ED087AF5EEC07AF1EE10FA8AB059
:103E80004FF0000304F1200444D9079308930993E9
:103E900006AB019300F5A05007AB03AA04A9009359
:103EA000103005AB02F08AFEDDED080A9DED070A31
:103EB00088F03AFBDDED090A88F036FBD4ED007A94
:103EC0009DED047A77EEA76AB4EEE70AF1EE10FAF8
:103ED000F4EEC76AACBF01200020F1EE10FA0CD856
:103EE00002309DED037AF4EEC77AF1EE10FA0CD8A9
:103EF000003818BF01200AB010BDF4EEC77AF1EE09
:103F000010FA9CBF0130C0B2EBE7012894BF00203B
:103F10000120F0E70020EEE738B500F50055044633
:103F200095F8F13E5A071AD443F0040385F8F13EA0
:103F30003AF0BAF90122112139F06EFF084BD3F89B
:103F4000880A03689B68984718B995F99D34032B34
:103F500005D120460621BDE8384000F01FBD38BD20
:103F6000B055002008B500F5005090F8F13E5A0712
:103F70000BD56FF3820380F8F13E3AF095F9BDE876
:103F800008400022112139F047BF08BD2DE9F04358
:103F9000054685B005F5A058684608F1100806F0FA
:103FA000DBFC6946404602F0E5FED8B105F500535A
:103FB000434CD3F8F42E434F127B42B103F5946384
:103FC000D3ED007AF5EEC07AF1EE10FA0DD8238821
:103FD00023F4FF7323F00103238028460023FB739F
:103FE000FFF7C0FF05B0BDE8F083284601F0C6F832
:103FF000064618B9284601F087F806462846FFF716
:1040000035FF814640B93EB12378002B41D163781A
:1040100003F00103FB73E5E76378DB07F7D423784C
:104020000133DBB2082B237006D12846FFF71EFFB1
:1040300010B1404602F02EFE2378092B02D14046F3
:1040400002F020FE2378092BE1D9238823F4FF73A3
:1040500023F0010343F4857323803AF025F902220B
:10406000102139F0D9FE5EF00BFB6368C01A47F2ED
:104070003053984209D905F53250134A022138309D
:104080003DF094FD5EF0FCFA60602846FFF744FFC7
:10409000BDE7013B23702388C3F30803B3F5807F9A
:1040A000B5D1637860F3000363703AF0FDF84A46D7
:1040B000102139F0B1FE2846FFF754FFA7E700BFF3
:1040C0004C610020CD6100203C760A0837B50446DB
:1040D00000F5A05001A9103004F5005502F0ECFBEA
:1040E000D5F8A43C834206D0C5F8A40C3AF0DCF81D
:1040F0003E2139F071FE04F5805395F9A81C93F820
:10410000202793F92037994213D0FF2A11D085F840
:10411000A83C3AF0C9F895F8A82C182139F07CFE93
:1041200004F5325095F9A83C034A042138303DF09B
:104130003DFD03B030BD00BF4C760A082DE9F043C9
:1041400095B006465EF09CFA06F5A05803AB0193C5
:1041500008F1100802AB0024009305460EAB0BAA31
:1041600008A94046089409940A940B940C940D9461
:104170000E940F94109402F00FFDDFED437A9DED45
:104180000A7AB4EEE77AF1EE10FA074637DB9DEDD6
:104190000D7AB4EEE77AF1EE10FAACBF4FF00109F8
:1041A0004FF0000907AB019311AB009304AA06ABD3
:1041B00005A9404611941294139402F0FFFC06F5F1
:1041C0000054002894F9483C08BF002783B17FB110
:1041D000D4F8F43E1B7B5BB1B9F1000F08D09DED24
:1041E000057AF7EE007AB4EEE77AF1EE10FA09D527
:1041F00094F8AC3C73B90023C4F8B03C0FE04FF026
:104200000009CFE7D4F8B00C20BBC4F8B05CC4F808
:10421000B40C04E0D4F8B40C20B9C4F8B45C15B004
:10422000BDE8F083281A43F698239842E3D9002585
:1042300084F8AC5CC4F8B45C3AF036F82A461D2128
:1042400039F0EAFD06F53250104A022138303DF0CF
:10425000ADFCD0E72D1AB5F57A7FE0D994F8AC3CE7
:10426000002BDCD1012584F8AC5C3AF01DF82A461D
:104270001D2139F0D1FD06F53250054A02213830B2
:104280003DF094FCCBE700BF0000003464760A08E0
:104290007F760A0810B504463AF006F80022052198
:1042A00039F0BAFD04F53250034ABDE8104004214C
:1042B00038303DF07BBC00BF9C760A0800F500500A
:1042C00090F8E13E9B065ABF90F8E00EC0F3001054
:1042D0000120704737B5044600F5555034305CF086
:1042E00031FD04F50052C0F3803592F8E13EC3F38E
:1042F0000011A9421DD065F3041304F5325482F86D
:10430000E13E38346DB139F0CFFF02220B2139F094
:1043100083FD094A0221204603B0BDE830403DF04C
:1043200045BC39F0C1FF2A460B2139F075FD034A1F
:10433000F0E703B030BD00BFB4760A08BF760A08C4
:1043400070B500F50055044695F98634B3B3D5F839
:10435000706E9EB35EF094F905F5456393ED000A27
:10436000DFED177A9FED171ADFED170A861B20EE97
:10437000270A6B2018F09AF9BCEEC00A10EE103A2A
:104380009E4209D295F8F13E9A0717D520460021A2
:10439000BDE87040FDF7F0BB10D995F8F13E9B07E2
:1043A0000CD420460121FDF7E7FB04F53150012232
:1043B000BDE8704012212C30FDF74CBB70BD00BF32
:1043C00000007A440000804F000000000B46012BE3
:1043D00010B4114604D0052B06D05DF8044B70478D
:1043E0005DF8044B00F0DABA00F531505DF8044B8B
:1043F000012214212C30FDF72DBB00002DE9F041E6
:10440000044604F5005839F04FFF0122052139F028
:1044100003FD98F98A542046003D18BF0125FFF797
:104420004DFF04F53256383698B11E4A0421304605
:104430003DF0BCFB04F53150012210212C30FDF77A
:1044400009FB0025294620460322BDE8F041FFF77D
:10445000BDBF04F54057D7F8880A03689B6A9847A0
:1044600068B197F8793453B197F97834012B06DCA9
:104470000D4A042130463DF099FB0125E2E7D7F8CB
:10448000880A03689B6A984718B1D8F84C3C1B0708
:1044900005D4064A042130463DF088FBD2E7044AA1
:1044A000E7E700BFD4760A08EF760A081D770A0806
:1044B0002C770A0870B50446154639F0F5FE01223E
:1044C000062139F0A9FC2046FFF7F8FE04F5325624
:1044D000383698B104F53150012207212C30FDF710
:1044E000B9FA154A042130463DF060FB0025294603
:1044F00020460422BDE87040FFF768BF04F5405332
:10450000EDB2D3F8880A03689B6A984768B104F54E
:104510000053D3F84C3C1B0707D535B1074A04219B
:1045200030463DF043FB0125E1E7054A04213046D2
:104530003DF03CFBDBE700BF50770A08F7760A083E
:104540006D770A08F8B504465EF08EF8284BB4F88B
:10455000BE201988274E914205460ED01A80264B60
:1045600018603378A3B10024347039F09DFE2246E0
:104570001321BDE8F84039F04FBC33781F4FC3B961
:104580003B782BB11C4B1E4A1B68C31A934200D8C0
:10459000F8BD0123337004F50053D3F8F40E037B08
:1045A0000BB1FEF7BBF939F07FFE0122132139F080
:1045B00033FC3B78002BEBD03378002BE8D00E4A4D
:1045C00010491368EB1A8B42E2D904F500541560C8
:1045D000D4F8F42E137B002BDAD0002313730A4A8D
:1045E000D4F8F40E1371BDE8F840FEF767B800BFC9
:1045F0005661002054610020586100205561002060
:1046000080841E0040420F00CD61002070B500F58F
:10461000005300F55555343586B093F8AC1C04466C
:1046200028465CF03DFB02A806F096F904F5A05080
:1046300002A9103002F04EFB04F54053049AC3F86F
:104640009424059AC3F8982428465CF07BFB8206E4
:104650001AD528465CF080FB04F55255FDEEC07A71
:104660000C3504F5805417EE901A0222284617EEF6
:10467000906A06F077F994F88C36DB0706D40122AD
:104680003146284606F06EF906B070BD0121284675
:1046900006F02CFA0028F2D0F6E70000012070475F
:1046A00000207047002070470020704700207047AE
:1046B000002070470020704700207047002070479E
:1046C0009FED010A704700BF000000007047000026
:1046D0000F4A02600F4A426002F1540181600E49A4
:1046E000C1600E49016102F67C21416102F5286139
:1046F000816102F2DC71C16102F5FC61016202F2CA
:10470000E47102F5FD628262054A4162C26270474D
:10471000F8770A08284A0020245B0020C0390020CE
:10472000C8260020042917D8DFE801F003070B0F83
:10473000130000F56A503C30704700F56A500C30A9
:10474000704700F56B502C30704700F56C501C30F2
:10475000704700F56D50FAE70020704700F54050B3
:10476000D0F8880A03685B681847000038B500F580
:1047700040550446D5F8880A03685B699847094B99
:1047800004F50052187492F8E42ED5F8880ADA700D
:1047900003685B6A9847014604F59E50BDE83840BF
:1047A00032F012B9CD6100202DE9F84F00F5005A22
:1047B00006469AF8E43E8B420F46914605D18AF8A8
:1047C000E52E01252846BDE8F88FFFF7ABFF04462C
:1047D00020B9304637F004FD2546F3E7DAF8F43E19
:1047E0001B7B06F5325883F0010B08F13808E3B95A
:1047F000236859461B6820469847054678B306F556
:1048000040534A46C3F8884A394606F58F508AF81D
:10481000E47E8AF8E59E38F00FFF4046002144F020
:1048200027FE3046FFF7A2FFCCE703689B68984756
:10483000E0B11C4800F08CFC0546B8B9236820465E
:104840001B6A9847184A0346042140463DF0AEF9DA
:1048500039F02AFD3A460A2139F0DEFAB2E7236838
:1048600020461B6A9847114A0346EDE70D4800F0C1
:104870008DFC0028BCD106F54053D3F8880A0368A4
:10488000DB6898470028B3D023682046DB68984748
:1048900005460028ACD1236820461B6A9847044A85
:1048A0000346D1E7B025002080770A08D2770A08AE
:1048B000A9770A080148FFF777BF00BFB02500209D
:1048C00070B5234B93F8F13EDB0705460C461646C0
:1048D00005D5002363602360A360336070BD45F09D
:1048E000C1FC037F002BF4D0EB699FED1A7A1B68A3
:1048F000B3F9083007EE903AF8EEE77AC7EE876A28
:10490000C4ED016A2B6A1B68B3F9083007EE903AD0
:10491000F8EEE77AC7EE876AC4ED006A6B6A1B6837
:10492000B3F908305B4207EE903AF8EEE77AC7EE4B
:10493000876AC4ED026AAB6A1B68B3F9083007EEF8
:10494000903AF8EEE77AC7EE876AC6ED006AC5E7E7
:10495000B045002000007A440020704701207047D5
:104960000020704700207047004870473C780A08D4
:10497000004870473C780A0843691A680023C2F867
:10498000D43042691268C2F8D83042691268C2F85D
:10499000DC3042691268C2F8E03070470A4608B558
:1049A0000021FFF701FF034A137843F00803137057
:1049B00008BD00BFEC610020012070470020704757
:1049C00001207047002070470048704790780A081F
:1049D0000048704798780A0830B5084B03F55252E2
:1049E0003432044600F1300507CA85E8070003F5B4
:1049F000B0531C3301201B68E36330BDB025002099
:104A000030B52DED028B044687B05A4D002301AA24
:104A100003A995ED378A039304930593FFF750FF9D
:104A200063689DED037AD3ED0F7A68EE277A27EE5F
:104A3000277A8DED037A9DED047A67EE277ACDED26
:104A4000047AD3ED107A28EE277ADDED057A67EE49
:104A5000877ACDED057AD3ED117A93F9483028EEB7
:104A6000278ADDED017A27EE888A8DED018A1BB950
:104A700003A92846FDF7A2FB3F4B94ED0C7AD3ED3A
:104A8000007A626894ED0F0AD2ED0F6A77EE677ACA
:104A9000A3F2B443F0EEE77AF4EEE67AF1EE10FA20
:104AA00044BFDDED037A77EE877A03F5976148BF5F
:104AB000C4ED0C7A94ED0D7AD1ED007AD2ED0F6A47
:104AC00077EE677A03F2BC43F0EEE77AF4EEE67A2B
:104AD000F1EE10FA44BFDDED047A77EE877A94EDBB
:104AE0000E7A48BFC4ED0D7AD3ED007AD2ED106A8C
:104AF000236977EE677AF0EEE77AF4EEE67AF1EE84
:104B000010FA42BFDDED057A77EE877AC4ED0E7AB2
:104B1000D3ED837A30EE670A17F0B4FD6368D3ED06
:104B2000117AB0EEC00AB4EEE70AF1EE10FA09D538
:104B300094ED0F0ADDED017A30EE270A17F0A2FDA1
:104B400084ED0F0A00230D488DF808308DF80930E8
:104B50008DF80A308DF80B30029BD0F8F80E04F176
:104B60003C0204F13001FEF70BFB07B0BDEC028BF9
:104B700030BD00BFB0250020645A0020B0450020A1
:104B800000207047012070470120704700207047C7
:104B900000487047EC780A0800487047F4780A0823
:104BA0001FB5044600236A4601A9019302930393AB
:104BB000FFF786FE6369029A1B68C3F8D420636915
:104BC000019A1B68C3F8D8206369009A1B68C3F870
:104BD000DC206369039A1B68C3F8E02004B010BDB1
:104BE0000120704700207047012070470020704767
:104BF00000487047AC440A0800487047AC440A08B3
:104C0000012070477FB5002303930493059301931C
:104C1000094800238DF808308DF809308DF80A30E6
:104C20008DF80B30029BD0F8F80E01AA03A9FEF70D
:104C3000A7FA07B05DF804FBB045002001207047DB
:104C400000207047012070470020704700487047DF
:104C500094790A0800487047A0790A0810B50446FC
:104C600086B0002301AA03A9039304930593FFF7D9
:104C700027FE63689DED037AD3ED0C6ADDED047ABF
:104C800093F9483027EE267A67EEA67A8DED037AFF
:104C9000CDED047A1BB9144803A9FDF78FFA6368B8
:104CA000DDED057A93ED0D7A104867EE877A93ED86
:104CB0000E7ACDED057ADDED017AD0F8F80E0023FD
:104CC00067EE877A8DF808308DF809308DF80A3054
:104CD0008DF80B30029BCDED017A01AA03A9FEF7F6
:104CE00069FD06B010BD00BFB0250020B045002012
:104CF00038B5044646F03AFE46F00CFF04F5005481
:104D0000054646F09DFE46F029FBD4F8F40EFDF76B
:104D1000D5FC2846BDE8384046F09ABE70B500F58F
:104D20000055044695F97C3C43B1D5F85C2C344ED3
:104D3000B2F90820002A02DD0023338070BDD5F8C7
:104D4000602CB2F90820B2F5617F31DDB6F9003090
:104D5000642BDCBF01333380B6F90030142B0DD146
:104D6000D5F8F43E197B0029E8D100F53150012235
:104D70002C30FCF7D5FD08B93080DFE7B6F90030FC
:104D8000642BDBD1D5F8F43E1B7B002BD6D095F8F5
:104D9000E43E012BD2D104F532501A4A06213830B4
:104DA00004F540543CF002FFFA23A4F87C3AC5E72E
:104DB00012F5617FC0DA022BBED100F54053D3F863
:104DC000880A0368DB68984718B995F8E03EDB0667
:104DD000B2D5B6F90030142BB0DC01331BB2142B62
:104DE0003380ABD1D5F8F43E1B7B002BA6D004F565
:104DF00031500122BDE8704000212C30FCF72ABE62
:104E00005C610020F4790A0810B500F50054142103
:104E1000D4F8540C45F070FAD4F8580C142145F02D
:104E20006BFAD4F85C0C1E2145F066FAD4F8600CDD
:104E3000142145F061FA45F015FA036805211B6855
:104E40009847BDE81040002145F056BA38B50546F0
:104E500045F008FA45F0DEF905F50054C4F8540CA5
:104E600045F000FA45F0E0F9C4F8580C45F0FAF9BD
:104E700045F0E4F9C4F85C0C45F0F4F945F0E8F9C4
:104E80004FF47A71C4F8600CD4F8540C45F030FA41
:104E9000D4F8580C4FF47A7145F02AFAD4F8600C23
:104EA0004FF47A7145F024FAD4F85C0C4FF47A711F
:104EB00045F01EFA2846FFF7A7FF94F8E13E43F0BD
:104EC000080384F8E13E38BD08B546F023FE46F0FD
:104ED000C7FBBDE8084046F079BB000000F5005074
:104EE000D0F8F40EFDF71ABD38B500F500540546AC
:104EF00094F98A34BBB1B4F88C348B421DD994F840
:104F0000F13EDA070FD445F0ADF9037F1BB9D4F8B1
:104F1000F43E1B7B3BB194F8F03E01335BB2022BB5
:104F200002DC84F8F03E38BD032384F8F03E012112
:104F30002846BDE83840FCF705BE94F8F03E013B3A
:104F40005BB2002BEDDC94F8F13E0021DB0784F826
:104F5000F01EE8D5EDE7000038B50D4604465DF0DB
:104F60008FFB002D0B4B09DD04F50054186094F8FD
:104F7000E13E6FF3C30384F8E13E38BD1B68C01AFD
:104F8000B0F5C87FF9D904F5005494F8E13E43F038
:104F90000803F0E760610020F7B504465DF070FBA0
:104FA000064645F05FF945F005F804F50055A8B34D
:104FB00095F8E03E43F0200385F8E03ED5F85C3CF0
:104FC0002046D988FFF790FFD5F85C3C04F54057A0
:104FD000B3F908102046FFF7BFFFD7F8803A9FEDDE
:104FE000267AF31A07EE903AD5F85C3CF8EE677A29
:104FF000B3F9083067EE877A6A46CDED007A07EE9E
:10500000903AF8EEE77A01A904F55250CDED017A15
:105010003BF0A6FEC7F8806A03B0F0BD95F8F13EFC
:10502000DB07F9D404F54053D3F8800A361A45F06B
:105030004BF8002814BF4FF47A734FF4FA73B3425D
:10504000EAD895F98A34002BE6D045F00BF9037FB6
:1050500023B9D5F8F43E1B7B002BDDD039F024F9C1
:105060000222114638F0D8FE0121204603B0BDE8E7
:10507000F040FCF767BD00BF6F12833A38B50446B5
:1050800000F58C65284604F071FA94F871049FEDE0
:10509000097A242202FB0055D5ED0B7A67EE877A58
:1050A00004F54053FDEEE77A17EE902AC3F87C240E
:1050B00038BD00BF0000C842FEF72AB80148FFF71C
:1050C00041BA00BFB025002038B500F5A055103515
:1050D0000446284600F01EFD04F58053022283F8A2
:1050E0002426B4F9A43004F6C8001BB9B4F8A230E1
:1050F000A4F8A430B4F8A41016F060FE2846BDE869
:10510000384000F001BE000013B5044600F5A05081
:10511000103000F003FF98B104F5555004F5005429
:1051200034305BF00FFED4F8F42E0190127BC3B242
:10513000C0F3001032B918B99DF80500C0F3400063
:1051400002B010BD0028FBD083F08000C009F7E753
:1051500038B500F50053054693F8F13E5B070AD4D5
:10516000FFF7D2FF044620B905F5A050103000F03B
:10517000D5FE204638BD0024FBE7000008B500F549
:10518000A050103000F0CAFE002008BD13B5044640
:1051900000F5A050103000F0C1FE58B104F5555094
:1051A00034305BF0CFFD4207C3B203D5C3F34010E8
:1051B0009B0600D4002002B010BD000038B500F5F9
:1051C0000055044695F8E03E590719D5D5F8F43E48
:1051D0001B7B2BB920460021BDE83840FCF79CBC66
:1051E00000F54053D3F8880A0368DB68984738B164
:1051F00095F8E13E1A0703D595F8F13EDB07E9D5AE
:1052000038BD000037B500F58F55044604F500544D
:105210002846019138F070F994F8E03E019960F366
:10522000C303284684F8E03E03B0BDE8304038F0C0
:1052300061BE00000720704700487047047A0A08E2
:1052400037B5154BB3F9A42005461AB9B3F8A22017
:10525000A3F8A420B3F8A4100191EC2005F076FE89
:10526000044610B10199FDF7C9F905F50050C0F8E1
:10527000F44E24B990F9DC14084805F02DFB0849D8
:10528000204634F081FC012034F00EF903B0BDE873
:10529000304034F071BC00BFB02500200C7A0A0801
:1052A00090360A08F7B5044600F59E5031F058FBD9
:1052B0002046FFF75BFA04F53C50083004F006FE88
:1052C00004F59850103004F58C6746F0EBFD384635
:1052D00004F082FC04F53250383040F055FE6C4E3C
:1052E0002046FFF7B3FD2046FFF7AAFFB6F9A4302A
:1052F0001BB9B6F8A230A6F8A430082005F026FEA7
:1053000018B14FF07E530360436004F50055C5F8B3
:10531000F80E44F0A7FF9922292145F05FFF44F0E1
:10532000A1FF44F047FF2046FFF7CEFD95F8E13E90
:1053300004F59C5043F0400385F8E13E0C3049F001
:1053400081FA544B54491B68986A03684FF47A7287
:10535000DB6A98470423C4F8A43104F590700DF07B
:1053600089FD06F06BFB4FF40053036306F066FB08
:1053700007F02AFC8023C4F874340121384604F075
:1053800005FA464B0193009602AB13E9060004F5BB
:105390008F5037F069FF2046FFF796FE4FF4002349
:1053A000C4F8B83DD5F8F40EFDF732F904F53150E4
:1053B00001212C30FCF7B8F810B12046FFF78EFD24
:1053C000B4F9A43004F5535008301BB9B4F8A23036
:1053D000A4F8A430B4F8A420D5F8F43E00EE102AC6
:1053E000D3ED390AB8EE400AF2EE0E1AB6EE001A04
:1053F0003CF0B8F9B4F9A43004F554500C301BB9A2
:10540000B4F8A230A4F8A430B4F8A420D5F8F43E3F
:1054100000EE102AD3ED390AB8EE400AF2EE0E1A69
:10542000B7EE001A3BF0B2FFB4F9A43004F55550C2
:105430001BB9B4F8A230A4F8A430B4F8A420D5F86D
:10544000F43E00EE102AD3ED390AB8EE400AF2EE2F
:105450000E1AB1EE041A3BF099FF95F897141A2230
:105460002046FFF7A1F960B9212201212046FFF76C
:105470009BF995F8E13E43F0020385F8E13E03B065
:10548000F0BD074A137843F008031370F1E700BF3B
:10549000B025002040610020BD500108B95001082E
:1054A000EC6100207047000000207047704700004A
:1054B0000020704700207047002070470020704790
:1054C0009FED010A704700BF000000009FED010A38
:1054D000704700BF000000007047000000207047C8
:1054E0007047000010B50446143000F019F804F1BC
:1054F0002C0000F015F804F174005DF0CDF804F113
:10550000F4005DF0C9F84FF0FF33C4F85031204685
:1055100010BD0000014B1868704700BF6461002097
:1055200070470000F0B52DED048B91B004466D4638
:10553000284605F011FA94F8BC33002B72D004F51C
:105540007A730FCB85E80F0094F8F833D4EDEC8A2A
:1055500094EDED8A94EDEE9A002B63D094F8D0335D
:10556000002B5FD02D22002104A8D4F8C073D4F8FA
:10557000C463D4F8C853D4F8CC4389F057FBA323B1
:105580008DF8103095238DF8113046238DF81230A8
:105590005DF07EF89FED250A9FED257ACDF8171076
:1055A00068EE807ACDF8130067EE877AFDEEE77A31
:1055B00017EE903A68EE007A29EE000A67EE877AD5
:1055C000ADF81B30FDEEE77A20EE070A17EE903AB1
:1055D000ADF81D3017F02AF8DDED017A9FED157A50
:1055E000CDF82D70BCEEC00AF8EEE77A10EE103A56
:1055F00067EE877AADF81F3017EE903ACDF821307C
:10560000029BCDF82530039BCDF82930CDF83160D1
:10561000CDF83550CDF8394038F046FE2D2204A99A
:1056200037F04AFE11B0BDEC048BF0BDE02E6542B0
:105630000000C8420AD7233C30B52DED028B8BB059
:10564000044624220D4601A8002189F0EFFAA32385
:105650008DF8043095238DF8053048239FED1F8A7F
:105660008DF806305DF014F8D4ED817A2B68CDF812
:105670000F3067EE887A95ED020ACDF80B1017EE21
:10568000903AD4ED827ACDF8133067EE887A6B6861
:10569000CDF8173017EE903ACDF80700CDF81B3053
:1056A00016F09AFF10EE103A94ED830ACDF81F30F1
:1056B00020EE080A16F090FF10EE103ACDF82330D5
:1056C00094F80C338DF8273038F0EEFD242201A930
:1056D00037F0F2FD0BB0BDEC028B30BDE02E654221
:1056E00030B587B014460D4618220021684689F06F
:1056F0009DFAA3238DF8003095238DF801304923BE
:105700008DF802305CF0C4FFA3680393E368049350
:105710006368CDF807100593CDF803008DF80B50A2
:1057200038F0C2FD1822694637F0C6FD07B030BD1B
:1057300010B58EB0044602A805F00EF902A9204665
:1057400001F0C8FA002845D001F00EFD694601F0CD
:1057500047F91F22002106A889F068FAA3238DF8D3
:10576000183095238DF819304A238DF81A305CF0E3
:105770008FFFDDED037A9FED1B7A049BCDF823307C
:10578000F8EEE77A059BCDF8273067EE877ACDF8FB
:105790001B0017EE903ADDED007ACDF82B30F1EEDC
:1057A000677A17EE903ACDF81F10204601A9CDF880
:1057B0002F3000F01DFC78B1DDED017AF1EE677A53
:1057C00017EE903ACDF8333038F06EFD1F2206A95F
:1057D00037F072FD0EB010BD38F066FDDFED027AD5
:1057E000EEE700BF0AD7233C5241C07F002303608D
:1057F00043608360C360036143618361C36103628B
:105800007047000090F8F432B02202FB030390F8D6
:10581000382393F8D13012B1012B28BF0123184649
:10582000704700002DE9F04F04468BB04FF0000A9E
:105830000D461AF0AFFD84F814A204F506704FF07F
:105840007E575BF0EDFD4FF47A73A4F8623284F872
:105850006852C4F84872C4F84C72C4F8507204F527
:105860001B70002505F078F804F52B790323C4F8A4
:10587000803204F53476C4F89452C4F89852C4F8CF
:105880009C52C4F8A052C4F8A452C4F8A852484686
:10589000FFF7ACFF04F5487B3046FFF7A7FFC4F8DD
:1058A0001453C4F81853C4F81C535846FFF79EFF0E
:1058B000C4F84453C4F84853C4F84C53C4F8505384
:1058C000C4F85453C4F85853C4F85C53C4F8605334
:1058D000C4F86453C4F86853C4F86C53C4F87053E4
:1058E000C4F88C53C4F89053C4F89453C4F8A85324
:1058F000C4F8A453C4F8A053C4F8B053C4F8B453C4
:10590000C4F8B853C4F8CC53C4F8C853C4F8C4534B
:10591000C4F89C73C4F8C07304F5757005F01CF8E6
:1059200004F57A7005F018F804F58063C4F8FC53A8
:105930001D6004F5816304F583601D605D609D60FA
:1059400005F00AF804F22C4304F264481D605D601F
:105950009D606D4BC4F83C3404F50D73C4F84034BD
:1059600004F50E73C4F8443404F50F73C4F84834D6
:1059700004F51073C4F84C3404F24523C4F85034D1
:1059800004F51173C4F8543404F58B6340461D606C
:105990005D609D60FFF72AFF04F59160FFF726FF29
:1059A00004F5976304F23C421D605D609D6004F263
:1059B000C44304F2BC501D605D609D6004F59A63B1
:1059C0001D605D609D6004F2DC431D605D609D6054
:1059D00004F2EC431D605D609D6004F2FC431D60B9
:1059E0005D609D6004F5A1631D605D609D6004F2D3
:1059F0002C53C2F8E070C2F8E4701D605D609D60D9
:105A000004F5A7631D605D609D6004F244531D6052
:105A10005D609D6004F5AC631F605D6004F28453BB
:105A20001D605D609D6004F5B2631D605D609D60FA
:105A300004F5B5631D605D609D6004F08DFF04F2A8
:105A4000CC5324221D605D6004F2D45351461D6086
:105A50005D6004F2DC5340461D605D6089F0E6F84D
:105A600004F2FC50C8F82070C8F81070C8F8007034
:105A7000FFF7BCFE04F5C46304F5CA601D605D60F9
:105A80009D6004F22C631D605D609D6004F5C7633A
:105A90001D605D609D6004F244631D605D609D60FB
:105AA00004F05AFF194B1A491C60204633F05EFE81
:105AB00051462422584689F0B9F8C4F84073C4F816
:105AC0003073C4F8207304F5257207CA04F52873EF
:105AD00083E80700484694EDAA1AD4EDA90A94ED8C
:105AE000A80A17F0DBF93546494668466E4617F0B6
:105AF000F7F80FCE0FC50FCE0FC533682B602046C9
:105B00000BB0BDE8F08F00BF807C0A086861002000
:105B1000487B0A0810B5044688B001F0F1FB94F9FF
:105B20003232012B02D1274804F0F4FE022B0AD1B5
:105B3000032384F8323204A9012304F111008DF803
:105B4000103034F0DBFB94F8323284F8903204F2F7
:105B50003C4001F049FB94F93132642B30D165238C
:105B600004A904F231208DF8103034F005FC04A9AA
:105B7000204632F065FF18B304238DF81830002357
:105B8000CDE9013303930F230593694604A833F04D
:105B9000D7F8059B28B108AA02EB8302009942F8C6
:105BA000581C0133112B0593EFD959F0D5FD9DED0C
:105BB000031ADDED020A9DED010A652159F08AFD07
:105BC00008B010BD2C7A0A0870B500F5257600F5EE
:105BD00028758CB004463146284618F035FEE0B9E9
:105BE00096E8070085E8070004F52B7194EDAA1AE2
:105BF000D4EDA90A94EDA80A0191084617F04EF9D0
:105C000002AD019902A817F06BF80FCD04F53474BA
:105C10000FC40FCD0FC42B6823600CB070BD000003
:105C200013B540F2411200F50671044601A812F0C6
:105C30007BFD04F23C4001F001FD20461AF0F2FD2C
:105C400001A812F093FD02B010BD0000F8B50B687A
:105C5000C0F804324B68C0F808328B68C0F80C32C8
:105C600001F10C0607460C4600F548750FCE0FC52E
:105C70000FCE0FC533682B6004F1300207CA07F559
:105C8000457383E8070004F13C0207CA07F5517326
:105C900083E8070004F1480207CA07F5547383E854
:105CA0000700543494E8070007F5577383E80700AA
:105CB000384601F039FC3846BDE8F84001F01CBC1C
:105CC00013B5044600F23C40019003F0FFF804F5E0
:105CD000BE610198009102F009FC0099204602B0D3
:105CE000BDE81040FFF7B2BF4A78064BC2F340123E
:105CF0001A754A78C2F380125A750A78C2F30012F4
:105D00009A757047CD61002013B540F2F522044624
:105D100000F5067101A812F007FD002104F23C40D5
:105D200001F000FF94F8603223B120461AF096FF8C
:105D300084F8600201A812F019FD02B010BD000045
:105D400038B590F80C3305460C462BB1032B0BD01D
:105D500095F86832DB070CD405F5CA630FCB84E8ED
:105D60000F0095F8600603E01AF0DCFD0028EFD084
:105D700038BD0020FCE7000000F23C4090ED380AFE
:105D80007047000000F23C4090ED390A7047000077
:105D900010B490F80C230C462AB1032A0AD0002034
:105DA0005DF8044B704700F5B56007C884E807004C
:105DB0000120F5E75DF8044B1AF072BD90F88403FA
:105DC000431E58425841704738B590F80C330D4681
:105DD0008BB900F23C4001F0A3FC044610B900244A
:105DE000204638BD01F0F0FBD5ED007A27EE800AA1
:105DF00085ED000AF4E7D0EDE07AC1ED007A90F885
:105E00007C43002CEBD090EDDE7ADFED086AB4EE37
:105E1000E67AF1EE10FAF7EE006AB8BFB0EE667AF5
:105E200067EE877AC1ED007ADAE700BF0000003440
:105E300090F80C33032B01D11AF0B2BC002070474C
:105E400090F80C23032A01D11AF030BE00F23C4036
:105E500002F0CAB830B590F80C3385B004460D4650
:105E60008BB1032B18D004F5257018F027FD2846B8
:105E700001A98DED010ACDED020A8DED031A18F08E
:105E8000AFFA012006E000F23C4001F0F3FB0028ED
:105E9000E9D1002005B030BD90F86032002BF8D079
:105EA0001AF0DEFDDFE700007FB590F80C2332B179
:105EB000032A4FF0000309D0039304930CE000F28F
:105EC0003C4007B05DF804EB01F0B0BC03A90393BC
:105ED000049305931AF05AFC9DED030ADDED040AC4
:105EE00007B05DF804FB000007B590F80C3333B140
:105EF00000F57F7003B05DF804EB18F009BC00F208
:105F00003C4001F093FC68468DED000ACDED010A9E
:105F100018F0FEFB03B05DF804FB000090F80C03E2
:105F2000003818BF0120704708B590F80C23032AE9
:105F300005D0BDE8084000F23C4001F05FBC1AF01B
:105F400025FC012008BD000010B590F80C230C467C
:105F50001AB1032A07D0002010BDBDE8104000F29E
:105F60003C4001F0EFBB1AF027FC012084ED000A51
:105F7000F2E7000090F80C33032B01D11AF030BD8A
:105F80000020704730B590F80C3385B005460C46BC
:105F900023B1032B09D0002005B030BD00F23C40F6
:105FA00005B0BDE8304002F0D1BA002302A9029347
:105FB00003931AF0D3FB0028EDD001A928461AF06C
:105FC000D9FB0028E7D0029B2360039B6360019B01
:105FD000A360E1E790F80C231AB1032A05D0002052
:105FE000704700F23C4002F0E5BA1AF0B7BB00007F
:105FF00090F80C231AB1032A05D00020704700F254
:106000003C4002F0C9BA1AF0B5BB000090F9323238
:106010003BB990F8683213F0010F14BF0320002041
:106020007047032070470000F7B50446FFF7EEFF06
:106030000546002862D0032839D194F860326BB34A
:1060400094F86832D8072BD501A920461AF038FFFA
:10605000BDF80430002B18BF002594F8146206F038
:10606000FD06012E4AD10023032D019307D101A97A
:1060700020461AF031FF20461AF030FD064604F2A1
:106080003C4002F015FB08B994F809039DF8043070
:10609000D90703D55A0701D59F0632D400252DE034
:1060A00020461AF0CBFA002808BF0025D5E70025C6
:1060B000D3E713F0020F2EE094F9443223B99DF890
:1060C0000430DB092FD0E9E7002EF8D00EF01AFAE1
:1060D000FFF798FB022807D99DF805309806DDD513
:1060E0009DF80430D906D9D5FB6A93F89C30002B73
:1060F000E5D118E0DA0601D41B0718D5284603B00D
:10610000F0BD0028FAD094F80923B4F96436002AC7
:10611000CFD013F0010FF1D1154B1F68FB6A93F834
:106120009C30002BC8D19DF804309C07E2D405F0C8
:1061300085FC05F081FB0028B0D10EF0E3F9FFF7F4
:1061400061FB0228AAD90EF0DDF990F8F432B022F2
:1061500002FB030090ED3B7AF0EE007AB4EEE77AB2
:10616000F1EE10FA9AD59DF80530DB09C6D195E716
:10617000406100202DE9F04790F8603292B004466B
:10618000002B00F0948020461AF0E6FF2046FFF72F
:106190004BFF03287BD104F5487800274146204671
:1061A0000097019702971AF031FC694620461AF0D1
:1061B00023FC009BC4F80432019BC4F80832029B04
:1061C000C4F80C32204601F0AFF9204601F094F9F2
:1061D00015F04EFD054620461AF0B2FA0028A8BF79
:1061E000C6B203AA4FF0FF312046BCBF95F8EB942E
:1061F00095F8EC640397A8BFB146049705971AF089
:10620000E9FA03A818F05AFB4FF00C0A0AFB0950F0
:1062100084EDD10AC4EDD20A84EDD31A04F551718C
:1062200000F55C7018F05AFB04F557770AFB065529
:1062300084EDC50AC4EDC60A84EDC71A3A464FF08C
:10624000FF31204605F500751AF0D8FA95E80700E9
:1062500006AE86E807003946304618F0A5FB04F57F
:106260002B72414609A816F0CBFC314609A816F05E
:1062700049FC09A9204684EDD40AC4EDD50A84ED71
:10628000D61A1AF029FE09A92046FFF72DFD94F829
:106290006636002B3AD109A804F05EFB09A9204616
:1062A0001AF04CFB90B3012384F866362EE0D0F848
:1062B00064321BB95CF0E4F9C4F86402154B1B6846
:1062C000D86A03685B68984788B15CF0D9F9D4F85C
:1062D0006432C01AB4F86232984204D920461AF0E7
:1062E000BDFC84F8600294F860327BB14BE75CF04F
:1062F000C7F9D4F86432C01A41F287339842E4D81F
:1063000037F0D2FF37F012FE0028DED112B0BDE820
:10631000F08700BF4061002090F80C3323B1032BBD
:106320004FF0000007D0704790F93222032A04D1C1
:106330000A70012070470870FBE71846704700009C
:1063400073B50D460DF107010446FFF7E5FF06465C
:1063500028B19DF807302BB1032B09D00026304619
:1063600002B070BD04F5CA630FCB85E80F00F6E7F5
:10637000294620461AF0D6FA94F86062EFE700004A
:106380007FB50E460DF103010446FFF7C5FF054634
:1063900018B90025284604B070BD9DF8033083B1BC
:1063A000032B16D004F5257018F088FA01A93046A1
:1063B0008DED010ACDED020A8DED031A18F010F8EB
:1063C000E8E7314604F23C4001F054F90028E9D1F5
:1063D000DFE794F86032002BDBD0314620461AF01C
:1063E0003FFBDFE737B50D460DF107010446FFF728
:1063F00093FF28B19DF8073023B1032B0FD0002065
:1064000003B030BD04F5BE631B682B6004F2F45387
:1064100004F5BF641B686B602368AB60F0E720463F
:1064200029461AF0E9FA94F86002E9E710B5044643
:10643000FFF7ECFD18B1032807D0002010BD04F2CF
:106440003C40BDE8104001F03FB994F86032002BA9
:10645000F3D020461AF0F2F80028EED094F8143267
:1064600003F0FD03012BE9D194F80C03C31E58423D
:106470005841E3E710B50446FFF7C8FD80B1032893
:1064800010D194F8600250B15CF0FAF8D4F864329C
:10649000C01A44F62063984294BF0020012010BD2A
:1064A0000120FCE70020FAE708B50246FFF7AEFD41
:1064B000032804D110461AF00FFD012008BD00206A
:1064C000FCE7000030B585B004460191FFF722F8E3
:1064D0000199054610B9002005B030BD0191FEF7C5
:1064E000E9FF01990028F6D02846FEF7E7FF0028CB
:1064F000F1D0B4F864365907EED494F80933002B80
:10650000EAD00B4A1268D26A92F89C506DB103A986
:106510002046FFF7C9FF30B19DF80E309A07DBD552
:10652000C3F38000D8E72846D6E71846D4E700BF73
:106530004061002010B50446FFF768FD032804D130
:106540002046BDE810401AF0C3B9002010BD00007D
:106550002DE9F04190F80C338CB00027032B064650
:106560000C46154600970197029719D11AF0E8F8E2
:106570006A4680464FF0FF3130461AF03FF9B8F1D5
:10658000FF3FA760676027600DD115F071FB2B46B8
:1065900090F8EC14224614F09BFA0CB0BDE8F081A0
:1065A0004FF0FF38EBE715F063FB2B4622465FFA0E
:1065B00088F114F08DFA95ED000A684618F0BAF9E2
:1065C00003A920468DED051A8DED030ACDED040AD1
:1065D00018F0EAF906F52B7206F5487103A816F0D3
:1065E0000FFB214603A816F08DFA84ED021A84ED04
:1065F000000AC4ED010A95ED007ADFED037AA7EEFB
:10660000271A84ED021AC8E70AE81C411FB5DFED1E
:106610000B7A20EE270A0C461946094BCDE90042B9
:10662000BDEEC00A18688DED020A064B9DF81820D1
:10663000C06A12F057FA04B010BD00BFE02E6542E8
:1066400040610020407A0A082DE9F0472DED028BC9
:1066500092B0002504460F464FF07E5A00F548716F
:1066600006A89046CDF818A009950895079517F04B
:1066700001FB05F0E3F905F0DFF881462046FFF75E
:10668000C5FC032803D094F80C33032B4FD19FEDA6
:10669000558ADFED558A00262379F2B2934247D915
:1066A0000AAA71B22046CDF828A00D950C950B953D
:1066B0001AF0B6F90AA906A817F004FFB4EEC80A42
:1066C000F1EE10FA0DDD494ACDF800803B4648490D
:1066D0002046FFF79BFF002012B0BDEC028BBDE807
:1066E000F0870AA906A803950495059517F0D4FE2E
:1066F00003A90EA88DED0E0ACDED0F0A8DED101A2F
:10670000CDED111A17F03CFCB9F1000F0DD09DED45
:10671000050AB0EEC00AB4EEE80AF1EE10FA04DDA4
:10672000344ACDF800803B46D1E70136B4E7002378
:1067300094F8686216F0010001D0012BCCD104F26C
:10674000FC510AA8CDF828A00D950C950B9517F0D3
:1067500091FA0AA906A817F0B5FEDFED227AB4EE89
:10676000E70AF1EE10FA05DD204ACDF800803B463D
:106770002149ADE72046FFF749FC03282DD12046EB
:106780001AF0A0F994F86832DB0728D438BB0AA9BC
:1067900006A803950495059517F07EFE03A90EA89B
:1067A0008DED0E0ACDED0F0A8DED101ACDED111AFB
:1067B00017F0E6FBB9F1000F11D09DED050ADFEDF2
:1067C0000A7AB0EEC00AB4EEE70AF1EE10FA06DD7E
:1067D000084ACDF800803B46CAE70020D2E70120F6
:1067E0007AE700BFC2B8323EC2B8B23E6C7A0A083D
:1067F000777A0A0883310A087C7A0A082DE9F74378
:106800001446054688460193FFF710FE019A074695
:1068100038B92448244B00682146C06A12F062F956
:10682000019A019221462846FFF70EFF064630B333
:106830002846FFF7EBFB95F80C33019A83420DD005
:1068400005F0FCF804F0F8FF019A38B1174B154831
:1068500000682146C06A12F045F910E02846FFF7AB
:10686000D5FB18B103280FD0114BF0E71346414672
:10687000224605F23C4000F03BFF00B107B900267C
:10688000304603B0BDE8F08395F86092B9F1000F8F
:1068900001D1084BDBE7134641462246284619F052
:1068A000DDFEEAE740610020807A0A088C7A0A0857
:1068B000BC7A0A08AB7A0A0890F80C33032B01D192
:1068C0001AF020BB0020704737B5054600F5067169
:1068D00040F6033201A811F027FF2846FFF796FB88
:1068E000044640B103280AD0002401A811F03EFF5D
:1068F000204603B030BD284619F0AEFFF5E7284624
:1069000019F0AAFF0446F0E708B50246FFF77EFB40
:1069100010B1032806D008BDBDE8084002F23C4093
:1069200000F09CBEBDE8084010461AF0E1BA000035
:106930000B4610B411462BB1032B09D000205DF893
:10694000044B70475DF8044B00F23C4000F09CBEE5
:106950005DF8044B19F0F2BF13B50446FFF756FB80
:106960000A46014620460192FFF7E2FF70B9084B44
:10697000019A1B68DB6A93F89C0038B194F80C13F9
:10698000204602B0BDE81040FFF7D2BF02B010BDF4
:106990004061002037B504460D4640F2B25200F582
:1069A000067101A811F0C0FE2946204619F0E4FF47
:1069B00094F80C33032B054610D148B104F58361DC
:1069C0002046FFF7C9FF84F82804204600F0DCFDCC
:1069D00001A811F0CBFE284603B030BD0025F7E733
:1069E00070B590F87C32DB0786B004460D460CD4B7
:1069F00003F022F8437C242202FB0300D0ED0B7A43
:106A0000F1EE677AC5ED007A3BE002A803F0A4FF3F
:106A100001A92046FFF7ECFAE8B90DF073FD94F9EF
:106A20004432022B0646E3D1FEF7ECFE0228DFD902
:106A300096F8F4029FED147AB02303FB0066D4F8B5
:106A40007032D6F8E0209B1A07EE903AF8EEE77A1B
:106A500067EE877AD6E702A92046FFF77DFF002878
:106A6000DBD0D4F87022039BDFED076A9DED017A3D
:106A70009B1A07EE903AF8EEE77AA7EEE67A85EDF4
:106A8000007A06B070BD00BF0AD7233CF0B50C46B3
:106A900087B000F50671064640F6863201A811F06F
:106AA00043FEA36853B9E36843B9636833B9002769
:106AB00001A811F05BFE384607B0F0BD204604F097
:106AC00053F80028F3D094E80F0002AD85E80F00DA
:106AD0000021284604F00AF807460028E7D096F877
:106AE0007C32DB0704D437F0DFFB192137F074F96F
:106AF00095E80F0006F51B7C8CE80F0096F87C32B9
:106B000043F0010386F87C32304600F03DFD41F051
:106B100091FE462142F0ACFC41F08CFE452142F052
:106B2000A7FC054BA2681B68DB6A1A61E2685A6120
:106B300062689A61BCE700BF4061002038B5144B21
:106B40001B68DD6A2B6804465B6828469847F0B1ED
:106B50002B690BB96A69D2B1C4F874326B69C4F895
:106B60007832A969002204F51B7003F0FBFE94F84B
:106B70007C3223F0030343F0030384F87C3241F0BA
:106B800059FEBDE83840034A06213BF00FB838BD36
:106B900040610020D07A0A0813B504460193FFF73C
:106BA00035FA0328019B05D1204602B0BDE810400C
:106BB00019F060BF002002B010BD000010B588B011
:106BC00004460593FFF722FA0328059B4FF00000C7
:106BD0000AD10690079006A802900B9801900A9897
:106BE0000090204619F054FF08B010BD38B5044697
:106BF000FEF790FC0546D0B194F80C33032B03D07C
:106C000095F84E41204638BD204619F055FEFF2824
:106C10000446F5D001462846FEF750FC0028EFD088
:106C200021462846FEF746FC0028E9D0EAE704465C
:106C3000E8E7000008B590F80C33032B05D015F0F9
:106C400017F890F9EB04C0B208BD19F079FD431CA8
:106C5000F9D1F4E708B590F80C3383B1032B03D1D5
:106C6000BDE8084019F064BD35F00CFD40F6ED427A
:106C70004FF4801135F0BEFC4FF0FF3008BD1846D0
:106C8000FCE7000090F80C33032B01D11AF0B0BBE5
:106C90007047000090F80C33032B01D119F02CBC85
:106CA0007047000019F0B2BC10B504461CF02EFC71
:106CB0002046FEF737FC2046BDE81040FEF738BD01
:106CC00090F80C330BB1032B01D11AF00DBC00204E
:106CD0007047000030B500F5757304460D460FCBC4
:106CE00085E80F0094F8E40330BD00007FB5054649
:106CF00068460E4603F030FE95F87C32DB0703D47D
:106D00000024204604B070BD69462846FFF7E2FF24
:106D100004460028F4D0694605F51B7004F034F8E9
:106D200086ED000AC6ED010AEBE70000D0F88033DB
:106D30000B6090F87C037047D0F888330B6090F8B4
:106D40008503704710B500F5637203460C4607CA09
:106D500084E8070093F8980310BD000030B500F5F3
:106D6000677304460D460FCB85E80F0094F8AC031B
:106D700030BD000030B500F5836304460D460FCBEF
:106D800085E80F0094F8280430BD000010B500F22B
:106D90002C4203460C4607CA84E8070093F83804DF
:106DA00010BD00002DE9F0432DED028B8BB00546A0
:106DB0000E461746FFF71AFF014680462846FFF7A2
:106DC00081FB0446002848D0FEF7A4FB4146FEF7AD
:106DD00077FB86ED000A95F93032002B3ADD0DF095
:106DE00091FBFEF70FFD012834D90DF08BFB90F8D5
:106DF000F432D5EDDE7ADFED5D8A96ED000AB02241
:106E000002FB030095F93032D0ED3B0A07EE103A51
:106E1000F4EEE87AB8EEC77AF1EE10FAB7EE008A2F
:106E2000B8BFF0EE487A37EE201A20EE270A70EE4F
:106E3000C70A40F2B63015F039FCD5EDDE7AF4EE33
:106E4000E87AF1EE10FAB8BFF0EE487A80EE277AD1
:106E500086ED007A01233B7003E095F8083333B9DF
:106E6000387020460BB0BDEC028BBDE8F08395F87E
:106E70000C334FF00009CDF80490CDF80890CDF810
:106E80000C9043B1032B10D0CDF81090CDF8149096
:106E9000CDF818907CB902233B703246414605F28A
:106EA0003C4001F0C9FB0446DBE701A9284619F084
:106EB000F7FC0446E8E795F80C33002BEBD004A967
:106EC0002846FFF763FF04460028E4D001A904A880
:106ED00017F01AFD07A8CDED080A8DED091A8DED02
:106EE000070A18F025F904A8B0EE408A18F020F936
:106EF00095F93032002B30DD07EE903AF8EEE77A64
:106F00004FF47F7070EE670A37EE801AF5EEC00A14
:106F1000F1EE10FA48BFDFED160AF4EE410AF1EE89
:106F200010FAB0EE480AC8BFB0EE601A15F0BEFB0A
:106F3000B0EE408AD5EDDE7A9FED0C7AF4EEC77A9A
:106F4000F1EE10FAB7EE007AB8BFF0EE477A88EEAD
:106F5000277A032386ED007A7DE7B5EEC08AF1EE4D
:106F600010FA48BF9FED028AE4E700BF000000343A
:106F70000000000010B50446FFF75CFE84F80D0326
:106F80002046FFF757FE84F80E032046FFF752FE17
:106F900084F80F032046FFF75DFE04F55A7184F86C
:106FA00010032046FEF7F4FE84F8740300F00CFB97
:106FB00004F5617284EDDE0A04F560712046FFF786
:106FC000F1FE04F5627184F87C032046FEF7FCFEB6
:106FD00004F5637184F885032046FEF729FF04F564
:106FE000677184F898032046FEF734FF04F56C714E
:106FF00084F8AC032046FFF7F5F904F5707184F8C6
:10700000BC032046FFF7BCF904F5757184F8D00382
:107010002046FEF795FE04F57A7184F8E4032046D5
:10702000FFF78EF984F8F8032046FEF73DFF04F5DC
:10703000806384EDFF0A2046C3ED000AFEF754FF8B
:1070400004F2044383ED000A04F2144204F5816162
:107050002046FFF77DFA04F583612046FFF77CFCAC
:1070600004F22C4184F828042046FEF75DFF84F8E2
:10707000380410BD37B50D46044600F041F91DB97E
:1070800014F0F6FD13F0F8FB4FF4BE7204F5067130
:1070900001A811F049FB94F869322BB92046FFF79B
:1070A0004DFD012384F86932224B1D68A86A0368EC
:1070B0009B6998472046FEF787FD2046FEF700FEB5
:1070C000204600F093FA2046FFF754F8286B30B1C1
:1070D0000368D4EDD20ADB6894EDD10A9847D4F85E
:1070E000100208B15CF03AFA204600F07DF8204624
:1070F000FEF79AFF94F8903284F80C0383420ED086
:1071000084F8900298B10C4D0C4B032808BF1D4623
:1071100041F090FB0A4A2B4606213AF047FD2046F3
:10712000FFF728FF01A811F021FB03B030BD054D8A
:10713000EEE700BF406100200B4A0A08777A0A0890
:10714000E87A0A087C7A0A08D0EDDE7A9FED057AA3
:10715000F4EEC77AF1EE10FAB7EE000AA8BFB0EE6F
:10716000670A704700000034014B1868704700BF81
:10717000686100204FF0FF30704700000120704729
:1071800070470000002070470020704770470000E3
:1071900070470000002070470020704700207047B3
:1071A0000020704700207047002070470020704783
:1071B000012070470368D3F89430184700207047C7
:1071C0000020704700207047002070470020704763
:1071D0000020704700207047002070470020704753
:1071E00000207047704700007047000008B514F099
:1071F0003FFD90F8EC0408BD08B514F039FD90F897
:10720000EB0408BD30B52DED028B9FED1A1ADFEDB2
:107210001A0A91ED000A87B005462D200C468DED27
:10722000011ACDED000A15F041FA9DED011ADDEDD0
:10723000000AF0EE408A2E2094ED010A15F036FA8D
:107240009DED011ADDED000AB0EE408A2F2094ED8D
:10725000020A15F02BFA03A905F52570CDED038A76
:107260008DED048A8DED050A33F06AF907B0BDECA7
:10727000028B30BDC2B8323EC2B832BE70B52DED01
:10728000048B00F5257403460E4694E8070084B08D
:10729000D3EDA57A9FED181A93EDA69A01AD85E876
:1072A000070030EE270AF0EE608A3A20DFED130A7D
:1072B00015F0FCF93B20B0EE408A9FED0F1ADFED90
:1072C0000F0A38EE890A15F0F1F98DED018A8DED7E
:1072D000020A95E8070084E8070046B1002120462D
:1072E00004B0BDEC048BBDE8704031F0C5BB04B008
:1072F000BDEC048B70BD00BFC2B8323EC2B832BE16
:1073000010B504465BF0BCF9D4F8F4321BB1C21AD4
:10731000B2F57A7F12D30A4A1268D26A92F89C2098
:1073200002B15BB9C4F8F40294F8314214F0A0FC45
:1073300080F8E24404F082FB80F8254010BD00BFD5
:10734000406100202DE9F0432DED028B91ED007A94
:10735000D1ED037A87B08DED047AB0EEC77AB5EE41
:10736000C07AF1EE10FADDE91087DDF84C90CDED32
:10737000057A0C4615461E4606DCF0EEE77AF5EE79
:10738000C07AF1EE10FA02DD04A817F03FFA6B2084
:10739000B7EE001AFFEE000A9DED050A15F086F91A
:1073A0006C2089ED000AB7EE001AFFEE000A9DED91
:1073B000040A15F07BF904A888ED000A17F082F999
:1073C000B7EE008A002852D00023C9F8003088EDBB
:1073D000008AD4ED067A67EEA77AF4EEC87AF1EE69
:1073E00010FA4ADB0023336085ED008ADFED3F0AA7
:1073F00096ED000A7C20B7EE001A15F057F986EDDD
:10740000000A95ED000A7D20B7EE001AFFEE000A93
:1074100015F04CF985ED000AD4ED067A129BDFEDEC
:10742000346AF1EE677AC3ED007A96ED007AF0EEF9
:10743000C77AF4EEE67AF1EE10FA2BD503AB02AA86
:1074400001A9204615F08AFD9DED018AB0EE480A9B
:1074500084F0E4FF85ED000AB0EE480A85F034F9C7
:1074600087ED000A07B0BDEC028BBDE8F08304A8ED
:1074700017F014F90028A7D1ABE738EE670A15F02A
:1074800071F886ED000A94ED087AC7EE007AC5ED32
:10749000007AABE794ED076AC6EE077AC7ED007A8B
:1074A00096ED007AB0EEC77AB4EEE67AF1EE10FA15
:1074B000C4D495ED007ADFED0F6AB0EEC76AB4EE82
:1074C000666AF1EE10FAB9DCB4EE477AF1EE10FA22
:1074D000B4D6B0EEE77AB4EE667AF1EE10FAADDC2F
:1074E000F4EE677AF1EE10FABCD7A7E700000000CF
:1074F00000000034FFFF7F7F1FB500F51773039373
:1075000000F51673029300F51573019300F51473DB
:10751000009300F5127200F5137300F54871FFF740
:1075200011FF05B05DF804FB9FED156A90ED817ABF
:10753000DFED146AD0ED837A27EE067A67EE867A5D
:1075400027EE267A67EEA67ABDEEC77AFDEEE77AD9
:1075500080ED7E7A90ED827A27EE067A17EE903AE9
:1075600027EE267A002BB8BF03F50C43BDEEC77A91
:10757000B8BFA03380ED7F7AC0F80032704700BFFB
:10758000E02E65420000C8421FB50E4B1B68044642
:10759000B3B1684603F0E0F969462046FFF7EAFB1D
:1075A00020B16A4600212046FEF79AF894F87C3212
:1075B000DB0705D504F51B7201212046FEF790F884
:1075C00004B010BD1864002008B502F035FABDE81B
:1075D000084001F0C3BD000010B580F8F812044661
:1075E0005BF04EF8C4F8FC0210BD000010B590F836
:1075F000F832044653B15BF043F8D4F8FC32C01AB9
:10760000B0F57A7F84BF002384F8F83294F8003311
:1076100053B15BF035F8D4F80433C01AB0F57A7F73
:1076200084BF002384F8003310BD000000F5B6705D
:107630000B4607C883E80700012070470023C0F805
:107640009C30C0F89830C0F89430C0F8A830C0F82A
:10765000A430C0F8A030C0F8AC30704770470000CC
:10766000024B0B604FF07C531360704700004842A0
:107670007047000008B50B4600F12801184616F0C7
:10768000F9FA012008BD000010B500F5C0700C46E5
:107690000FC884E80F00204603F04EF930B1FFF721
:1076A00063FD00F51B700FC884E80F00204603F04F
:1076B00043F980F00100C0B210BD000010B50446CF
:1076C00003F04CFC204610BD10B5D0F878310446CC
:1076D0005BB15AF0D5FFD4F87831C01A41F2883343
:1076E000984294BF0020012010BD0120FCE700005B
:1076F00013B5009303680192D3F890309847DDE901
:107700000021044628B90448044B0068C06A11F0FF
:10771000E9F9204602B010BD40610020807A0A08D5
:1077200013B504460191FDF7F5FE2368019A1B6D20
:10773000014608B190F84E11204602B0BDE8104055
:107740001847000030B585B00023019302930393DE
:1077500003680D46DB6D01A99847044620B1039BE1
:107760002B60204605B030BD02F066F9417C01F087
:1077700031FE04460028F4D002F05EF901F090FDDD
:10778000B1EE400A85ED000AEBE7000090ED007ACB
:10779000DFED0F7AB0EEC77AB4EEE77AF1EE10FAC9
:1077A00014D590ED017AB0EEC77AB4EEE77AF1EE37
:1077B00010FA0BD590ED027AB0EEC77AB4EEE77A04
:1077C000F1EE10FA4CBF01200020704700207047F6
:1077D0000000003410B5FDF79DFE044658B190F846
:1077E0004E11FDF767FE30B194F84E112046BDE80A
:1077F0001040FDF763BE002010BD000038B50D46F7
:107800000CF080FE0446FDF7FDFF022881BF94F8CE
:10781000F402B02303FB004000F5827089BF07C863
:10782000002085E80700012038BD00002DE9F04365
:107830002DED028B8FB003680025DB6C039504955A
:1078400005950695029502A904469847064638B163
:10785000FFF7BAFEDDED027A27EE800A8DED020A0F
:107860000CF050FEFDF7CEFF0746002E50D0DDEDA8
:10787000027AD4ED6A6A94ED6B7A23680B9527EE51
:10788000877A67EEA67A8DED097ACDED0A7A0C95A6
:107890000D959B6C0BA9204609AD98470BA928466E
:1078A00016F06AFE012F8DED030ACDED040A40F2B9
:1078B000B3800CF027FE90F8F432DFED5B7AB02550
:1078C00005FB030090ED3C8A28EE278AB0EE480ABB
:1078D00084F0A4FDF0EE408AB0EE480A84F0F4FE95
:1078E000CDED0B8A8DED0C0A0CF00CFE90F8F43205
:1078F00005FB030090ED3B0A0BA816F05DFE09ADF9
:107900008DED050ACDED060A05A896BB03C885E0F6
:107910000128CED89DED020AB5EEC00AF1EE10FAAC
:107920007FDD07AED4F8AC21D4F8A83107923046F9
:10793000089316F06BFE23680B950C950D959B6CC8
:107940000BA920469847DDED077A9DED0B7A77EE7F
:10795000877A9DED0C7ACDED077ADDED087A77EE2A
:10796000877A09ABCDED087A96E8030083E8030037
:1079700049E0236993ED000AB7EE008A38EE408AA9
:1079800016F01AFE04F5C8798DED090A4846B0EEE6
:10799000480ACDED0A0A16F00FFE0BA92846CDEDD8
:1079A0000C0A8DED0B0A16F0E7FD04F5D07603AF57
:1079B000C4ED650A314684ED640A384616F0ECFDE4
:1079C00004F5CC788DED090A4046B0EE480ACDEDBD
:1079D0000A0A16F0F1FD0BA928468DED0B0ACDED34
:1079E0000C0A16F0C9FD97E8030084ED660AC4EDA1
:1079F000670A86E803004946404616F0BDFD8DED56
:107A0000090ACDED0A0A9DED090ADDED0A0A0FB05B
:107A1000BDEC028BBDE8F083DDE9030185E80300DE
:107A2000F1E709950A95EEE735FA8E3C10B590F826
:107A30004213044603F02CFC7C23C0B203FB004439
:107A4000D4F8A00010BD0000044B026F1B68DB6A75
:107A50005A60426F9A60826FDA607047406100201E
:107A6000F0B58FB0044614F003F90023029303939A
:107A7000049390F8EB1401AB02AA054612F0CAFF7A
:107A800004F19407D8B39DED010AB5EEC00AF1EEFA
:107A900010FA34DD02A816F05DFF04F1B00684EDA3
:107AA0002C0AC4ED2D0A84ED2E1A3946304616F004
:107AB00061FF04F17C01304616F010FF04F18801EB
:107AC00005A88DED050ACDED060A8DED071A16F015
:107AD00005FF08A88DED080A9DED010ACDED090A04
:107AE0008DED0A1A16F026FF0BA904F128008DED82
:107AF0000B0ACDED0C0A8DED0D1A15F0DBFA95F899
:107B0000EB040C2303FB0050394600F55C7016F0C3
:107B1000E5FE84ED2C0AC4ED2D0A84ED2E1A0FB07B
:107B2000F0BD00002DE9F047824B00251F682DEDC8
:107B3000028BC0F89C50C0F89850C0F89450C0F820
:107B40008450C0F88050C567C0F89050C0F88C5081
:107B5000C0F88850C0F8B850C0F8B450C0F8B05061
:107B60000446F86A03688AB05B680E46984704F1D9
:107B70002809002854D05AF083FD42F20F7398422E
:107B80004ED8FB6A9FED6C8A93ED010A84ED1C0AC6
:107B9000D3ED020AC4ED1D0A93ED031A484684EDA5
:107BA0001E1A15F07BF940F045FED4ED1E7A67EE03
:107BB000887A054617EE900AF8F7A6FCD4ED1D7AF0
:107BC00067EE887ACDE9040117EE900AF8F79CFC7D
:107BD000D4ED1C7A67EE887ACDE9020117EE900A9F
:107BE000F8F792FC554ACDE900010621284639F004
:107BF000DDFF94ED1E8AB0EE480A84F00FFC84EDA0
:107C00006B0AB0EE480A84F05FFD84ED6A0A5AF010
:107C100037FDC4F87C010AB0BDEC028BBDE8F087EB
:107C2000A6B194ED1C0AB4EE400AF1EE10FA0DD69E
:107C3000D4ED1D0AF4EE600AF1EE10FA06D694EDCA
:107C40001E1AB4EE411AF1EE10FA52D714F010F8E1
:107C500090F8EC344FF00C0A0AFB030303F50073B1
:107C6000074693E8070007AE86E807004FF01508BF
:107C7000B2EE028AF2EE068A304617F059FAB4EEF6
:107C8000C80AF1EE10FA38D508F1FF3818F0FF08ED
:107C90003CD1304617F04CFAF1EE047AB4EEE70A24
:107CA000F1EE10FA43DD9DED090ADDED087A9DED58
:107CB000078A20EE000AA7EEA70A84F01BFFF0EE69
:107CC000400AB0EE480A84F0CBFDDDED090A84EDF0
:107CD0001D0A9DED080AF1EE600AB1EE400A84F03B
:107CE000BFFD84ED1C0A9FED161AD4ED1D0A94ED1C
:107CF0001C0A484615F0D2F87BE7304617F018FA10
:107D0000B4EEE80AF1EE10FABEDCC2E7384612F033
:107D1000D1FC384612F0B0FD97F8EC340AFB03733F
:107D200003F5007393E8070086E80700A4E72567DA
:107D30006567D8E740610020E02E6542087C0A08AC
:107D4000000000000021FFF7EDBE000037B504463B
:107D500008461546019117F0EBF9B7EE007AC7EE29
:107D6000007AB4F8DC3001980133A4F8DC3094EDEB
:107D7000367A37EE277A84ED367AB0EE007AF4EE72
:107D8000C77AF1EE10FA06D5B6EE007AF4EEC77AAD
:107D9000F1EE10FA0DDC9FED0E7AF4EEC77AF1EEFB
:107DA00010FA13D59FED0B7AF4EEC77AF1EE10FAC4
:107DB0000CDDB0EE670A16F0BDFD012085ED000A6E
:107DC000C5ED010A85ED021A03B030BD0020FBE7C6
:107DD00000247449BD37863570B52DED028B00F156
:107DE000280600F134058AB029460446304616F0CC
:107DF0001DFEB6EE008A20EE088A2846B0EE480A3C
:107E000016F098FD07A93046CDED080A8DED091A48
:107E10008DED070A16F078FD30468DED010AB0EEC3
:107E2000480ACDED020A8DED031A16F083FD07A96D
:107E300028468DED070ACDED080A8DED091A16F0DA
:107E400063FD04A901A88DED040ACDED050A8DEDB1
:107E5000061A16F0FFFD324601A920468DED070AED
:107E6000CDED080A8DED091AFFF770FF58B95AF0E9
:107E700007FC0121C4F878012046FFF753FE0AB041
:107E8000BDEC028B70BD2A4604A92046FFF75EFFB9
:107E90000028ECD004F1400207A92046FFF756FF66
:107EA0000028E4D0EBE7000030B52DED028B0D4645
:107EB00083B091F842130446284603F0E9F9C1B2B1
:107EC0007C2000FB0151903104F1280014F076FE73
:107ED00068468DED000ACDED010A16F019FCDFEDC4
:107EE0001C7AB4EEE70AF1EE10FA05D59FED190AF7
:107EF00003B0BDEC028B30BD684616F087FC6846C7
:107F000016F0E0FB0028F1D1284694ED488A03F0F2
:107F100023FBF0EE400AB0EE480A14F0EFFA80B905
:107F2000284603F019FB84ED480AB0EE408A84F03D
:107F300075FA84ED490AB0EE480A84F0C5FB84ED79
:107F40004A0A04F59271684616F08AFBD0E700BF32
:107F500000000034000000009FED0C7AB4EEC70A68
:107F6000F1EE10FA0BD4DFED0A7AB4EEE70AF1EE87
:107F700010FA07DCC0EE077AB0EE670A7047F7EE3A
:107F8000007AF9E7F2EE047AF6E700BFF3665F3FA6
:107F900058A00B4108B51C3016F0BAFBF1EE007A80
:107FA000B4EEE70AF1EE10FA9DBFF1EE027A37EE79
:107FB000C00ADFED047A9FED040A98BF20EE270A7D
:107FC00008BD00BFCDCC4C3ECDCCCC3D08B58369BF
:107FD00093F9000038B10CF095FAFDF713FC012875
:107FE00094BF0020012008BDF8B52DED028B054699
:107FF00003F024FD03F020FC0446B8B3FFF7B4F807
:1080000090F8093393B32846FFF7E0FF064668B3BC
:108010000CF078FA90F8F432B02707FB030090EDEB
:108020003B7AF0EE087AB4EEE77AF1EE10FA1DD45E
:1080300095ED1E8A0CF066FA90F8F432DFED1E7AA8
:1080400007FB030090ED3C0A98EE270A14F0DAFAD9
:10805000DFED1A7AB0EEC00AB4EEE70AF1EE10FADC
:1080600008DC5AF00DFB3446C5F86801BDEC028B04
:108070002046F8BD05F5B67017F05AF8B0EE408A04
:108080000CF040FA90F8F4329FED0D7A07FB0303F1
:10809000D3ED3B7A67EE877AB4EEE78AF1EE10FA19
:1080A000DFD55AF0EDFAD5F86841001BB0F5FA6F4C
:1080B0008CBF00240124D9E7E02E65420000344241
:1080C000CDCC4C3F10B50A4B1B68DB6A93F89C3053
:1080D00004465BB95AF0D4FAD4F87C31C01A44F69D
:1080E0001F6398428CBF0020012010BD0020FCE7D8
:1080F00040610020F8B52DED068B04460CF002FA25
:10810000054603F09BFC064606F0D2F9002840F035
:10811000AB802046FFF768FF002800F0A8803046BB
:10812000FFF784FCD4F8E830984200F01A8130461A
:10813000FFF77CFCD4F8E830DFED8F7AC31A08EE45
:10814000903AF8EE688A304668EEA78AFFF76EFC30
:1081500094F8BC30C4F8E800F3B9304603F07EFB75
:10816000D0B104F1280796F842233946304603F08F
:10817000F7F9D4ED1D0AB0EE401A384694ED1C0A0A
:1081800014F08CFE0023C4F89030C4F88C30C4F88E
:108190008830012384F8BC3020463146FFF784FE46
:1081A00095F8F40205EB0015B0EE408AD5F8A03042
:1081B000C4F8EC3004F1B000D4ED129A16F0B8FF18
:1081C0006368DFED6E7A93ED007AB4EEE77AF1EE54
:1081D00010FA68EE299AB0EE40AA01D5C3ED007AF4
:1081E0002046B0EE4A0AFFF7B7FE636820EE299AF0
:1081F00093ED000A29EE009AFFF7CCFE29EE009AD3
:10820000204684ED249AFFF75DFF38B1D4ED247A3F
:10821000B2EE007A67EE877AC4ED247AF0EE007A47
:10822000F4EEE78AF1EE10FA10D5DFED557AB4EEF0
:10823000E7AAF1EE10FA09D5DFED527A69EEA79AB6
:10824000D4ED2A7AE9EEA87AC4ED2A7A9FED4E0A97
:1082500094ED397ADFED4D7AB0EEC88A28EE008AC7
:10826000A7EE278A84ED398ABDEC068BF8BDFEF7B0
:108270007BFF90F80933002B73D02046FFF7A6FE52
:1082800000286ED095F8F42205EB0213D3F8A01065
:10829000D4F8EC308B4264D0B02606FB025292ED4B
:1082A0003B7AF0EE087AB4EEE77AF1EE10FA58DB9A
:1082B000CB1AC4F8EC1008EE903A95F8F4329FED22
:1082C000341A94ED1E0ADFED337A06FB0353D3ED27
:1082D0003C9A69EE819AF8EE688A39EEC00A68EE37
:1082E000A78A14F0CFF9B0EE409A84F0EDF994F833
:1082F000BC30B0EE408AF3B1F3EE047AF4EEE78AD4
:10830000F1EE10FA17DC95F8F40206FB005595ED36
:108310003B7AF2EE027AB4EEE77AF1EE10FAFFF66B
:1083200049AFDFED1D7AB0EEC99AB4EEE79AF1EEEF
:1083300010FAFFF63FAF9FED198AD4ED1D0A94EDB8
:108340001C0AB0EE691A04F1280014F0A7FD0123FD
:1083500084ED248A84ED238A84ED228A84F8BC305B
:1083600028E7BDEC068B04F188009FED0D0ABDE8FF
:10837000F84016F033BB00BFBD378635CDCC4C3D41
:10838000C2B8B23E0AD7233CCDCC4C3ECDCC4C3FFC
:1083900035FA8E3C6F12833A1904863F00000000C4
:1083A000EC51783F30B50C2303FB010101F1C00310
:1083B000144693E807008BB004AD85E8070094E805
:1083C000070083E807002846FFF7E0F907AB58B13C
:1083D00094E8070083E807009DED070ADDED080A31
:1083E0009DED091A0BB030BD95E80700F2E70000DB
:1083F000F0B52DED028BD0F830318B60D0F83431F0
:10840000CB6085B004460D4601F016FB06460CF025
:1084100079F8A36993F90030022B07464BD1FDF799
:10842000F1F9022847D997F8F432B02202FB03731E
:10843000D3F8E0100022284602F094FAD4ED500A56
:1084400094ED4F0A284602F075FD94F8443163B369
:108450005AF016F99FED228A97F8F4128DED018AF1
:1084600001AA064638460BF0D1F8D4F838019FED42
:108470001D0A361A07EE906AF8EE677A4FF48760A5
:1084800027EE800AB6EE001AF0EE480A14F00EF954
:10849000DDED017A30EE270A04F584708DED010AD6
:1084A00016F08AF8284602F045FD94F8440105B01C
:1084B000BDEC028BF0BD707C242303FB006696EDBF
:1084C0000B8AFEF751FED0ED9C7A9FED077AF8EE0D
:1084D000E77AE8EE077AFDEEE77A17EE901AA9E759
:1084E000000000006F12833A0000C842F8B5036F25
:1084F0000B60436F4B60836F8B6000F14C050E4641
:10850000074601F10C040FCD0FC40FCD0FC42B682B
:10851000236007F1B00207CA06F1300383E80700C1
:1085200007F1940207CA06F13C0383E8070007F14C
:108530001C0207CA06F1480383E8070006F1600140
:108540003846FFF755FF86F87000F8BD30B589B0A2
:10855000044668460D4602F0FFF969462046FFF7DB
:1085600093F818B90024204609B030BD04A802F0E1
:10857000F3F9204604A9FFF73BFF04460028F1D099
:1085800004A9684602F02EFC85ED000AC5ED010A3B
:1085900085ED021AE7E700001FB500230C4601A98C
:1085A000019302930393FFF7D1FF08B1039B23606C
:1085B00004B010BD30B585B001AD00230C4629468E
:1085C000019302930393FFF7C1FF034618B195E8A7
:1085D000030084E80300184605B030BDF8B5064630
:1085E0000F461546FCF796FF044690B13946FCF756
:1085F00061FF70B120463946FCF760FF044640B188
:10860000FCF788FF3946FCF75BFF85ED000A204642
:10861000F8BDFEF7A9FD90F8083343B13046FFF7E7
:10862000D5FC044618B1D6F864312B60EFE7D6F8D4
:1086300064312B600024EAE770B52DED048B1646FB
:10864000FFF7CCFF054670B3FEF78EFD90F9304280
:108650004CB30BF057FFFDF7D5F8012823D9E4B24E
:1086600007EE904AB8EE678A0BF04CFF90F8F432B0
:1086700096ED009AB02202FB0300D0ED3B8AFEF794
:10868000A3FF38EE281A78EEC80A40F2614029EEBE
:10869000000A14F00BF8B0EE408AFEF795FFC8EE22
:1086A000007AC6ED007ABDEC048B284670BD000050
:1086B00008B503F0C3F9BDE8084003F0BDB80000F9
:1086C00010B5044616F0E2F950B904F10C0016F0AA
:1086D000DDF928B904F11800BDE8104016F0D6B94C
:1086E000012010BD38B500F1280504462846FFF7E3
:1086F000E7FF28B120460121BDE83840FFF712BA54
:10870000D4ED107AB7EE007AF4EEC77AF1EE10FAF3
:1087100006D5BFEE007AF4EEC77AF1EE10FA12DC5D
:108720002046FFF759FB2846FFF7CAFF0028E1D192
:10873000D4ED107AB2EE047AF0EEE77AF4EEC77A6E
:10874000F1EE10FAD6DC38BD10B5044616F0F0FC98
:108750002046BDE8104016F055B900002DE9F04F55
:108760002DED028BA3B000270446B0EE408A0A9795
:108770000B970C97FFF7BEFC13F07AFA04F1F00B9D
:1087800005465E464FF0000804F1280A95F8F131DD
:10879000022B5FFA88F1A8BF02238B423AD9284600
:1087A000019111F0A5FE019980B310AB13AA2846E0
:1087B00013971497159712F08BF99DED100AB5EEEB
:1087C000C00AF1EE10FA21DD13A816F0C3F81CA9B7
:1087D00050468DED1C0ACDED1D0A8DED1E1A14F0CC
:1087E00091F916A88DED160AB0EE480ACDED170ADC
:1087F0008DED181A16F09EF81CA930468DED1C0A56
:10880000CDED1D0A8DED1E1A16F0B4F808F1010821
:108810000C36BBE795F8EC140C2303FB015101F572
:108820000071504614F06EF984ED070A94ED450A84
:10883000C4ED080A30EE088A84ED091A84ED458AF1
:108840000BF060FE0646FEF78FFC90F809330393A9
:108850002046FFF7BBFB80B13046FCF7D3FF022870
:108860000BD996F8F4226169B02303FB026391F9F6
:10887000001093F80201884261DA94ED457ADFED49
:10888000847AB4EEE77AF1EE10FA62D494ED598A64
:10889000FEF7A0FF38B1FCF73DFE90F84E11FCF753
:1088A0000FFEB0EE408A236C626BA16A1E93B0EE9D
:1088B000480A1CA81D921C9116F03CF804F5B671EC
:1088C0000AA88DED0A0ACDED0B0A8DED0C1A16F0F3
:1088D00051F859F0D5FE0023019084F82C31204640
:1088E000FFF774FB00286BD096F8F422B02101FB4F
:1088F0000262D2F8E430C4F8303196F8F43201FB69
:108900000363D3F8E830C4F8343159F0B9FE0123D9
:10891000C4F83801C4F83C71C4F8407184F844319B
:10892000D4F81831002B5ED1019BC4F818310AAB82
:1089300093E8070004F5847484E8070009E006EB77
:108940000212D2F8A02001920199D4F818218A428B
:1089500004D123B0BDEC028BBDE8F08F03F5827328
:1089600093E8070094F82C310DF1280C8CE80700EF
:108970001BB904F5847383E807000123604684F87B
:108980002C3104F5B67115F0BFFF1CA904F14C00A1
:108990008DED1C0ACDED1D0A8DED1E1A14F0E0F8C8
:1089A000B5EEC00AF1EE10FA8DED1C0AD8BF9FEDAE
:1089B000370ACDED1D0A8DED1E1A84ED590A8EE79A
:1089C00094ED457AD4ED4F7ADDED0A6AE6EE877ACA
:1089D000DDED0B6AC4ED4F7AD4ED507AE7EE267ADE
:1089E000C4ED507A9CE7D4ED457A254B0D97F5EE12
:1089F000C07AF1EE10FA0E970F93AAD9214B9FED92
:108A0000227A1B68DB6A67EE877A93F89C300293C0
:108A1000B7EE007AC7EE278A002B4BD094F82C31A2
:108A200013B9039B002B43D0E36804F5847193EDE5
:108A3000008A0AA815F068FF28EE888A8DED1C0AC6
:108A40001CA8B0EE480ACDED1D0A8DED1E1A15F0DA
:108A500071FF16A90DA88DED160ACDED170A8DED43
:108A6000181A15F087FF0DA8FFF76EFE0DA816F077
:108A700027F8F8B159F004FEC4F8780169E700BF9F
:108A8000000080BF406100200AE81C410000000097
:108A9000CDCC4C3ECDCC4C3FCDCC4C3D920A06BF0C
:108AA000920A063FC2B8B23E728A0E3C5B82183907
:108AB000039B02931822002116A886F0B7F818220B
:108AC00000211CA886F0B2F81FED108A05F20E53A3
:108AD0000DF170084FF000094FF0FF37059395F83E
:108AE000F131022B1A465FFA89F1A8BF02228A42AD
:108AF0007AD98B4204916BD9059B13F80930002B6E
:108B000066D0B0EE680A584615F068FF029B0499DB
:108B1000002B64D00C2222AB02FB0933A3F1180214
:108B2000049220465A460693FFF73CFC069B03ED51
:108B3000060A049BC3ED010A83ED021A4046FEF7C4
:108B400025FE002844D14046FFF7FEFD404615F0C3
:108B5000B7FF00283CD10C2303FB09F222AB1344DE
:108B600007920DA9A3F1300240460492069315F036
:108B700071FF069B03ED0C0A049B0DA9C3ED010ACE
:108B800083ED021A404615F051FF22AB079A03EB22
:108B9000890303ED1A0A16AB981816F0C9FA7A1C65
:108BA00004D0B4EEC08AF1EE10FA03DD4FFA89F773
:108BB000B0EE408A22AB03EB870353ED1A7AF5EE51
:108BC000407AF1EE10FAF7EE007A48BFB0EE678A0D
:108BD00009F1010908F10C080BF10C0B7FE79BE888
:108BE000070088E80700A9E77B1C3FF443AF84F83F
:108BF0001C712046FFF7F8F960B12046FFF7E6F94F
:108C0000002840F0348122AA0C2303FB0723002212
:108C100043F8282C16AA07EB470895F8EB3402EB2B
:108C2000880895F8F0219A4240F23C812B4493F851
:108C30000C35002B00F0368195F8EC3495F8F121D5
:108C40009A4240F22F812B4493F80E35002B00F00E
:108C500029810C2322AA4146504603FB072713F023
:108C60007FFF07ED0C0A47ED0B0A07ED0A1A404695
:108C700015F00CFF002840F02181404615F020FF40
:108C8000002840F01B815FED7E7A94ED387A28EE63
:108C9000278A5FED807AA7EE278A04F1B00084ED81
:108CA000388A16F045FAA3685FED857A93ED007A6D
:108CB000B4EEE77AF1EE10FAB0EE408A00F10281EC
:108CC0002046B0EE480AFFF747F9404615F032FE5D
:108CD000A3688DED130ACDED140A8DED151A93EDF1
:108CE000000A13A815F026FE204684ED1F0AC4EDE5
:108CF000200A84ED211AFFF7E5F928B1B2EE000A47
:108D000004F17C0015F06AFE039BB3B33046FCF718
:108D100079FD012831D996F8F402B02303FB0066EF
:108D200096ED3B7AF0EE087AB4EEE77AF1EE10FABF
:108D300023D595F8EC040C2303FB005595ED807AC0
:108D4000F1EE0C7AB4EEE77AF1EE10FA15DBD4ED21
:108D50001D7A1FEDAE7AF4EEC77AF1EE10FA0CDD53
:108D60001FEDB17AF4EEC77AF1EE10FA05D5B6EE42
:108D7000000A04F17C0015F031FE5FEDB67AB4EE26
:108D8000E78AF1EE10FA22D51FEDB90A404615F038
:108D9000D1FD10A88DED100A94ED450ACDED110A14
:108DA0008DED121A15F0C6FD13A904F1A0008DED8A
:108DB000130ACDED140A8DED151A15F0DBFDD4ED77
:108DC0002B7A94ED457A77EE877AC4ED2B7A94ED81
:108DD0002B7AF1EE047AB4EEE77AF1EE10FA4FF066
:108DE00000053BDB12F044FF5FEDD07A94ED2B1AC7
:108DF00094ED280A21EE271A40F2C530F1EE410A1F
:108E00008DED031ACDED020A13F050FC9DED031A0F
:108E1000DDED020A84ED280A40F2C63094ED290AFD
:108E200013F044FC9DED031ADDED020A84ED290ADE
:108E300040F2C73094ED2A0A13F038FC04F1A00187
:108E400084ED2A0A04F1940015F094FDC4F8A850AA
:108E5000C4F8A450C4F8A050C4F8AC5018220021A3
:108E600004F1F00085F0E2FEC4F814515CE5E3681B
:108E7000F7EE000A93ED000A13F040FB00283FF4E0
:108E8000C2AE94ED1C0AB0EEC00A83F01DFC0C23A8
:108E900022AA03FB072353ED0A7A27EE800A03ED8B
:108EA0000A0AB7E60C2322AA03FB0727002347F888
:108EB000283C47F82C3C47F8303CD8E62046FFF7E2
:108EC00011FCD7E5C3ED007AFAE600BF2DE9F04DBD
:108ED0002DED048B9EB0044612F0CAFE00F59F6390
:108EE000D3ED007A90ED7F8AF4EE487AF1EE10FA35
:108EF00048BFB0EE678ADFED5C7AB4EEE78AF1EE48
:108F000010FA0DDD1822002104F1F00085F08EFE2C
:108F10000023C4F814311EB0BDEC048BBDE8F08D05
:108F20002046FEF79DFD2046FEF756FFB0EE480AAC
:108F30002046FFF713FC2046FFF7D4FBFEF714F999
:108F400014AD00F5347204F1280114A813F058FE92
:108F50000FCD04F14C060FC60FCD0FC62B68336042
:108F600004F1740204F1780304F1700104F14C007F
:108F700013F0F4FF94ED1E8AB0EE480A83F04EFA27
:108F800084ED6B0AB0EE480A83F09EFB204684ED28
:108F90006A0AFEF759FDFEF7E7F804F5C071FDF720
:108FA000E9FE59F06DFBD4F8B031C31A632BB2D986
:108FB000C4F8B00135F078F99FED2C9A054659F0C8
:108FC00067FBD4ED1C7A67EE897A074617EE900AA4
:108FD0000E46F7F799FAD4ED1D7A67EE897A824644
:108FE00017EE900A8B46F7F78FFA94ED1E0A20EEE3
:108FF000090A41EC180B13F0EFFAD4F8740110EEE3
:10900000108AF7F781FACDE91201D4F87001F7F769
:109010007BFACDE91001D4F86C01F7F775FACDE9C8
:109020000E01D4F8E400F7F76FFACDE90C01D4F89B
:10903000E000F7F769FACDE90A014046F7F764FA6C
:109040000B4B01930B4B0093CDE908018DED068B83
:10905000CDE904ABCDE90276074B084A084928461A
:1090600034F064FD57E700BFCDCC4C3EE02E6542A6
:10907000675C0A086D7C0A08347C0A083E7C0A0892
:109080007C7A0A0808B52DED048BB0EE609AF0EEFC
:10909000408A00F011F9B0EE408A89EE280A83F088
:1090A00049FCDFED0B7A20EE270A83F0DBFBDFEDD6
:1090B000097A38EE278ADFED087A28EE278AF7EE5C
:1090C000007A37EEC00A28EE000ABDEC048B08BD1A
:1090D00041D3423E33938843A1D81943FFF7D2BF0F
:1090E00008B52DED048B9FED189AF0EEE07AF4EEC2
:1090F000C97AF1EE10FAF0EE408AB0EE608A1ED422
:1091000000F0DAF8DFED117A9FED117A70EE277A30
:109110009FED100AE8EEC77A9FED0F7A27EE800ADE
:10912000C8EE007A87EE270AB4EEC90AF1EE10FA0B
:1091300005DBBDEC048BBDE8084083F0DBBCBDEC77
:10914000048BB7EE000A08BD000000343393884357
:10915000F4FDD43B48A18F43CDCC9C3F427CD0ED65
:10916000257A242101FB020292ED0B0AD2ED090AB5
:1091700030EE270AFFF7B4BF38B52DED088BDFEDD1
:1091800021AA9FED21AA9FED21BA0546B0EE409A93
:10919000F0EE609AB0EE408A1524013CA4B25CB3B4
:1091A000F0EE490A2846B0EE480AFFF76BFFF0EEF2
:1091B000490A70EE698A284638EE2A0AFFF762FFEC
:1091C000B0EEE87A70EE697AB4EECA7AF1EE10FA8F
:1091D00077EEE87A10D468EEAA8A40F2631088EE3F
:1091E000A70AB0EE4B1A38EE400AF0EE4A0A13F026
:1091F0005DFAB0EE408AD0E7B0EE480ABDEC088BCD
:1092000038BD00BFCDCCCC3D0AD7233C00247449E7
:10921000002343608360C360036143618361C36172
:10922000002380F82030704790F82020531CDBB2D8
:10923000062B80F8203000EB820288BF002382EDED
:10924000010A88BF80F82030704700004FF0FF33DC
:1092500010B543610E4BC0F8A8300023044680F8D7
:10926000C830A830FFF7D4FF0A4BC4F8A83004F583
:10927000867058F0D5F8084B08491C60204630F03D
:1092800075FAD4F89030C4F89430204610BD00BF71
:10929000907E0A08A07E0A086C610020387F0A08C8
:1092A00008B5A83037F0CEF8DFED027A20EE270AB5
:1092B00008BD00BF00007A4490ED3C0ADFED057A5E
:1092C000B0EEC07AB4EEE77AF1EE10FA48BF90ED56
:1092D0003D0A70470000003473B5D0F8A43004464E
:1092E0000E4663B159F0CCF9D4F8A430C01A42F25A
:1092F0000F73984203D894ED280A02B070BD114B49
:109300001D687DB195F84E112846FCF7D7F848B195
:1093100095F84E1101AA2846FCF7C6F810B19DED4C
:10932000010AEAE7242101FB064494ED0A0ADFED75
:10933000067AB4EEE70AF1EE10FA58BFB0EE670A0B
:10934000DBE700BF6461002000000C4208B561B19A
:109350000378022B02D9064859F060F95A1C0270B2
:1093600000EB83004160012008BD0846FCE700BF18
:10937000507D0A082DE9F84305460E469146002423
:1093800000F13C082B78A34211DD00234A46314608
:1093900001200FF03DF8242363430746002158F8CD
:1093A00003000FF045F8874204D00134EAE70020BB
:1093B000BDE8F8830120FBE7054B1B682BB1416931
:1093C0004A1C02D0184634F095BD0020704700BFFB
:1093D0001864002002290BD8242303FB010191F813
:1093E000390030B191F83A0018B191F83B0070475C
:1093F000002070472DE9F047044659F041F9D4F8B0
:10940000F86042F21073861B9E4288BFC4F8F800D1
:1094100000274FF0240942F2107A237CFDB2AB42C0
:109420001CD929462046FFF7D5FF70B109FB054836
:1094300098ED0D0AD8ED097AD4ED250A30EE270A09
:109440002046FFF799FE88ED0C0A564504D909FB22
:109450000540303030F062FB0137DEE7617C2046AA
:10946000FFF73AFF84ED3D0ABDE8F08770B504468A
:1094700086B059F005F9D4F89830C31AB3F57A7F5D
:1094800005464FD3344B94ED257A1B68DFED336AE4
:10949000DB6AD4ED247A93F89C60B0EEC76AB4EE30
:1094A000E66AF1EE10FA32D5B0EEE76AB4EEE66A9B
:1094B000F1EE10FA2BD502A801F04EFA96BBFDF79B
:1094C00053FE02A9FDF756FC60B3DDED037A9FED74
:1094D000247AF8EEE77A67EE877AC4ED257AC4F845
:1094E0009850FDF741FEFDF7EFF92046FFF782FFA8
:1094F0003FF0A0F90546D4F89400F7F705F8194AAB
:10950000CDE900010621284638F050FB0AE037EE8D
:10951000676AF7EE005AB0EEC66AB4EEE56AF1EE9D
:1095200010FA01DC06B070BDB0EEE76AB4EEE66A90
:10953000F1EE10FAF6D4002ECFD02046903080ED18
:10954000007A30F0EBFA3FF075F9074A012106B0D6
:10955000BDE8704038F02ABB4061002000000034B4
:109560000AD7233C917D0A086C7D0A08F0B52DEDE1
:10957000048B85B004464FF4537200F5867103A83E
:109580000FF0D2F8D4ED227AD4ED236A9FED796AF8
:10959000637C37EEE67A2422B0EEC77AB4EEC67A60
:1095A000F1EE10FAC1BF9FED747A67EE877A9FEDF6
:1095B000737AE6EE877A02FB03430025C4ED237A33
:1095C00093F839602378E9B28B4206D904EB810322
:1095D000013558685BF0E0F9F4E7DFED698A9FED4B
:1095E000698A9FED699A0027237CFDB2AB4264D95A
:1095F000242303FB054393F83920002A5BD0D3EDE5
:109600000C7AF4EEE87AF1EE10FA0BDBF4EE677AFE
:10961000F1EE10FA06D6F0EEE77AF4EE487AF1EEC3
:1096200010FA04DD242303FB05435A6A1A6324233A
:1096300003FB0543D3ED090AD3ED0D7A93F83820E7
:1096400070EEA70AA2B993ED0C0A2046FFF746FD7B
:10965000D4ED257A30EE670AB4EE400AF1EE10FA46
:1096600016D7242303FB0545002385F83A3022E072
:10967000012A09BFD3ED0C7A93ED0B0A77EEE00ACD
:10968000D4ED3B7A04BF80EE897A87EE270AE3E7C0
:10969000F0EEC07AF4EE487A2423F1EE10FA03FBE0
:1096A0000545E1DC012385F83A30D4ED237A37EE25
:1096B000800A85ED0B0A013796E7627C2046114649
:1096C000FFF788FE48B1242101FB024292ED0B0A0C
:1096D000D16904F1A80036F095FE94F99C10277C1E
:1096E000002907DBB94205DACAB211462046FFF766
:1096F00071FE68B900226274D5B2AF4209D9294619
:109700002046FFF767FE01320028F5D0657400E0BF
:1097100062742046FFF7AAFE2046FFF74DFE10B107
:1097200020465CF041F9637C242505FB034393F854
:109730003930B34216D034F0B7FD4FF6FF7134F034
:10974000D9FB78B1607C05FB004494F83930002BDC
:1097500014BF00220422019234F0A6FD019A1221C6
:1097600034F05AFB03A80FF001F805B0BDEC048BF0
:10977000F0BD00BF0AD7233C0AD7A33C48E17A3F9B
:1097800000000034FFFF7F7F002019462DE9F04FD5
:109790000446007C0F4687B004F13A030022012101
:1097A000D5B2A84203F1240305D903F8231C03F81A
:1097B000241C0132F4E76F4B1E68F06A03685B6893
:1097C000984740B13FF036F86B4A062107B0BDE834
:1097D000F04F38F0EBB93FF02DF8684A062138F029
:1097E000E5F9002303A904F18800039330F05AFD42
:1097F0000A2558F045FF80462046FFF7B7FE58F08F
:109800003FFFA0EB0800B0F5FA7F02D95C4801F0F9
:1098100081F8B06A03680A215B689847617C20463A
:10982000FFF7D8FD0028E7D0B06A036864215B68C1
:10983000013D984715F0FF05DBD1524B05951B887C
:109840008DF80650CDE90355ADF80430052558F0E4
:1098500017FF80462046FFF789FE58F011FFA0EB66
:109860000800B0F5FA7FD1D8617C2046FFF7B2FD41
:109870000028EFD094F810B00DF10C08A14601AA11
:109880004FF0000A5FFA8AF18B4516D92046FFF7A0
:10989000A1FD50B1D8ED007A99ED097A137877EEF1
:1098A000877A0133C8ED007A13700AF1010A08F1D2
:1098B000040809F124090132E4E7B06A036864216D
:1098C0005B68013D984715F0FF05C0D1A9464FF0F0
:1098D0002408237C5FFA89F6B34226D906AB3344C9
:1098E00013F8143C33B908FB064686F83B3009F1FF
:1098F0000109EEE7002FFAD007EE903A06AA02EB34
:109900008602F8EEE77A12ED030AD4ED250A204626
:1099100080EE270AFFF730FC08FB064002A9303032
:109920008DED020A30F0BEFCE1E7617CDFF85C906F
:109930002046FFF7D1FC002684ED3D0A4FF02408B5
:10994000237CF7B2BB420FD908FB074393F83B30A7
:1099500043B13EF06FFF7B1C4A46062138F026F9E2
:109960000135EDB20136EBE70DB907484FE707B017
:10997000BDE8F08F40610020AC7D0A08D77D0A0861
:10998000ED7D0A08682E0A08297E0A08077E0A0863
:1099900008B5037C022B02D9034858F03FFE5A1C3D
:1099A0000274184608BD00BF487E0A0838B5057C19
:1099B00002460024E1B28D4206D91046FFF70AFDA7
:1099C00001340028F6D138BD281E18BF0120FAE75F
:1099D00070B50D4609780729044606D8027E437EF5
:1099E00022B901228A401343437670BD002BFCD07C
:1099F00000262278F3B29A42F7D904EB8303294672
:109A000058680368DB6898470136F2E737B50D46BA
:109A10000192FFF7CBFF0199044630B90448054B8A
:109A200000682A46C06A0FF05DF8204603B030BDDA
:109A300040610020F3900B08014B1868704700BF8D
:109A40006C61002010B50446006810B103685B68C3
:109A50009847204610BD000013B500220B680A602D
:109A600001A901935BF0E8FA044601A8FFF7EAFFB9
:109A7000204602B010BD000013B500220B680A603A
:109A8000022201A901935CF0C3FC044601A8FFF780
:109A9000D9FF204602B010BD13B500220B680A6042
:109AA000012201A901935CF0B3FC044601A8FFF771
:109AB000C9FF204602B010BD13B500220B680A6032
:109AC00001A901935CF0A4FC044601A8FFF7BAFFCA
:109AD000204602B010BD000010B50446006810B169
:109AE00003685B689847204610BD00002DE9F04FE1
:109AF0008FB0D0F800310893344B354D1B68059377
:109B00000446586803689B68984794F99D3006900E
:109B1000002BA2BF012606FA03F3069305F1D80A2B
:109B20002B68089A1A420BD000274FF0010BB94658
:109B3000069A0BFA07F3134206D10137202FF7D10B
:109B40000C355545ECD12DE0F9B26B682A7A0991B4
:109B500020460793FFF70EFC0999804628B3CDE90C
:109B60000A990B9B0D930DA9079BCDE90B992046F4
:109B7000984701462046FFF7E9FB0DA8FFF762FF73
:109B80000CA8FFF75FFF0BA8FFF7A6FFB8F1000FC7
:109B900002D00AA8FFF7A0FF2378032B02D0237C72
:109BA000032BCAD10FB0BDE8F08F059B5868042283
:109BB0000368CDE90182074A00921B680A461E46E7
:109BC00001462B7A0BA8B047CBE700BF40610020CD
:109BD00028800A08801A060070B5D0ED247A9FED1F
:109BE000597AF0EEE77AF4EEC77A0123F1EE10FA33
:109BF0008AB00446037609D49030002309A9059061
:109C0000099330F04FFB05982FF088FF4E4B4F4AD9
:109C10001E680025E5632566C4F88450B1680B68AA
:109C200007A81B689847079B099309A92046CDE917
:109C300007555AF043FA01462046FFF787FB09A86B
:109C4000FFF700FF08A8FFF7FDFE079810B10368B3
:109C50005B6898472378032B49D0237C032B46D09D
:109C600094F99D10002918DA2046FFF73FFFD4F839
:109C70000031DA044BD40025637EEB40DB07EAB207
:109C80004BD40135082DF7D123781BB1237C0BB1C0
:109C9000636863BB2E4800F03DFE7722C9B22046C0
:109CA000FFF768FB054620B30023CDE90633079B89
:109CB0000993002209A92046CDE907225CF0A8FB00
:109CC00001462046FFF742FB09A8FFF7BBFE08A8A4
:109CD000FFF7B8FE07A8FFF7FFFE15B106A8FFF7CC
:109CE000FBFE2378032B02D0237C032BBCD10AB0CC
:109CF00070BD716804220B68CDE90102154A00921B
:109D00001E6894F89D20772307A8B047CFE7637EAD
:109D1000002BB0D101236376ADE73820059201F026
:109D200015F9064618B1059A21465CF00FFC31463C
:109D30002046FFF70BFB2378032BD8D0237C032B83
:109D40009FD1D4E700000034406100205C7E0A0807
:109D5000637E0A08801A060090F86035934207D99E
:109D600002F5A77250F8220010B103689B6A1847E9
:109D7000002070472DE9F34105466E4686E80C0049
:109D8000134B45F8043B04460F4600F5C8782846B7
:109D90002C3500F0C5FCA845F9D196E8030004F283
:109DA0006453C4F85C7583E80300089BC4F86C3501
:109DB000084920462FF0DAFC074B1A6812B1074811
:109DC00058F02CFC20461C6002B0BDE8F08100BFBA
:109DD00030830A08F8810A08706100203C810A0873
:109DE0002DE9F041A2B00C4607A92EF029FE00286B
:109DF00055D000210D220CA80591ADF818100B913B
:109E000084F014FF2B4B611C1F68C9B20BAD0129F4
:109E1000F86A0A9546D1284B062205A90EF062FE83
:109E2000264B019305AB0093002411222946244BB5
:109E3000F86A8DF819400EF055FE04AA0DF10F01D5
:109E400028468DF83C40049430F004F938B31D499D
:109E5000DFF86C80482210A884F09EFE062610AC25
:109E60002268531E049AC2F3513202EB8312237903
:109E70008DF82430A368019305AB00930892434604
:109E800011222946F86A0EF02DFE0021B7EE000AD5
:109E900007A82EF0A1FF013E04F10C04E0D122B08E
:109EA000BDE8F0810091084B062205A90EF01AFECC
:109EB000B6E700BF40610020756E0A086D810A0890
:109EC00067810A086C2E0A0860810A082DE9F74F9D
:109ED00090F860650446002E51D17F2380F87035DC
:109EE00000F5C87500F5A768071D5FFA86FA182205
:109EF000FF21284684F09AFE85F85FA097F9269006
:109F0000B9F10A0F5CD03DDCB9F1040F0FDCB9F1F7
:109F1000020F0FDD442001F019F8834620B13B46C3
:109F20002A4621465CF078FEC8F800B002E0B9F19C
:109F3000090F39D0D8F8000050B1696EC5F86090AB
:109F400031B12C4B43F826102FF01EFE2FF014FEDB
:109F500058F8040B0AF101095FFA89F940B1036866
:109F60009B68984784F8609551462046FFF738FF74
:109F70000136092E05F1680507F12C07B5D103B0AC
:109F8000BDE8F08FB9F1150F28D0B9F1190FD1D173
:109F9000482000F0DBFF83460028C5D03B462A4618
:109FA00021465EF00DF8BFE7382000F0CFFF834672
:109FB0000028B9D03B462A4621465DF093FAB3E724
:109FC000302000F0C3FF83460028ADD0CDF800A0BC
:109FD0003B462A4621465DF075FFA5E7782000F054
:109FE000B5FF834600289FD03B462A4621465DF0B8
:109FF000E1FA99E77461002090F860358B4283BFE5
:10A00000682303FB010090F8DD0100207047000089
:10A0100090F860358B4283BF682303FB010090ED0D
:10A020006A0A9FED010A70470000000090F8603551
:10A030008B4206D901F5A77150F8210008B15CF0F8
:10A040008BBF9FED010A70470000000010B490F82C
:10A0500060458C420A4614D901F5A77450F8244093
:10A060007CB1E468246A640603D55DF8044BFFF70D
:10A07000DDBF682101FB020393ED6A0A5DF8044B22
:10A0800070479FED010AF9E70000000090F8603585
:10A090008B420BD901F5A77150F8210038B1C36884
:10A0A0001B6A1A4214BF012000207047002070472D
:10A0B00070B590F86035934204460E46154601D8B7
:10A0C000002070BD02F5A77350F823000028F7D0D8
:10A0D00003689B6998470028F2D0682202FB054478
:10A0E000D4F8AC313360ECE770B590F8603593424A
:10A0F00004460E46154601D8002070BD02F5A77330
:10A1000050F823000028F7D003689B69984700287F
:10A11000F2D0682202FB0544D4ED6C7AF4EE677A43
:10A12000F1EE10FAE8D6C6ED007AE6E770B590F8E1
:10A130006035934204460E46154601D8002070BD96
:10A1400002F5A77350F823000028F7D003685B6975
:10A1500098470028F2D0682202FB0544D4F8B431B5
:10A160003360ECE790F8603593420ED902F5A7739F
:10A1700050F823305BB1682303FB020292F8EC0134
:10A1800030B1D2F8E8310B607047002070471846B4
:10A190007047000008299DBF2C2303FB0100406885
:10A1A000002070472DE9F04F4B4B2DED028B1B68C3
:10A1B000DB6A93F89C3089B00446002B00F086805F
:10A1C000DFF82CB19FED458A4FF0000994F8603517
:10A1D0005FFA89F5AB4279D905F5A77354F82300E6
:10A1E00000285DD003685B6B9847682303FB054339
:10A1F000074693F8DC31834252D2032861D8DFE866
:10A2000000F04F025259364E4FF000083EF012FB5C
:10A2100094F86025AA4284BF682202FB05424FF0F1
:10A22000680105F1010301FB05458CBFD2F8A821A7
:10A2300018EE102A8246D5F8B001CDE90632F6F7BD
:10A2400063F9079ACDE904011046F6F75DF9069B1C
:10A250000096CDE902015A460421504637F0A6FC8B
:10A260000123204A84F8713585F8DC71D372D4F863
:10A270006C354BB3002255B25957481C03D04145A9
:10A2800002F10102F7D194F97035AB4208DBD4F842
:10A290006835D4F8640542463146984784F87055CD
:10A2A00009F1010992E72C2303FB05430E4E93F9B4
:10A2B0002D80ABE72C2303FB05430C4E93F92E8036
:10A2C000A4E70026B046A1E71D46DCE709B0BDECD7
:10A2D000028BBDE8F08F00BF40610020000000004D
:10A2E00081810A08CD610020F29E0B0878810A085E
:10A2F00090810A0890F860358B4207D901F5A77163
:10A3000050F8210010B10368DB691847002070473E
:10A3100008299CBF682303FB010000F5C870704743
:10A3200090F86035934207D902F5A77250F82200E1
:10A3300010B103685B6A18470020704790F86035D9
:10A340008B420DD901F5A77350F8233043B1682330
:10A3500003FB0101012081ED730A81F8C8017047F8
:10A3600000207047F8B5002402460E4625462C27EB
:10A3700092F86035E1B28B4210D901F5A77352F81B
:10A3800023304BB107FB01239B689E4204D110464A
:10A39000FFF7D4FF2843C5B20134E9E72846F8BDEA
:10A3A0002DE9F04F002493B005460E46174621468E
:10A3B0002F2206A8059405F5A76984F037FC05F15E
:10A3C0002A0A4FF02C0B05F5F8730BFB04F259F831
:10A3D000040B1AF90210E5B230B951B90134092C55
:10A3E000F3D14FF0010813E0682262439A5891427A
:10A3F00012D01548154B006801930135EDB2009558
:10A40000134BC06A324639460EF06CFB4FF0000821
:10A41000404613B0BDE8F08F05A9332203935CF0EA
:10A420007DFE039B804605A90028D7D106480191EF
:10A430000135EDB200680095054BC06A32463946D9
:10A440000EF050FBE4E700BF40610020C6810A081F
:10A45000B8810A082DE9F04FDFF88090DFF880A07E
:10A46000DFF880B08DB00646002796F86035FCB264
:10A47000A3422ED9682505FB046595F8E43133B372
:10A4800095F8E51119BB4FF001082022444404A8B7
:10A4900089F8198084F0CAFB07EE904A4AF210430B
:10A4A000F8EEE77A03AA4C21ADF828305046242371
:10A4B000CDED037A39F090FA3EF0BCF99BF800300C
:10A4C000054A0094042137F071FB85F8E5810137D6
:10A4D000CBE70DB0BDE8F08FD0810A08CD61002038
:10A4E000A5640020F02200202DE9F04F2F4B1E68BC
:10A4F00085B0044646B1D0F85C15304633F0FAFC1E
:10A5000010B1304632F046FC58F0BAF84FF000086F
:10A5100001904FF02C0A4FF0680B94F860355FFA09
:10A5200088F5AB4239D904EB8507D7F8380588B3ED
:10A530000AFB05430BFB054993F92A20D9F8F011D2
:10A540008A4227D132B30268D2689047D7F83805DB
:10A550000268126B904799F8DD2112B1019BC9F88E
:10A56000E031BEB1D4F85C15304633F0C3FC88B19D
:10A5700058F08EF8CDE9021002460B46D7F83805A0
:10A5800029465DF011FBDDE90232D7F8380529468E
:10A590005DF088FB08F10108BFE72046FFF702FEE7
:10A5A000204605B0BDE8F04FFFF754BF1864002007
:10A5B0002DE9F0474FF000082DED028B0446894647
:10A5C000B0EE408A474601264FF0680A94F860359D
:10A5D0005FFA88F5AB421AD929FA05F3DB070AD5E9
:10A5E00005F5A77354F8230078B10368B0EE480A64
:10A5F0009B6B984706400AFB054508F1010895F852
:10A60000DC319F4238BF1F46E0E70646F3E727B933
:10A610007F23A4F87035034BDF72BDEC028B30460C
:10A62000BDE8F087CD61002090F860358B4207D9F6
:10A6300001F5A77150F8210010B10368DB6B1847D2
:10A64000002070470B46114690F860259A4207D9C2
:10A6500003F5A77350F8230010B103681B6C18476B
:10A660007047000070B504460E46002594F860352A
:10A67000E9B28B4205D932462046FFF7E3FF0135A8
:10A68000F4E770BD2DE9F84390F8605502460024C8
:10A6900000F12A062C2700F5F8784FF06809E1B29E
:10A6A0008D420FD907FB04F309FB04F0F35658F869
:10A6B0000000834209D11BB11046FFF79DFC10B189
:10A6C0000134ECE70120BDE8F8830020FBE700003F
:10A6D00010B590F860258A42044617D9682202FB1B
:10A6E000010393F8DC31022B03D004D9032B18BFEC
:10A6F0000023184610BDFFF797FF48B92046FFF723
:10A70000C1FF00280CBF06230123F2E70023F0E776
:10A710000623EEE7014B1868704700BF7061002008
:10A7200010B5034904462FF021F8204610BD00BFA4
:10A73000B0830A0810B50446203048F0BFFB044B34
:10A7400004491C6020462FF011F8204610BD00BFC0
:10A75000986100204C850A082DE9F3410022B7EEEC
:10A76000000A022105462EF06BFC28465DF090FCA5
:10A7700048F01EFC234B1E680446F06A03685B6ABF
:10A7800098470B46022102460091204648F0ACFB58
:10A79000B5F94A70002F13DDD6F82C80D8F80030B8
:10A7A00040465B68BCB2984728B198F84D3013B169
:10A7B000C92FA8BFC824B06A036821465B689847C0
:10A7C00095F949002022002111F0AEFFC4B24BF0F0
:10A7D000AFFA4BF04DFA70B9B06A036801345B68A8
:10A7E000E4B205219847072CF1D9074802B0BDE82B
:10A7F000F04157F00DB8072CF7D885F8494002B062
:10A80000BDE8F08140610020B0840A0810B504461C
:10A810005DF0F4FB2046BDE810405DF01FBC000079
:10A820002DE98048284BDFF8A490DFF8A4A0DFF8DA
:10A83000A4B01446012293B005460E461A704FF09C
:10A84000000857F01DFFD9F800300393A0EB080271
:10A8500041F287339A4207461FD9CDE90056039843
:10A860005346342205A9C06A0EF03CF9214605A8DA
:10A87000049456F0BDFFCDE9005603985B463422A0
:10A8800005A9C06A0EF02EF904943DF0D3FF049B95
:10A8900005AA022137F070F9B8463DF0CBFF3DF034
:10A8A00065FA3DF0C7FF3FF029F90A2105A80DF030
:10A8B00021FF039B986A036805215B68984705A8F8
:10A8C0000DF024FFBDE700BF9C6100204061002027
:10A8D0001DF90A08A5B80B080FB400B595B016AA63
:10A8E000002152F8043B039205A83C2201930491F5
:10A8F00084F09CF9054A019B402104A856F020FFF2
:10A90000039A034804A9FFF78BFF00BFC8840A0815
:10A91000DE840A080FB407B504AA034852F8041BE2
:10A920000192FFF77DFF00BFF0840A08014B186811
:10A93000704700BF9861002008B50449102284F0D8
:10A940001BF9B0FA80F0400908BD00BFA0610020EB
:10A950001022002184F06AB910B50446FFF7F8FF11
:10A96000204610BD0378416023F00D03022A0370D6
:10A9700008D0032A0AD0012A03D1DBB243F0010335
:10A9800003707047037843F00803F9E7037823F076
:10A99000050343F00503F3E773B504460E46154679
:10A9A0000193FFF7D5FF2046C4E90265069A019995
:10A9B000FFF7D8FF02B070BD0078420704D4030748
:10A9C00004D400F001007047032070470220704754
:10A9D000F0B587B004461546FFF7EEFF88420F46F4
:10A9E000064605D163682B600126304607B0F0BDEE
:10A9F00000230328019301D0032913D131F064F916
:10AA000008B90026F1E7012301AA214630F098FF9A
:10AA10000028F6D0DDED017A9FED337A67EE877A74
:10AA2000CDED017A032E32D8DFE806F002091624B4
:10AA30006468032FE5D8DFE807F02C2E3C49FCF7CB
:10AA400093FB90F87C32DB07DBD56468FCF78CFB6A
:10AA5000D0F870321C44ECE702A8FFF779FFFCF74E
:10AA600083FB02A9FCF786F906460028BDD064687E
:10AA7000039BEFE7D4ED017A9DED017AF8EEE77ADA
:10AA800077EE877AFDEEE77A17EE904AD1E7002459
:10AA9000CFE72C60A8E7FCF767FB90F87C6216F024
:10AAA0000106AED0FCF760FBD0F87032E41A2C60DF
:10AAB0009BE702A8FFF74CFFFCF756FB02A9FCF747
:10AAC00059F90646002890D0039BEFE707EE904A1D
:10AAD0009DED017AF8EEE77A77EEC77AFDEEE77A38
:10AAE000C5ED007A80E700BF0000C84273B501AA37
:10AAF00005460E46FFF76CFF044620B10199324629
:10AB00002846FFF72FFF204602B070BD13B514464C
:10AB100001AAFFF75DFF48B1DDED017A9FED047AF0
:10AB2000F8EEE77A67EE877AC4ED007A02B010BDDE
:10AB30000AD7233C07EE900A9FED090AF8EEE77A60
:10AB400008B527EE800A81F069FCDFED067AB4EEE5
:10AB5000E70AF1EE10FAD8BFB0EE670A08BD00BFF1
:10AB600050E0EF300AD7233C10B50446806811F05E
:10AB70005FFF20B1E068BDE8104011F06DBF10BD6F
:10AB800073B5856804460E461DBBC36823B98B6840
:10AB90008360CB68C3600125636873B92378DB07E2
:10ABA0000BD52046FFF708FF01AA01463046FFF704
:10ABB0000FFF10B1019B636005462046FFF7D4FFED
:10ABC00020B9B368A360F368E3600125284602B0AA
:10ABD00070BD0025E0E700000D4B83424FF00003FD
:10ABE0008B4106DA00F1255000F5311000F5E050F8
:10ABF0007047084B98424FF0FF3371EB0303BEBF21
:10AC000000F1564000F5130000F52440704700BFE6
:10AC100000D2496B002EB69490EA010F01D4401A7D
:10AC20007047C317401A63EBE1710D4B83424FF03D
:10AC300000038B4106DA00F1255000F5311000F5D4
:10AC4000E0507047074B98424FF0FF3371EB03031E
:10AC5000BEBF00F1564000F5130000F524407047D8
:10AC600000D2496B002EB69470B52DED028B84B0E6
:10AC7000044668460D46FFF76BFEFCF775FA694619
:10AC8000FCF778F8064608B3A368029ADFED128A4B
:10AC900003999B1A07EE903AF8EEE77A67EEA87AE6
:10ACA000C5ED007AE068FFF7B7FF08EE100AA0686C
:10ACB000024402EBD272B8EEC88A5010FFF73AFF96
:10ACC00028EE288A28EE000A85ED010A304604B0F5
:10ACD000BDEC028B70BD00BFF67C8E3F37B5002304
:10ACE0000C4601AA022105460193FFF771FE10B937
:10ACF000002003B030BD21462846FFF7B5FF0028ED
:10AD0000F6D0DDED017AF8EEE77AC4ED027AF0E7ED
:10AD100038B52DED028B0C460246C168E068FFF79E
:10AD20007BFF9568A46808EE100A601900EBD070EC
:10AD30004010641BFFF7FEFE07EE904AF8EEE77A3C
:10AD4000F8EEC80A87EE807ABDEEC70A10EE103A18
:10AD50005B4200EE103AB8EEC00A81F081FDDFEDF3
:10AD6000087A30EE270ABDEC028BB5EEC00AF1EE90
:10AD700010FA44BFDFED037A30EE270A38BD00BF7A
:10AD8000DB0FC93FDB0FC94030B52DED028B0B4601
:10AD900085B08C68D0E90251D868FFF73DFF08EE16
:10ADA000100A601900EBD0704010FFF7C3FE641B5F
:10ADB00007EE904AF0EE400AB8EEC88A9FED060A08
:10ADC000F8EEE77A28EE008A27EE800A68EE200A7D
:10ADD00005B0BDEC028B30BD8262363C82B002B061
:10ADE000FFF7D2BFF0B52DED028B0D4689B08C6810
:10ADF0000646D0E90271E868FFF70EFF08EE100A78
:10AE0000E01900EBD0704010FFF794FE73686A6899
:10AE10009FED0E1A9B1A07EE903AE41BB8EEE77A04
:10AE2000F0EE400A07EE904A9FED090AB8EEC88A94
:10AE3000F8EEE77A28EE008A27EE011A27EE800A5C
:10AE400068EE200A09B0BDEC028BF0BD0AD7233CA6
:10AE50008262363C10B52DED028B84688A680B4601
:10AE6000111B08EE901AC168D868FFF7D5FE22447E
:10AE700002EBD27208EE100A5010FFF75BFEB8EE3C
:10AE8000C88AF8EEE88A28EE000A20EE000AA8EE4A
:10AE9000A80A81F02FFEBDEC028BDFED027A20EED6
:10AEA000270A10BD8262363C094B984206DDC0F18C
:10AEB000D64000F5930000F5A4407047054B98423A
:10AEC000BEBFC0F1144000F5360000F538507047A1
:10AED00000E9A43500175BCAF8B52DED028BDFED54
:10AEE000148A076820EE280A0646FDEEC07A0D4651
:10AEF00017EE904A04EBD47007EB6000B0EE608A66
:10AF0000FFF718FE28EE288A3819C8EE007AFFF7F6
:10AF1000CBFF306017EE900AF6F720F82B68C018C8
:10AF200041EBE371FFF758FEBDEC028B2860F8BDE2
:10AF300002AAB34200F10C010830FFF7CDBF0000B8
:10AF40000148FFF705BD00BFA06100200121884234
:10AF500038BF08467FF048BBFFF7F8BF08B17FF065
:10AF600047BB7047FFF7FABF00214FF0FF3310B522
:10AF700000220363044601600171C0F805104172AC
:10AF800080F8251000F13C0300F50B70D9709A6031
:10AF9000DA601A615A619A61DA611A625A629A62D7
:10AFA000DA631A645A649A64DA641A655A659A65AF
:10AFB000DA65DA661A675A677C339842E6D1214629
:10AFC00004F5167007F016FC044B1A6822B9044900
:10AFD0001C6020462EF0CAFB204610BDB061002048
:10AFE000B0870A0873B5D0F83C3201919942044603
:10AFF00013D0D0F84032994218D0D0F844328B4266
:10B0000016D102200AE0D4F8343253B3D4F83832DF
:10B010004BB34FF0030002B070BD002094F8223013
:10B020008342F8D8431C84F82230F4E70120F5E786
:10B03000D0F83062002EE6D194F841233546B600B0
:10B040009AB1A319C3F83012A319019AC3F83C228C
:10B0500094F82230AB429CBF6B1C84F82230284607
:10B06000D9E70126E8E70226E6E704F50C7001A916
:10B0700030442FF025FAE7E738B504460D462FF0A7
:10B0800095F9291D201D2FF091F905F1080104F112
:10B0900008002FF065FA05F1140104F114002FF0F7
:10B0A0005FFA05F1200104F120002FF059FA05F1B3
:10B0B0002C0104F12C002FF00DF905F1300104F101
:10B0C00030002FF015FA05F13C0104F13C002FF09F
:10B0D00047FAAB6BA3636B6B636338BD2DE9F04339
:10B0E000A1B00023002500F13C0706468DF807506B
:10B0F00003930493059306930793089309930A9384
:10B100000B93109311931293139314931593169317
:10B11000179318931C931D931E9300F50F78B9464F
:10B1200058F8043BF3B1F26E934223D0D6F8E820EE
:10B13000934221D0D6F86421934213D10221EBB27D
:10B1400099420FD0C1EB411109EB8104214601A8BE
:10B15000FFF792FF39462046FFF78EFF01A93846D8
:10B16000FFF78AFF0135032D07F17C07D8D121B005
:10B17000BDE8F0830021E2E70121E0E72DE9F04797
:10B1800006460F461546804604464FF0000A3946EB
:10B190003046FFF727FF626FBA425FFA8AF90ED195
:10B1A000C3B2022B0BD87C2202FB0A66012086F870
:10B1B0003E0086F83F3085F80090BDE8F0870AF140
:10B1C000010ABAF1030F04F17C04E0D100243946EE
:10B1D0003046FFF707FFD8F86C205FFA84F912B900
:10B1E000C3B2022B22D90134032C08F17C08EED122
:10B1F00000244FF07C0906F13E0A39463046FFF73D
:10B20000F1FE034609FB04F05FFA84F81AF8002007
:10B2100012B9DBB2022B12D90134032CEDD196F80E
:10B220002300042814D9194857F0F8F97C2000FBB2
:10B230000464012084F83E0084F83F30BBE70644F4
:10B24000012086F83E0086F83F3085F80080B4E79C
:10B2500006F54371002251F8043BBB42D4B208D139
:10B26000A04202D8631C86F8233003342C700020DF
:10B27000A3E73BB9421C06EB800086F82320C0F808
:10B280000C73F2E70132052AE5D1F0E7EC850A08F4
:10B29000C9B200EB8101D1F83C3253B1026F934245
:10B2A0000AD0D0F8EC20934208D0D0F8682193421D
:10B2B00006D04FF003007047002070470120704710
:10B2C0000220704759B190F82030032B07D05A1C48
:10B2D00080F8202000EB83004161012070470020AE
:10B2E000704700002DE9F8430F469146044600F5EB
:10B2F000BA7894F83E5035B97C344445F9D10025EC
:10B300002846BDE8F88300234A46394601200DF05F
:10B310007FF800210646E06E0DF08AF88642EBD1F8
:10B32000EEE700002DE9F043DFF87C8085B00446AD
:10B3300000F50F7600257C27B14656F80C3CD9F86D
:10B3400000209342E9B206F1040619D1C3B12046A8
:10B35000FFF79EFFC0B207FB004090F83E307BB97C
:10B3600003A9A9F10C0003932FF0AAF83DF062FAAB
:10B3700056F8043C009342462B46012136F016FC59
:10B380000135032DD8D104F16C0504F5F07429685A
:10B3900021B9AB6813B128462DF06EFB7C35A54270
:10B3A000F5D105B0BDE8F08308860A0838B5044633
:10B3B0001546FFF76DFFC0B2022808D87C2303FBB7
:10B3C000004029465030BDE838402FF0B9B838BDAC
:10B3D00038B504461546FFF75BFFC0B2022808D80F
:10B3E0007C2303FB004029465C30BDE838402FF049
:10B3F000A7B838BD37B50D4604468DED010AFFF7F5
:10B4000047FF022D07D8C0B27C2303FB004001A9EF
:10B4100068302EF047FF03B030BD000038B5054658
:10B42000FFF736FFC4B2022C13D8C4EB4414A400B7
:10B430003C3504F10800284400212DF01DFB04F1E7
:10B44000340104F1300029442844BDE838402FF08D
:10B4500037B838BD70B505460E461446FFF718FFDD
:10B46000C3B2022B0DD87C2000FB035394E80700E5
:10B47000443383E8070031462846BDE87040FFF7B3
:10B48000CDBF70BD37B504461546FFF701FFC0B20A
:10B49000022809D87C2303FB00400DF1070140304E
:10B4A0008DF807502EF082FF03B030BD1FB590F924
:10B4B0002C30044623B390F921300BB36846FFF7D4
:10B4C0004BFAFBF751FE6946FBF704FCC0B1DDED1A
:10B4D000037A9FED0C0AF8EEE70ADDED027AF8EE4A
:10B4E000E77A0123C0EE800A84F83D3387EE800AB4
:10B4F00007F0C2FBDFED047A20EE270A84ED0A0A8A
:10B5000004B010BD8096184B35FA8E3C024690F977
:10B51000210058B192F8400340B1114491F92C0236
:10B5200020B192F92400033818BF012070470000B1
:10B5300038B590F8223005465BB100242346E1B2CD
:10B540002846FFF7E3FF08B10133DBB20134032CD7
:10B55000F5D1184638BD000090ED0A0A704700008A
:10B5600038B50C46D1ED066A11460546FFF790FE48
:10B57000C3B27C2000FB0353D4ED087AD3ED260A36
:10B5800094ED076AD3ED255A93ED245A26EE600A0E
:10B5900067EEA00AA5EEA70AF0EE607AE5EE867ADD
:10B5A000B7EE007AA6EEE67A67EEE60AB1EE400A5A
:10B5B000E5EE070A81F054F99FED071ADFED070A5F
:10B5C00040F61C0011F072F8D5ED0A7ABDE838405B
:10B5D00030EE270A11F056B8DB0F4940DB0F49C0A7
:10B5E0002DE9F04190F822308B4204460D4602D2FC
:10B5F0000020BDE8F081FFF74BFEC0B204F13C062D
:10B60000C0EB401006EB8000083013F091FDDFED39
:10B61000157AB0EEC00AB4EEE70AF1EE10FAE7D4FC
:10B6200029462046FFF734FEC5B27C2000FB0547C3
:10B630003B6F002BDCD0032DDAD000FB05603030EF
:10B64000D7F86C802EF068F9D7E91B32934201D10C
:10B65000984505D07C2000FB0544C4F86C80C7E702
:10B660000120C6E7000000342DE9F74F04460E46DE
:10B67000174600F50F7A4FF0000B5AF8049B5FFA5B
:10B680008BF8B9F1000F26D041462046FFF73EFF68
:10B6900008B341462046FFF7FBFD7C23C0B203FB05
:10B6A000004090F83E505DB908F101031B4ADBB23F
:10B6B0003946304656F044F8284603B0BDE8F08FCE
:10B6C0005AF8102C914506D0154A3946304656F0A6
:10B6D00037F80025F0E70BF1010BBBF1030FCCD1DC
:10B6E0004FF0000894F822305FFA88F18B420DD9B0
:10B6F00020460191FFF774FF054620B901992046C5
:10B70000FFF704FF20B908F10108EBE70125D3E7B3
:10B71000044A3946304656F013F8CDE730860A0819
:10B7200045860A086A860A082DE9F0412DED048B4A
:10B7300090F842139FED348ADFED348A9FED349AFE
:10B7400082B00646FFF7A4FD06F13C07C5B27C2097
:10B7500000FB057554354FF0000896F822205FFA7B
:10B7600088F39A424ED919463046FFF7CFFE10B9FA
:10B7700008F10108F1E719463046FFF789FDC4B228
:10B780007C2000FB0474D4ED157AF0EEE77AF4EE39
:10B79000C87AF1EE10FA04F154040ED5D4ED017A12
:10B7A000F0EEE77AF4EEC87AF1EE10FA05D5002053
:10B7B00002B0BDEC048BBDE8F0812946204613F0B1
:10B7C000CFFCB4EEE80AF1EE10FAF0DC2946204690
:10B7D00012F0B2FFB4EEC90AF1EE10FAE7DC21462E
:10B7E000284612F0D9FE68468DED000ACDED010A1B
:10B7F00012F08EFFDFED077AB4EEE70AF1EE10FAF1
:10B80000B6DDD4E70120D3E700000034DB0FC93FE9
:10B81000920A863F00004843022910B5044608D822
:10B82000FFF736FD7C23C0B203FB004494F83D00D3
:10B8300010BD0020FCE7000013B590F84213019101
:10B840000446FFF7E9FF30B10199204602B0BDE898
:10B850001040FFF75BBE02B010BD0000F7B590F9D5
:10B8600021500446002D73D090F84053002D6FD026
:10B8700090F84213FFF7D0FF94F83D33064613B912
:10B880002046FFF713FE002594F82020EBB29A42E1
:10B8900007D904EB83030135586903689B6898470F
:10B8A000F2E756F0EDFE0027224604F5BA7140F2A9
:10B8B000F315D2F89C30C31AAB428CBF002301238E
:10B8C00082F83D307C32914247EA0307F1D194F986
:10B8D0002430032B07D194F83C33002B3BD0D4F811
:10B8E0003803002849D167B1236B013309D032F006
:10B8F000DBFC216B32F0FEFA18B132F0D5FC31F0EE
:10B900005DFB94F92C32002B3AD194F92D32CBBB4C
:10B9100094F92E3213B1022384F8423394F842137F
:10B920002046FFF779FF8642054611D032F0BCFC75
:10B930004FF6FF7132F0DEFA50B1002D14BF002235
:10B940000422019232F0B0FC019A032132F064FA31
:10B95000284603B0F0BD012384F83C330420FFF7F0
:10B96000F5FA054610B1214606F0DAFF94F92430C5
:10B97000C4F83853032BB2D0B5E706F0DFFFB2E7C7
:10B980000023C9E70123C7E738B590F92130044601
:10B99000D3B190F84053BDB1FFF77AFCC0B2022892
:10B9A00012D87C2303FB0044D4ED1A7A9FED087A69
:10B9B000F4EEC77AF1EE10FA06D4B7EE087AF4EE98
:10B9C000C77AF1EE10FA00DD0025284638BD00BF29
:10B9D000ABAA2A3F70B5D0F8085315F400350446D9
:10B9E0000E460DD190F840335BB90A78072A07D884
:10B9F000012303FA02F290F83F33134380F83F33F8
:10BA000070BD94F82020EBB29A42F9D904EB83037D
:10BA1000314658690368DB6898470135F1E7000053
:10BA200038B505466C242B591BB1002128192DF07F
:10BA300023F87C34B4F5F07FF5D138BD014B18689C
:10BA4000704700BFB06100202DE9F04FB24BD3F832
:10BA500000800446D8F8040003688DB09B689847BE
:10BA6000002507464FF0010909FA05F33B4240F073
:10BA700092820135202DF7D1D8F804000368DB68E5
:10BA80009847002507464FF0010909FA05F33B42A4
:10BA900040F0C3820135202DF7D1D8F804000368A7
:10BAA0009B689847002507464FF0010909FA05F3FE
:10BAB0003B4240F0F1820135202DF7D1D8F8040047
:10BAC00003689B689847002507464FF0010909FA6B
:10BAD00005F33B4240F01C830135202DF7D1D8F807
:10BAE0000400DFF840B203689B6898470025049083
:10BAF000049A0123AB40134240F046830135202DC8
:10BB0000F6D1D8F80400DFF81CB20368DB68984768
:10BB100000250490049A0123AB40134240F00584B1
:10BB20000135202DF6D1D8F804000368DB6898476A
:10BB3000002507464FF0010909FA05F33B4240F0A2
:10BB4000BF840135202DF7D1D8F804000368DB68E5
:10BB50009847002507464FF0010909FA05F33B42D3
:10BB600040F0ED840135202DF7D1D8F804000368AA
:10BB70009B689847002507464FF0010909FA05F32D
:10BB80003B4240F01B850135202DF7D1D8F8040049
:10BB900003689B689847002507464FF0010909FA9A
:10BBA00005F33B4240F04A850135202DF7D1D8F806
:10BBB000040003689B689847002507464FF0010979
:10BBC00009FA05F33B4240F079850135202DF7D184
:10BBD000D8F804000368DB689847002507464FF053
:10BBE000010909FA05F33B4240F0A4850135202DF7
:10BBF000F7D14A4B089308AF0425D8F8040003682E
:10BC00009B689847002683460123B34013EA0B0F35
:10BC100040F0CB850136202EF6D1D8F80400036819
:10BC2000DB689847002683460123B34013EA0B0FD5
:10BC300040F001860136202EF6D1013D15F0FF05BA
:10BC400007F10107D9D1D8F8040003689B68984729
:10BC50004FF00109074609FA05F33B4240F02F86F1
:10BC60000135202DF7D1D8F804000368DB68984728
:10BC7000002507464FF0010909FA05F33B4240F061
:10BC80005A860135202DF7D1D8F8040003689B6847
:10BC90009847002507464FF0010909FA05F33B4292
:10BCA00040F085860135202DF7D1D8F804000368CF
:10BCB000DB689847002507464FF0010909FA05F3AC
:10BCC0003B4240F0B0860135202DF7D1144B07934D
:10BCD000D8F8040003689B68984700258346012331
:10BCE000AB4013EA0B0F41D000275FFA85F9D4F877
:10BCF000083313F4803A31D107AB4946DB5D049336
:10BD00001A462046FFF7EEFA049B0646002800F08C
:10BD1000C686CDE908AA07E0406100200C0D0E0F91
:10BD200020212223801A0600099B0B930022012167
:10BD30000BA8CDE9092204F06FFF01462046FFF76A
:10BD4000C1FA0BA8FDF77EFE0AA8FDF77BFE09A845
:10BD5000FDF7C2FE16B108A8FDF7BEFE94F8233029
:10BD6000052B00F048810137042FC0D10135202D6B
:10BD7000B5D1D8F804000368DB68984700258346EE
:10BD80000123AB4013EA0B0F38D000275FFA85F987
:10BD9000D4F8083313F4803A28D107AB4946DB5D69
:10BDA00004931A462046FFF79DFA049B0646002896
:10BDB00000F08486CDE908AA0022099B0B93114666
:10BDC0000BA8CDE9092204F027FF01462046FFF722
:10BDD00079FA0BA8FDF736FE0AA8FDF733FE09A88D
:10BDE000FDF77AFE16B108A8FDF776FE94F8233029
:10BDF000052B00F000810137042FC9D10135202D1A
:10BE0000BED1D8F8040003689B6898470026824694
:10BE10000123B34013EA0A0F31D010255FFA86F9E7
:10BE2000D4F8083313F0080B20D12A46494620469F
:10BE3000FFF758FA0746002800F04F86CDE909BB06
:10BE40000A9B002201210BA8CDE90A2301F048FC3E
:10BE500001462046FFF736FA0BA8FDF73DFE0AA87B
:10BE6000FDF73AFE17B109A8FDF736FE94F8233026
:10BE7000052B00F0C0800135EDB2142DD0D1013674
:10BE8000202EC5D1D8F8040003689B689847002687
:10BE900082460123B34013EA0A0F34D014255FFA17
:10BEA00086F9D4F8083313F4001B24D12A464946F6
:10BEB0002046FFF717FA0746002800F02186CDE953
:10BEC00008BB099B0B93002201210BA8CDE9092295
:10BED00002F018F801462046FFF7F4F90BA8FDF729
:10BEE000B1FD0AA8FDF7AEFD09A8FDF7F5FD17B1F4
:10BEF00008A8FDF7F1FD94F82330052B7BD0013520
:10BF0000EDB2182DCDD10136202EC2D1D8F80400C3
:10BF10000368DB689847002682460123B34013EA92
:10BF20000A0F34D014255FFA86F9D4F8083313F4D5
:10BF3000001B24D12A4649462046FFF7D3F907467D
:10BF4000002800F0ED85CDE908BB0022099B0B938A
:10BF500011460BA8CDE9092201F0D4FF0146204685
:10BF6000FFF7B0F90BA8FDF76DFD0AA8FDF76AFD14
:10BF700009A8FDF7B1FD17B108A8FDF7ADFD94F8CC
:10BF80002330052B37D00135EDB2182DCDD1013638
:10BF9000202EC2D12FE0D4F8083313F0010A25D1A6
:10BFA0005FFA85FB1E2259462046FFF79BF906469D
:10BFB00020B3CDE908AA099A0B9200230822012197
:10BFC0000BA8CDE9093303F0C7FA01462046FFF775
:10BFD00079F90BA8FDF736FD0AA8FDF733FD09A88E
:10BFE000FDF77AFD16B108A8FDF776FD94F8233029
:10BFF000052B7FF43EAD0DB0BDE8F08FD8F80410EE
:10C0000004220B68CDE90102B84A0092D3F800A0DF
:10C010005A461E2309A8D047CDE7D4F8083313F0B9
:10C02000010A24D15FFA85FB1E2259462046FFF7FC
:10C0300059F9064608B3CDE908AA099B0B930622D5
:10C0400000210BA8CDE9091103F086FA014620462C
:10C05000FFF738F90BA8FDF7F5FC0AA8FDF7F2FC8D
:10C0600009A8FDF739FD16B108A8FDF735FD94F8CC
:10C070002330052B7FF40EADBDE7D8F80410042261
:10C080000B68CDE90102994A0092D3F800A05A4604
:10C090001E2309A8D047D0E7D4F8083313F4805AF8
:10C0A00021D15FFA85FB0D2259462046FFF71AF988
:10C0B0000646F0B1CDE909AA0A9B0022CDE90A2380
:10C0C000012108220BA804F0B5FA01462046FFF72B
:10C0D000F9F80BA8FDF700FD0AA8FDF7FDFC16B165
:10C0E00009A8FDF7F9FC94F82330052B7FF4E3ACA5
:10C0F00081E7D8F8041004220B68CDE901027B4ADD
:10C100000092D3F800A05A460D230AA8D047D3E7DF
:10C11000D4F8083313F4801A21D15FFA85FB2C225E
:10C1200059462046FFF7DEF80646F0B1CDE909AAE8
:10C130000A9B0022CDE90A23012108220BA804F062
:10C14000A7FB01462046FFF7BDF80BA8FDF7C4FC8E
:10C150000AA8FDF7C1FC16B109A8FDF7BDFC94F8CB
:10C160002330052B7FF4B8AC45E7D8F8041004223F
:10C170000B68CDE901025D4A0092D3F800A05A464F
:10C180002C230AA8D047D3E7D4F8083313F48077D8
:10C190003FD15FFA85F90C2249462046FFF7A2F805
:10C1A0000646002800F08480CDE90677079B0A93B5
:10C1B0004FF0000A692249462046CDF81CA0FFF73F
:10C1C00091F80746002800F08180CDE908AA099B74
:10C1D0000B9300221A2309920BA901220AA801F04D
:10C1E00007F801462046FFF76DF80BA8FDF774FC31
:10C1F00009A8FDF771FC17B108A8FDF76DFC0AA8A6
:10C20000FDF76AFC07A8FDF767FC16B106A8FDF765
:10C2100063FC94F82330052B3FF4EDAED4F80833DB
:10C2200013F480777FF46AAC5FFA85F90C224946F3
:10C230002046FFF757F80646002859D0CDE9067783
:10C24000079B0A934FF0000A682249462046CDF822
:10C250001CA0FFF747F80746002857D0CDE908AAE9
:10C26000099B0B9300221A2309920BA901220AA809
:10C2700000F0BEFF01462046FFF724F80BA8FDF7AB
:10C280002BFC09A8FDF728FC17B108A8FDF724FC32
:10C290000AA8FDF721FC07A8FDF71EFC16B106A8A9
:10C2A000FDF71AFC94F82330052B7FF427ACA2E6A7
:10C2B000D8F8041004220B68CDF800B0CDE90102D3
:10C2C0004A461F6807A80C23B8476FE7D8F8041040
:10C2D00004220B68CDF800B0CDE901024A46D3F83C
:10C2E00000A009A86923D04771E700BF801A0600A3
:10C2F000D8F8041004220B68CDF800B0CDE9010293
:10C300004A461F6807A80C23B84799E7D8F80410D5
:10C3100004220B68CDF800B0CDE901024A46D3F8FB
:10C3200000A009A86823D0479AE7D4F8083313F48B
:10C3300080773DD15FFA85F90C2249462046FEF709
:10C34000D1FF0646002800F08180CDE90677079BE3
:10C350000A934FF0000A692249462046CDF81CA0F6
:10C36000FEF7C0FF074600287ED0CDE908AA099B4A
:10C370000B9300221A230BA90AA8099200F038FF98
:10C3800001462046FEF79EFF0BA8FDF7A5FB09A876
:10C39000FDF7A2FB17B108A8FDF79EFB0AA8FDF761
:10C3A0009BFB07A8FDF798FB16B106A8FDF794FBC9
:10C3B00094F82330052B3FF41EAED4F8083313F461
:10C3C00080777FF4ADAB5FFA85F90C2249462046B1
:10C3D000FEF788FF0646002855D0CDE90677079B73
:10C3E0000A934FF0000A682249462046CDF81CA067
:10C3F000FEF778FF0746002853D0CDE908AA099B2D
:10C400000B9300221A230BA90AA8099200F0F0FE50
:10C4100001462046FEF756FF0BA8FDF75DFB09A875
:10C42000FDF75AFB17B108A8FDF756FB0AA8FDF760
:10C4300053FB07A8FDF750FB16B106A8FDF74CFB10
:10C4400094F82330052B7FF46BABD4E5D8F80410B7
:10C4500004220B68CDF800B0CDE901024A461F68FE
:10C4600007A80C23B84772E7D8F8041004220B6819
:10C47000CDF800B0CDE901024A46D3F800A009A8E2
:10C480006923D04773E7D8F8041004220B68CDF86D
:10C4900000B0CDE901024A461F6807A80C23B8473F
:10C4A0009DE7D8F8041004220B68CDF800B0CDE960
:10C4B00001024A46D3F800A009A86823D0479EE7A6
:10C4C000D4F8083313F0200A24D15FFA85FB1C222C
:10C4D00059462046FEF706FF064608B3CDE908AAEE
:10C4E0000022099B0B9311460BA8CDE9092203F00A
:10C4F00031FC01462046FEF7E5FE0BA8FDF7A2FA47
:10C500000AA8FDF79FFA09A8FDF7E6FA16B108A8F0
:10C51000FDF7E2FA94F82330052B7FF412AB6AE5BD
:10C52000D8F8041004220B68CDE90102B84A009241
:10C53000D3F800A05A461C2309A8D047D0E7D4F866
:10C54000083313F0200A24D15FFA85FB1E225946D6
:10C550002046FEF7C7FE064608B3CDE908AA00222A
:10C56000099B0B9311460BA8CDE9092203F0F2FBBE
:10C5700001462046FEF7A6FE0BA8FDF763FA0AA8BF
:10C58000FDF760FA09A8FDF7A7FA16B108A8FDF7AC
:10C59000A3FA94F82330052B7FF4E4AA2BE5D8F80E
:10C5A000041004220B68CDE90102994A0092D3F8E5
:10C5B00000A05A461E2309A8D047D0E7D4F8083374
:10C5C00013F0200A25D15FFA85FB1C22594620462C
:10C5D000FEF788FE064610B3CDE908AA099A0B9229
:10C5E0000023022201210BA8CDE9093303F0B2FB9D
:10C5F00001462046FEF766FE0BA8FDF723FA0AA8BF
:10C60000FDF720FA09A8FDF767FA16B108A8FDF7AB
:10C6100063FA94F82330052B7FF4B5AAEBE4D8F83D
:10C62000041004220B68CDE90102794A0092D3F884
:10C6300000A05A461C2309A8D047CFE7D4F80833F6
:10C6400013F0200A25D15FFA85FB1E2259462046A9
:10C65000FEF748FE064610B3CDE908AA099A0B92E8
:10C660000023022201210BA8CDE9093303F072FB5C
:10C6700001462046FEF726FE0BA8FDF7E3F90AA8BF
:10C68000FDF7E0F909A8FDF727FA16B108A8FDF7AC
:10C6900023FA94F82330052B7FF486AAABE4D8F86C
:10C6A000041004220B68CDE90102594A0092D3F824
:10C6B00000A05A461E2309A8D047CFE7D4F8083374
:10C6C00013F0400A21D15FFA85FB0C22594620461F
:10C6D000FEF708FE0646F0B1CDE909AA0A9B002242
:10C6E000CDE90A23012106220BA800F047FD0146EF
:10C6F0002046FEF7E7FD0BA8FDF7EEF90AA8FDF7C7
:10C70000EBF916B109A8FDF7E7F994F82330052BEA
:10C710007FF45BAA6FE4D8F8041004220B68CDE91B
:10C7200001023B4A0092D3F800A05A460C230AA803
:10C73000D047D3E7D4F8083313F0400A20D15FFA8A
:10C7400085FB0C2259462046FEF7CCFD0646E8B193
:10C75000CDE909AA00220A9B11460BA8CDE90A23BC
:10C7600000F00CFD01462046FEF7ACFD0BA8FDF7DE
:10C77000B3F90AA8FDF7B0F916B109A8FDF7ACF9AD
:10C7800094F82330052B7FF431AA34E4D8F8041050
:10C7900004220B68CDE901021D4A0092D3F800A0E3
:10C7A0005A460C230AA8D047D4E7D4F8083313F02C
:10C7B000800A26D13B78F1B21A462046CDE904130F
:10C7C000FEF790FDDDE90413814618B3CDE909AA0F
:10C7D0000A9B0022CDE90A2301210C220BA803F0B9
:10C7E00087F901462046FEF76DFD0BA8FDF774F9A9
:10C7F0000AA8FDF771F9B9F1000F02D009A8FDF7F9
:10C800006BF994F82330052B7FF404AAFFF7F3BBF0
:10C81000801A0600D8F80400B84AD0F800E0009268
:10C820004FF0040CCDE9019C0A46DEF800A0014659
:10C830000AA8D047CCE7D4F8083313F0800A26D1F1
:10C840003B78F1B21A462046CDE90413FEF74AFDC3
:10C85000DDE90413814608B3CDE909AA0A9B002249
:10C86000CDE90A2300210C220BA803F041F901466F
:10C870002046FEF727FD0BA8FDF72EF90AA8FDF7C5
:10C880002BF9B9F1000F02D009A8FDF725F994F8AA
:10C890002330052B7FF4CEA9FFF7ADBBD8F80400F9
:10C8A000964AD0F800E000924FF0040CCDE9019CCC
:10C8B0000A46DEF800A001460AA8D047CEE7D4F821
:10C8C000083313F4004A20D15FFA85FB0C22594645
:10C8D0002046FEF707FD0646F0B1CDE909AA0A9BFE
:10C8E000002201210BA8CDE90A2302F077FF0146BF
:10C8F0002046FEF7E7FC0BA8FDF7EEF80AA8FDF7C7
:10C90000EBF816B109A8FDF7E7F894F82330052BEA
:10C910007FF4A6A9FFF76FBBD8F8041004220B68B8
:10C92000CDE90102754A0092D3F800A05A460C23C3
:10C930000AA8D047D3E7D4F8083313F4004A20D12B
:10C940005FFA85FB0C2259462046FEF7CBFC0646D3
:10C95000F0B1CDE909AA00220A9B11460BA8CDE946
:10C960000A2302F03BFF01462046FEF7ABFC0BA872
:10C97000FDF7B2F80AA8FDF7AFF816B109A8FDF760
:10C98000ABF894F82330052B7FF47BA9FFF733BB7A
:10C99000D8F8041004220B68CDE90102574A00922E
:10C9A000D3F800A05A460C230AA8D047D3E7D4F8FE
:10C9B000083313F4007A20D15FFA85FB3022594600
:10C9C0002046FEF78FFC0646F0B1CDE909AA0A9B86
:10C9D000002201210BA8CDE90A2303F087FC0146C0
:10C9E0002046FEF76FFC0BA8FDF776F80AA8FDF7C6
:10C9F00073F816B109A8FDF76FF894F82330052BEA
:10CA00007FF450A9FFF7F7BAD8F8041004220B6896
:10CA1000CDE90102394A0092D3F800A05A463023EA
:10CA20000AA8D047D3E7D4F8083313F4007A20D10A
:10CA30005FFA85FB302259462046FEF753FC064636
:10CA4000F0B1CDE909AA00220A9B11460BA8CDE955
:10CA50000A2303F04BFC01462046FEF733FC0BA8EB
:10CA6000FDF73AF80AA8FDF737F816B109A8FDF75F
:10CA700033F894F82330052B7FF425A9FFF7BBBAD0
:10CA8000D8F8041004220B68CDE901021B4A009279
:10CA9000D3F800A05A4630230AA8D047D3E7D8F8E5
:10CAA000041004200A68CDE9016014480090D2F80F
:10CAB00000A009A84A46D047FFF736B9D8F80410B5
:10CAC00004200A68CDE901600C480090D2F800A06B
:10CAD00009A84A46D047FFF76FB9D8F804100422D6
:10CAE0000B68CDE90102054A0092D3F800B04A462E
:10CAF0002B460AA8D847FFF7A3B900BF801A060043
:10CB0000D8F8041004220B68CDE901020C4A009207
:10CB1000D3F800B04A462B4609A8D847FFF7D1B949
:10CB2000D8F8041004220B68CDE90102044A0092EF
:10CB3000D3F800B04A462B4609A8D847FFF705BAF4
:10CB4000801A060073B50446FEF77EFF94F8233082
:10CB5000052B32D0002594F83F33EB40DA07E9B2D9
:10CB600016D40135082DF6D194F82330052B24D0A6
:10CB700094F8203013B194F82230F3B9104B1149D6
:10CB80001B68986903681B6802B0BDE870401847CD
:10CB9000D4F808339B030CD42C200191FEF7D6F96E
:10CBA000064610B1019903F019FC31462046FEF704
:10CBB00089FB94F82330052BD3D102B070BD00BFA0
:10CBC0004061002084860A082DE9F04F90F9213059
:10CBD00089B00446002B00F00481012300F50C7598
:10CBE00080F84133024600F50F712B462E46D06E79
:10CBF000002859D0002384F8413394F94030642B45
:10CC00005BD094F9BC30642B00F08D8094F93831FE
:10CC1000642B00F08A80D4F830722FBB01A9204623
:10CC20002BF00EFF00B30C230593012306978DF81C
:10CC30001830714B07936946BDF80430049704A877
:10CC4000ADF810308DF800702CF07AF89DF90010D6
:10CC500051B1022908DC38B1C9B27C2303FB014180
:10CC60006C3128462DF044FC94F841B3BBF1000F21
:10CC70005DD0E36E6367D4F8E830C4F8F030D4F8E0
:10CC80006431C4F86C3194F8233003F1C30204EB2F
:10CC900082020021042B7CD852F8040B106101336E
:10CCA00042F8041CDBB2F5E753F8040B0028A1D1CD
:10CCB0008B4202F17C029AD19FE7002066238DF817
:10CCC00010307C2303FB004004A940302DF054FBBE
:10CCD00004A920462BF0B4FE00289CD004238DF834
:10CCE00018300023CDE901330393312305936946BE
:10CCF00004A82CF025F8059B28B108AA02EB8302B2
:10CD0000009942F8E01C0133332B0593EFD952F020
:10CD100023FD9DED031ADDED020A9DED010A66215A
:10CD200052F0D8FC77E70120C8E70220C6E70127C8
:10CD3000A94655F8043B23B1AB600137042FF7D166
:10CD400097E7AA46B8465FFA88F3022BF5D8DAF8D7
:10CD5000002055F8043C9A4205D104A95046CDF86C
:10CD600010B02DF0C5FB5AF8043B08F101020BB9D5
:10CD70009046E8E704A906EB88000193CDF810B0CF
:10CD80002DF0B6FB019BAB6001A948462DF0B0FB2E
:10CD9000D3E794F8413313B92046FEF79FF994F88E
:10CDA00022300BB3154B1B68986A036864215B68DB
:10CDB00098472046FEF752FD94F83E3003B9E366EB
:10CDC00094F8BA300BB9C4F8E83094F836310BB99E
:10CDD000C4F86431FAF7C8F9FAF792FA0123A4F813
:10CDE000403309B0BDE8F08F2046FFF7ABFE94F862
:10CDF0002230002BE0D0D5E75C230B0840610020F7
:10CE00007047000001207047012070474368986810
:10CE10007047000010B5054B03600446806A10B1EE
:10CE200003685B689847204610BD00BF448B0A0822
:10CE3000406803685B6A184733B46C46406884E80E
:10CE40000C0003689D6A94E80C00AC4602B030BC4C
:10CE50006047000010B50446FFF7DCFF2046FEF7F0
:10CE60007DF8204610BD000040680BF003BA0000BA
:10CE7000406801230BF0FEB940680BF0D7B9000001
:10CE800040680A220BF07CB940680BF091B90000B1
:10CE900040680BF013BA000090F82E2022B190F8F1
:10CEA0002D10002201F06EB97047000073B50446E2
:10CEB00005250026A06A8DF8076003680DF10702BA
:10CEC000DB680121984778B19DF807300C2B09D019
:10CED000102B05D0092B07D184F8303002B070BD7B
:10CEE0001523F9E71423F7E7013DE3D12846F5E7D9
:10CEF00010B4806A03681C690822A44601235DF807
:10CF0000044B31216047000010B4806A03681C693B
:10CF10000122A44600235DF8044B32216047000043
:10CF2000F0B50446806A036885B05B69984705469A
:10CF3000002800F08480A06A03685B699847036852
:10CF40009B689847A06A03689B69984760B93D4B06
:10CF50003D491B68986903681B6898472B682846F9
:10CF6000DB689847002667E02046FFF7CDFF0028E2
:10CF7000F4D02046FFF79AFF0028EFD0A06A03689C
:10CF80000121DB6A98472046FFF7B2FF30B92D4BED
:10CF90002E491B68986903681B68DEE7A06A03686E
:10CFA000DB69984730B9274B29491B6898690368A2
:10CFB0001B68D2E7A06A94F83010012784F82E701D
:10CFC00003685B6A9847A06A03689B6A984704F104
:10CFD0002D020146204601F023F906460028BDD067
:10CFE000A06A94F82D10036801919B6A98470199F3
:10CFF0000246204601F018F994F82C302BB194F831
:10D000002D103A46204601F023F994F82F2094F889
:10D010002D10204601F03EF92B682846DB68984722
:10D02000A06A029403681D6A0A4B039304AB13E9D8
:10D030000C0042F21071A847304605B0F0BD06461C
:10D04000FAE700BF40610020B08A0A08D68A0A08C1
:10D05000F58A0A084DD1010870B5002586B0CDE9E2
:10D06000005500230446806A8DF808500593039309
:10D07000049303686A469E6810210923B047A0B153
:10D080009DF8003013F0010615D194F831300133CA
:10D09000DBB2052B84F8313007D12046FFF734FF8F
:10D0A0002046FFF725FF84F83160A06A03681B6BF8
:10D0B000984706B070BD9DF8083084F831501B07C2
:10D0C000F3D4BDF901309FED1F6A06EE903ABDF929
:10D0D000033007EE103ABDF90530F8EEE66A07EEC8
:10D0E000903ACDED036AF0EEE66AB8EEC77AF8EE54
:10D0F000E77AF4EEC66AF1EE10FA8DED047ACDED22
:10D10000057A0DD5B0EEC77AB4EEC67AF1EE10FA14
:10D1100006D5F0EEE77AF4EEC67AF1EE10FAC4D452
:10D120009FED090A03A811F059FCB2EE040A03A806
:10D1300011F054FC94F82D200A2303A9204601F095
:10D140000FF9B2E7000000349A99193EFFF784BF47
:10D1500010B5044B044640F8043BFCF7BDFC2046E8
:10D1600010BD00BF5C8B0A0810B50446FFF7F0FF46
:10D170002046FDF7F3FE204610BD0000F7B503681A
:10D180000F4616461BB90024204603B0F0BD00240C
:10D19000046008200193FDF7D9FE054620B1124B2B
:10D1A0000360019B4360019401A8FCF795FC002DEE
:10D1B000E9D03420FDF7CAFE04460028E3D000F091
:10D1C000E1FE0A4BA562236084F82C7084F82F607E
:10D1D0002046FFF7A5FE05460028D5D12368204646
:10D1E0005B6898472C46CFE75C8B0A08448B0A089B
:10D1F0002DE9F74F046806460D4690469946002CE7
:10D200006CD00B68002B49D0236820465B6A984796
:10D2100003689B689847012328680DEB03020021EF
:10D220000BF028F898B39DF80130EA2B2FD1DFF8E6
:10D23000F0B04FF0060A28680023802206210AF089
:10D24000F5FF20B3DBF80070B86A03680A215B6859
:10D250009847002328681A4606210AF0E7FFB0B174
:10D26000B86A03680A215B689847012328680DEBB8
:10D27000030206210AF0FEFF48B19DF8014014F0B8
:10D2800040042FD00AF1FF3A1AF0FF0AD3D13068D8
:10D2900003685B6A98470368DB68984700241DE0D1
:10D2A000022223460F2128680AF0C0FFB86A0368EB
:10D2B00001215B689847306803685B6A9847036898
:10D2C000DB689847336834604A46414601A80193B9
:10D2D000FFF754FF044601A8FCF7FEFB204603B00D
:10D2E000BDE8F08F224623460F2128680AF09EFFF2
:10D2F000B86A036801215B689847022321463068B9
:10D300000DEB03020AF0B6FF04460028C8D0B86946
:10D31000024903681B689847B9E700BF1C8B0A08DD
:10D320004061002090F82C10002200F02BBF00007C
:10D3300070B504468CB00426013E76B2731C4AD008
:10D34000A06A15236A465D210AF094FF0028F3D0F5
:10D35000A06A152306AA5D210AF08CFF0546002865
:10D36000EAD0152206A9684681F006FC0028E3D120
:10D370009DF8003084F82E309DF8073084F8303066
:10D380009DF8143084F83A309DF813309DF8102041
:10D3900084F83B309DF80F3043EA0223A3879DF8C1
:10D3A000013084F82F309DF8083084F83130039B29
:10D3B0009DF80C20C3F30F2363869DF80B3043EADE
:10D3C0000223A386049BC3F30F23E386019BC3F3CD
:10D3D0000F23238707E0054B05491B6898690368FD
:10D3E0001B689847002528460CB070BD406100209E
:10D3F000908B0A082DE9FF4104460023806A8DF8CE
:10D4000007300368DFF868815B6A984703689B68A8
:10D410009847A06A03680A219B6C9847A06A0A2271
:10D4200004210AF0ADFE0425013D6DB26B1C32D023
:10D4300000234B21A06A82220AF0F8FED8F800608F
:10D440000746B06A036802215B689847002FEBD05B
:10D4500001231A464B21A06A0AF0E8FE0746B06A8B
:10D46000036802215B689847002FDDD0A06A012382
:10D470000DF1070240210AF0FDFE0028D4D09DF8EE
:10D480000720322A10D0002DCED1B069364903686A
:10D490001D683223A847A06A03685B6A984703683F
:10D4A000DB68984700255BE02046FFF741FF002836
:10D4B000F1D0A06A0123172251210AF0B7FE0028FB
:10D4C000E9D05222A06A012311460AF0AFFE0028DB
:10D4D000E1D0A06A012338224C210AF0A7FE0028DF
:10D4E000D9D0A06A03685B6A98470368DB689847ED
:10D4F000A06A05210AF05CFEA36A04F12C02996877
:10D50000204600F08DFE054650B3A36A94F82C1017
:10D510009A68204600F088FE94F8442094F82C1075
:10D52000204600F0B7FE94F845302BB194F82C104B
:10D530000122204600F08CFEA06A036802219B6C49
:10D540009847A06A029403689E6A084B039304AB51
:10D5500013E90C0044F21B11B04755F091F8206418
:10D56000284604B0BDE8F081B88B0A08DDD6010872
:10D570004061002070B5858F90F93B60AD03B5FB2D
:10D58000F2F2A2F5804404FB04F2D51190F83A209F
:10D590000498D201624306FB05225212A03002F524
:10D5A0008012424312134A43DB0003EB623000B2A5
:10D5B00070BD000010B5448E53005C43B0F93830A4
:10D5C000C91A838FD31AB0F93620B0F93400534307
:10D5D00004F500449B10C3EBC13300EB2440044925
:10D5E00093FBF0F04FF400420FF08EF800B210BD44
:10D5F0000080FFFF10B52DED028B8AB00446082392
:10D60000806A05AA42210AF035FE18B1BDF81A2039
:10D61000D30719D4A06A0AF051FE55F031F8236CF3
:10D62000C31AFA2B0CD92064002382224B21A06A52
:10D630000AF0FCFD0123A06A1A464B210AF0F6FD10
:10D640000AB0BDEC028B10BDBDF9141094F9303056
:10D650000093920894F92E300392C9102046FFF7E8
:10D6600089FFBDF9161094F93130039A009308EE42
:10D67000900A94F92F30C9102046FFF77BFFBDF9BF
:10D680001810039A491008EE100A2046FFF792FF7F
:10D6900007EE900AF8EEE88AF8EEE77AB8EEC88A64
:10D6A000B3EE000A07A8CDED097ACDED078A8DED1E
:10D6B000088A11F0A7F9B2EE040A07A811F08EF952
:10D6C00054F0DEFF94F82C2020640A23204607A99A
:10D6D00000F046FEA06A0AF0F1FDB1E7FFF78ABF4D
:10D6E000F7B503680D4616461BB90024204603B063
:10D6F000F0BD002707604820CDE90073FDF726FC48
:10D70000044650B100F03EFC0E4B2360019BA36227
:10D71000019784F8446084F8455001A8FCF792F919
:10D720006846FCF78FF9002CDFD02046FFF762FE39
:10D7300005460028DAD1236820465B6898472C46C6
:10D74000D4E700BFF08B0A0810B5044B044640F83C
:10D75000283BFCF777F9204610BD00BFF08B0A0884
:10D7600010B50446FFF7F0FF2046FDF7F7FB204613
:10D7700010BD000090F82C10002200F003BD000046
:10D78000F8B504460D4617461E4600F0FBFB094B54
:10D7900023602B68A362002200232A6084F82D7086
:10D7A00084F82E6023656365A365E365236663667D
:10D7B0002046F8BD088C0A08F8B51C460933164601
:10D7C000DB086A46A2EBC30300AF9D46806AA31C38
:10D7D0006A460AF04FFD054628B122460DF10201C6
:10D7E000304681F0D9F92846BD46F8BD2DE9F34110
:10D7F00006460F46144654F043FF114BD3F8008001
:10D800000546D8F82800036801215B689847012382
:10D810000DF1070207213046FFF7CEFF60B19DF8FA
:10D820000730DA0702D4B7EB531F05D054F028FFB6
:10D83000431BA342E5D3002002B0BDE8F08100BF46
:10D84000406100202DE9F041DFF8608292B004468B
:10D8500002AF002646F02002A06A0023D2B2502177
:10D860000AF0E4FC002800F00C810325013D6DB2B4
:10D870006A1C00F00681D8F80030986A03684FF4FB
:10D8800096719B68984701230DF1060255212046A9
:10D89000FFF792FF002800F0F4809DF8063013F0A7
:10D8A000E00F40F0EE80DB07E0D502230DF1060229
:10D8B00052212046FFF780FF002800F0E280BDF8EB
:10D8C000063001365BBA202E27F8023BC2D1BDF8E4
:10D8D00024309DF826109FED6D7ADFED6D6A9FED87
:10D8E0006D6A43F30B0207EE902A1B0903F4706381
:10D8F000BDF82620F8EEE77A0B4343F30B03C4EDA3
:10D900000C7A07EE903A02F470639DF82820F8EE46
:10D91000E77A134343F30B03C4ED0D7A07EE903A15
:10D920009DF92230F8EEE77AC4ED0E7A07EE903AD0
:10D930009DF92930F8EEE77A67EE877A07EE103A1C
:10D94000B8EEC77A9DF92A30C4ED0F7A27EE267A11
:10D95000DFED517A84ED107A07EE103AB8EEC77A0F
:10D960009DF92B30E7EE267AC4ED117A07EE903A56
:10D97000F8EEE77A9DF9233067EEA67ADFED476A85
:10D98000C4ED127A07EE903A9DF92C3007EE103A6A
:10D99000B8EEC77A9DF92E3027EE267AF8EEE77AB0
:10D9A00084ED147A67EE867A07EE103A9DF93030EE
:10D9B000C4ED137A07EE903AF8EEE77A9DF92D3030
:10D9C00067EEA67AB8EEC77AC4ED167A27EE267A05
:10D9D00007EE903A84ED157AF8EEE77A9FED307A0B
:10D9E0009DF92F3067EE877AC4ED177A07EE903AEB
:10D9F0009DF93130F8EEE77A06EE903A67EE877AD5
:10DA0000F8EEE66AC4ED187ADFED267ABDF9383013
:10DA1000E6EE877A07EE103A9DF93230C4ED197AB6
:10DA2000B8EEC77AF3EE077AE7EE067A07EE103A19
:10DA3000DFED1D6AC4ED1A7AB8EEC77A27EE267AB2
:10DA400084ED1B7A9DF9333007EE103AB8EEC77AB1
:10DA50009DF9343027EE267A84ED1C7A07EE103AD1
:10DA60009DF9353007EE903AB8EEC77AF8EEE77ACE
:10DA700027EE267A67EEA67A84ED1D7AC4ED1E7A2B
:10DA800000E0002012B0BDE8F08100BFCDCC4C3EDC
:10DA90000000803B0000003B0AD7233C0000003D13
:10DAA0000000803817B7D1B80AD7A33A40610020E8
:10DAB00073B501230E460DF1070206210446FFF758
:10DAC0007BFE18B90025284602B070BD9DF80730CE
:10DAD000013B012B0CD80023A06A1A4606210AF04C
:10DAE000A5FB0028EED0062200212046FFF77EFE8F
:10DAF000A06A0023324606210AF098FB054600285A
:10DB0000E0D0262231462046FFF770FEDBE700001A
:10DB100013B501230DF1070207210446FFF74CFE60
:10DB200010B9002002B010BD9DF807301B070CD5BE
:10DB30000023A06A1A4606210AF078FB0028F0D0DC
:10DB4000062200212046FFF751FEA06A002307228B
:10DB500006210AF06BFB0028E3D0132207212046A0
:10DB6000FFF744FE0028DCD0A06A0023052206212E
:10DB70000AF05CFB0028D4D0172205212046FFF7CD
:10DB800035FE0028CDD001212046FFF791FFC9E7DF
:10DB9000F7B50446806A5B4F03685B6A9847036881
:10DBA0009B689847A06A03680A219B6C9847A06A03
:10DBB0000A2204210AF0E4FA0525013D6DB26B1C2E
:10DBC00000F09680A06A0023B6227E210AF02EFB88
:10DBD0000028F2D03B68986A036818215B686E469B
:10DBE00098470123324600212046FFF7E5FD002833
:10DBF000E3D09DF80030332BDFD12046FFF722FE23
:10DC0000002875D0A06A0023802250210AF00EFB64
:10DC100000286DD02046FFF77BFF002868D0A06A5F
:10DC2000002386222E210AF001FB002860D0A06A82
:10DC30000023242204210AF0F9FA002858D0A06A0F
:10DC40000023022206210AF0F1FA002850D0142203
:10DC500002212046FFF7CAFDA06A00230722052102
:10DC60000AF0E4FA002843D001212046FFF720FF04
:10DC700000283DD0A06A036803219B6C9847A06AE6
:10DC800003685B6A98470368DB689847A06A1721B6
:10DC90000AF08EFAA36A04F12C029968204600F07B
:10DCA000BFFA054608B3A36A94F82C109A68204678
:10DCB00000F0BAFA94F82E2094F82C10204600F0C8
:10DCC000E9FA94F82D302BB194F82C10012220465B
:10DCD00000F0BEFAA06A03689F6A0B4B00940193A0
:10DCE00096E80C0042F21071B847284603B0F0BD28
:10DCF000A06A03685B6A98470368DB689847002559
:10DD0000F3E700BF4061002001DF010810B586B0D5
:10DD10000C236A4631210446FFF74EFD002800F02F
:10DD2000DF809DF801309DF80020DFED717ADFED96
:10DD3000715A1B0403EB02239DF8022003EB0263DC
:10DD40001B1206EE903A9DF804309DF803201B0448
:10DD500003EB02239DF8052003EB02631B1207EE81
:10DD6000103A9DF807309DF806201B0403EB0223B0
:10DD70009DF8082003EB02631B1206EE103A9DF893
:10DD80000A309DF809201B0403EB0223F8EEE66A33
:10DD9000B8EEC77A9DF80B2066EEA76A27EE277AC1
:10DDA000B8EEC66ADFED547A03EB02631B1226EE6F
:10DDB000276A07EE903AF8EEE77A67EEA57AF5EE75
:10DDC000C07AF1EE10FA40F38D80DFED4C5A77EE19
:10DDD000E57AD4ED134A94ED0F5A94ED1C4AD4ED34
:10DDE0001D3A94F82C20F7EE005A74EEA54AF0EE96
:10DDF000632AA4EEA75A0A2303A9D4ED107AD4ED1E
:10DE00000C4A77EEA57A2046E7EEA64AD4ED1A7AB8
:10DE100075EE677A94ED145AF0EE646AD4ED174A01
:10DE2000E5EE276AB0EE655AA7EEA45AC6EE854A1B
:10DE300094ED115AD4ED0D6A35EE255AE5EE076AD8
:10DE400094ED157AE7EE876A94ED187AB0EE655A8C
:10DE5000A7EE875A86EE857A94ED125AD4ED0E6AB3
:10DE600035EE255AE5EE066A94ED166A94ED195AD8
:10DE7000E7EE866AB0EE656AA7EE856AF0EE657A2F
:10DE800086EE863A94ED1B6AF0EE646AE6EE447A1A
:10DE9000E6EE476A86EEA75AF0EE476AE4EE646A59
:10DEA000C6EEA75AD4ED1E6AD4EE262AE6EE636AC1
:10DEB000B2EE046A27EE667A65EE066AA2EEA47AEE
:10DEC000CDED036A65EE866ACDED046AC7EE276A7A
:10DED00076EE837A67EE867ACDED057A00F040FA29
:10DEE00006B010BD44BFDFED055A77EEA57A70E7A6
:10DEF00047ABE73B5B9E803AF61BEB3B85EBCB41A8
:10DF0000FFF704BF30B51346026885B00D461AB955
:10DF10000024204605B030BD002101607C20019323
:10DF20000392FDF713F8044620B1019B2A4603A98A
:10DF3000FFF726FC03A8FBF785FD002CE8D0204660
:10DF4000FFF726FE05460028E3D1236820465B68DC
:10DF500098472C46DDE7000010B5044B044640F816
:10DF6000283BFBF76FFD204610BD00BF088C0A0858
:10DF700010B50446FFF7F0FF2046FCF7EFFF204600
:10DF800010BD0000064B10B503600446FDF756FDBA
:10DF9000606004F1080053F043FA204610BD00BF52
:10DFA000208C0A0873B50646144675687C2303FB6B
:10DFB0000253C4EB441405EB8404084693F8A41000
:10DFC000019010F0A1FD94F93C3001983BB97368C1
:10DFD00093F8251002B0BDE8704010F095BD94F89C
:10DFE0004010F7E737B5446801917C2505FB0245F1
:10DFF00095F83F3004EB8304D4F84C325BB154F015
:10E000003FFBC5F89C000199D4F84C0203B0BDE871
:10E01000304003F0A7BF03B030BD00002DE9F04F42
:10E02000C2EB421447684FEA840881460E4607F166
:10E030003C0B08F108018BB015465944304610F0EE
:10E0400099FCD9F8040029460BEB8404FDF79CFCED
:10E0500038B17C2303FB057393ED1A0A304610F0A8
:10E06000BDFC7C2303FB057393ED146ADFED3A7A64
:10E07000D3ED156AB0EEC67AB4EEE77AF1EE10FA97
:10E080000FD5B0EEE67AB4EEE77AF1EE10FA08D5E5
:10E0900094ED077AB0EEC77AB4EEE77AF1EE10FAB3
:10E0A0001BD47C2303FB0573D86D196E5A6E9B6DD0
:10E0B000029003910490079101A831468DED016A09
:10E0C000CDED056A0692089209930EF01BFD86EDD0
:10E0D000000AC6ED010A86ED021A7C2303FB0577D0
:10E0E0000023C7F88C30C7F88830C7F88430D9F8D7
:10E0F000040090F95C3208F13C0A08F14808DA445F
:10E10000D84463B15DB9414600F5167004F0E2FBF6
:10E11000414630460BB0BDE8F04F10F02BBC90F9F3
:10E120003430012B0BD190ED0E0A504610F002FC5A
:10E1300084ED120AC4ED130A84ED141AE8E7022BE9
:10E14000E6D1FCF7E7FA002201A9FBF7B1FF0028AE
:10E15000DED09DED010AE8E70000003410B5436809
:10E160007C2404FB023407C904F1900383E8070010
:10E1700054F086FAC4F89C0054F076FAC4F8A00073
:10E1800010BD0000F0B5074685B00D46164600F1FB
:10E190000801A92203A80AF0C7FA7C687C2303FBC4
:10E1A0000543D3F8B42022B903A80AF0DFFA05B07A
:10E1B000F0BDBEB196ED007AD3ED2A7A67EE877A8C
:10E1C000C3ED2A7A96ED017AD3ED2B7A67EE877A42
:10E1D000C3ED2B7A96ED027AD3ED2C7A67EE877A2F
:10E1E000C3ED2C7A7C2607EE902A06FB0541A83168
:10E1F000B8EE670A0846019110F004FC01992A461E
:10E200003846FFF7ABFF06FB05410023C1F8B030ED
:10E21000C1F8AC30C1F8A8300023C1F8B430C3E76E
:10E220004068FCF7ABBF0000F7B5064640680192B6
:10E230007C2707FB01000D466C3001A914462CF029
:10E2400037F9716807FB05152C6703B0F0BD0000B6
:10E2500007B540687C2303FB010393F93C30022B94
:10E260000BD000F13C03C1EB411003EB80000DF13A
:10E2700007018DF807202CF075F803B05DF804FB5A
:10E2800043687C2202FB013191F93C00003818BF41
:10E290000120704743687C2000FB013181F8A420F5
:10E2A00070470000F8B5054608460F4610F008FC18
:10E2B00010B100242046F8BD384610F0E7FB0446B4
:10E2C0000028F6D16B6893F934637EB1384610F0BC
:10E2D0002FFF95ED087ADFED1F7AF0EEC76AF4EEB6
:10E2E000E76AF1EE10FA03D585ED080A0124E1E7AB
:10E2F00077EE407A30EE076AF0EEE77AC7EE866A8C
:10E30000F6B207EE906A9FED146AF8EE677A26EE91
:10E31000866AF4EEC67AF1EE10FA48BFB2EE046AED
:10E32000DFED0E7A45BF6B6A66EE866AB0EE676A0D
:10E3300087EEA66A46BF01336B620124F7EE007ACE
:10E3400077EEC67A20EE060AA7EE270A85ED080AC0
:10E35000B0E700BF0000003400004843CDCCCC3D06
:10E360002DE9F74304460E4615461F46FFF71AFEF1
:10E370002A4631462046FFF735FE314620462A46DA
:10E38000FFF74CFE31462046FFF78CFF28B39B2257
:10E3900004F1080101A80AF0C7F964684FF07C098C
:10E3A00009FB054808F1A8083146404610F0E2FA9A
:10E3B00009FB0542D2F8B4100131C2F8B4104FB1D4
:10E3C000B94207D34908C2F8B410B0EE000A40467B
:10E3D00010F018FB01A80AF0C9F903B0BDE8F083FA
:10E3E00010B50446FCF754FFC0B23C34C0EB4010FB
